:020000040800F2
:100000000050002059A900089FA90008A1A90008D4
:10001000A3A90008A5A90008A7A9000800000000DE
:10002000000000000000000000000000A9A9000876
:10003000ABA9000800000000ADA90008050A0008EF
:10004000B3A90008B5A90008B7A90008B9A9000814
:10005000BBA90008BDA90008BFA90008C1A90008E4
:10006000C3A90008C5A90008C7A90008C9A90008B4
:10007000C1990008CDA90008CFA90008D1A900089E
:10008000D3A90008D5A90008D7A90008D9A9000854
:10009000DBA90008DDA90008DFA90008E1A9000824
:1000A000E3A90008E5A90008E7A90008E9A90008F4
:1000B0002D760008EDA90008EFA90008F1A90008B5
:1000C000F3A90008F5A90008F7A90008F9A9000894
:1000D000FBA9000899740008C938000801AA0008A3
:1000E00003AA000805AA000807AA000810B5054CD5
:1000F000237833B9044B13B10448AFF300800123D4
:10010000237010BDA80200200000000088FA00083B
:1001100008B5064B1BB106480649AFF300800648F8
:10012000036813B1054B03B1984708BD00000000F8
:1001300088FA0008AC020020A8020020000000009D
:10014000154B002B08BF134B9D46A3F5803A0021A9
:100150008B460F461348144A121A0AF084FD0F4BBF
:10016000002B00D098470E4B002B00D09847002062
:10017000002104000D000D48002802D00C48AFF308
:1001800000800AF023FD2000290007F07FFB0AF021
:1001900009FD00BF00000800005000200000000022
:1001A00000000000A8020020143A00200000000017
:1001B0000000000070B5354D86B02C681CB10123DD
:1001C0002B6006B070BD684609F0D4FF01A809F0A5
:1001D000DBFD4FF400400AF02DF9112001210AF057
:1001E00095F94FF400602023C4F201006946ADF890
:1001F00000308DF8034009F059FF4FF400700121E1
:100200000AF084F94FF4105001264FF46023C4F231
:10021000010001A9039301948DF808408DF809406D
:1002200004948DF8146009F089FD4FF41050C4F265
:10023000010005213246234609F0D8FD4FF4105045
:10024000C4F20100314609F0A9FD4FF41050C4F288
:10025000010009F0ADFD4FF41050C4F2010009F0A7
:10026000ADFD0028F7D14FF41050C4F2010009F0A1
:10027000A9FD4FF41050C4F2010009F0A9FD0028B7
:10028000F7D1034B01221A6099E700BFC802002092
:10029000783800204FF4105008B5C4F20100012155
:1002A00009F09AFD40F2C423C2F2000301221A6051
:1002B00008BD00BF38B50D4C054623680BB90020BA
:1002C00038BD4FF41050C4F20100022109F0DEFDE8
:1002D0000028F4D04FF41050C4F2010009F0D2FD10
:1002E000002328802360012038BD00BFC402002005
:1002F00070B448F6396301EB4104951EC3F6E3037D
:100300000229C1EBC40183FB014348F21F54D8BF4B
:100310001546C5F2EB14D8BF013A84FB0264C91735
:10032000C1EB630128180818D51CD317043032EA32
:10033000220228BF2A46A3EB641100EBA202C3EB02
:10034000E413521842F29340D218C9F2492080FBBC
:100350000230D3178018C3EBA000C0EBC000101A06
:1003600070BC704770B40646002922D00078F0B106
:1003700000231846F25CA2F13004E4B2092CA2F189
:1003800041050DD9052DA2F161049CBFA2F13704EE
:10039000E4B205D9052C9ABFA2F15704E4B20024B7
:1003A0000133DDB204EB0010A94280B2E2D870BC88
:1003B00070470846FBE700BF4FF48050C4F20100CD
:1003C0004FF40051002209F0E3BE00BF4FF480500B
:1003D000C4F201004FF40051012209F0D9BE00BF60
:1003E00000B583B001A809F0C5FE102001210AF074
:1003F0008DF84FF40053ADF804304FF480500223D1
:10040000C4F2010001A98DF8063010238DF80730E1
:1004100009F04CFEFFF7DAFF03B000BD00B583B072
:1004200001A809F0A7FE042001210AF06FF840237B
:100430004FF40060ADF80430C4F20100482301A974
:100440008DF8073009F032FE03B000BD4FF40060B4
:10045000402108B5C4F2010009F094FED0F101007A
:1004600038BF002008BD00BFF0B4114A0346106831
:10047000D8B110490E68104964360D680F49013D26
:100480000C680F495E610F680E491D610968DF60E5
:1004900099600D49096859600021072C08BF0C4676
:1004A0009C610F2419621C601160F0BC704700BF92
:1004B000F4020020CC02002008030020E00200200B
:1004C000D002002004030020DC02002070B582B0BE
:1004D00001A809F04FFE4FF44064082001210AF002
:1004E00015F8C4F201044FF4807301A902262046D6
:1004F000ADF8043004238DF807308DF8066009F05C
:10050000D5FD01A809F036FE0820012109F0FEFF03
:100510004FF40075204601A91023ADF804508DF862
:1005200006608DF8073009F0C1FD204629460122FA
:1005300009F02EFE02B070BDF8B5A44C2368FF2B65
:1005400056D04FF44060C4F201004FF4807109F0BE
:1005500019FE0546002833D0FFF72EFF236801203F
:10056000012B9A4D33D04AD3022B4DD0984B1A68A9
:10057000904200F08680974E022132682960911FD8
:100580001229186063D9052A94BF9348934806F04E
:100590004DFF934F934806F049FF002323603B68CB
:1005A0000F2B00F0CC81102B6ED0FF2B3AD00133F3
:1005B0003B2B3B6000F0CE8134D90023236031E037
:1005C000FFF704FF23682846012B804DCBD1804BD9
:1005D0001A68824229D01860002814BF0322022220
:1005E0007F4B2260FF221A607A4B00221A60F8BD0E
:1005F0007D4B1A68642A19D001321A60F8BD0123B4
:100600002B60734B1860F8BD714B1A68904238D05C
:10061000704E032132682960782A186012D9704B15
:1006200000221A6000233360F8BDF8BD4FF440602B
:10063000C4F201004FF40071002209F0A9FD00236B
:100640002360F8BD4A2AEDD800232B60EAE7644F07
:100650000F2A3B6834D8232B00F097813A2B00F007
:1006600085811C2B9CD1614A1268D0079FD56048B8
:1006700006F0DCFE5B4806F0D9FE002323603B68F1
:100680008EE7544B1A68B7E75A4A002313605A4A58
:100690001360564A1360594A1360594A1360594A05
:1006A0001360594A1360594A1360594A1360594AF2
:1006B0001360594A1360594A136011233B60B1E734
:1006C000A3F11102292A3FF66BAF01A151F822F0E4
:1006D00037090008A1050008A1050008A1050008C8
:1006E000310900082B090008250900081F09000826
:1006F00019090008130900080D090008FD08000881
:10070000F7080008F1080008EB080008E5080008F1
:10071000DF080008D9080008C9080008C308000855
:10072000BD080008B7080008B3080008AF080008B3
:10073000AB080008A50800089F08000899080008F1
:10074000930800088D08000887080008830800083F
:100750007F0800086D0800085B08000849080008C9
:100760003708000825080008BB070008A90700088B
:100770009707000879070008214A126812F001055E
:100780007FF415AF264806F051FE164806F04EFEDF
:1007900025603B6804E72149194A0D681068503507
:1007A00001300D601060FEE61C49154A0D681068A6
:1007B000283501300D601060F5E61849104A0D68C3
:1007C0001068143501300D601060ECE62000002048
:1007D000F0020020D80200200CBD00082CBD00084B
:1007E0001C00002040DF0008D40200200C03002081
:1007F0004CBD0008F4020020E4020020EC020020BE
:1008000000030020F8020020DC0200200403002086
:10081000E0020020D002002008030020CC020020CB
:1008200094BD00086549664A0D6810680A350130B4
:100830000D601060B7E66149614A0D6810680835BF
:1008400001300D601060AEE65C495D4A0D681068CD
:10085000043501300D601060A5E65849584A0D680E
:100860001068023501300D6010609CE65349544A0F
:100870000D681068013501300D60106093E6514934
:10088000D1E75049D8E74F494D4ADFE74D494C4A37
:10089000E5E74C494A4AEBE74B49494AD6E74A491A
:1008A000474ADCE74849464AE2E7484986E747497C
:1008B000B9E74649C0E74549414AC7E74349404A85
:1008C000CDE742493E4AD3E7414A126812F001059A
:1008D0007FF46DAE3F4856E73F493D4A6FE73E49DA
:1008E0003B4AA1E73C493A4AA7E73B49384AADE7CA
:1008F0003949374AB3E73849354AB9E7374A1268C0
:1009000012F001057FF453AE35483CE73549334AD0
:100910004CE73449314A52E73249304A84E7314999
:100920002E4A8AE72F492D4A90E72E492B4A96E70F
:100930002C492A4A9CE72C4A0121116033E62B4BB3
:100940001A6822B12A4A0121116000221A6010237C
:100950003B6067E6274B204A196812689142264996
:1009600022D0204800681A6008605BE6144A1268CA
:10097000D2077FF51CAE214806F058FD204806F04E
:1009800055FD00223B682A600AE6114A1268D10729
:100990007FF50DAE0F4806F049FD194806F046FDFB
:1009A00000232B603B68FBE50E480C6800680134AF
:1009B0008442D8D10D4C01252560D4E7CC0200201B
:1009C0000003002008030020E0020020D0020020E5
:1009D000EC02002070BD0008040300200C0300207E
:1009E0004CBD0008DC020020F8020020E4020020D8
:1009F000F4020020E8020020FC02002094BD000860
:100A000040DF0008034B1A6812B11A68013A1A60F5
:100A1000704700BF7C380020064B074A1B68012B3B
:100A20001EBF064B1B68B0FBF3F010601368002B71
:100A3000FCD17047100300207C38002028000020E3
:100A4000044B054A1B6803FB00F010601368002B81
:100A5000FCD17047240000207C380020084B4FF464
:100A60007A711B6810F1FF3001FB03F1054A06D3D0
:100A700011601368002BFCD110F1FF30F8D27047E1
:100A8000240000207C380020012810B423D0022844
:100A90002CD01C4B64221A601B4B0A221A6042F2B3
:100AA00010710320194A4EF210031468CEF20003AD
:100AB000B4FBF1F101394FF46D425960CEF20002FE
:100AC000F02182F8231000229A6007221A60104B4E
:100AD000186010BC70470B4B44F2402118600A4B61
:100AE0004FF47A721A60C0F20F01DBE7054B0A225D
:100AF0001A60054B48F2A06164221A60C0F201013D
:100B0000D0E700BF2800002024000020F4010020CE
:100B1000100300202DE9F00140F2941240F2581326
:100B200040F26011C2F20003C2F20001C2F2000200
:100B3000D2F8008093F800C05F789E780D784C78EA
:100B400040F2541040F26C0240F270038978C2F215
:100B50000002C2F20003C2F20000C0F8008082F876
:100B600000C0577096701D705C709970BDE8F00100
:100B7000704700BF40F2211008F030BF40F25D1016
:100B800008F02CBFF8B506460F4640F2211440F29B
:100B90005D1520463146013408F0A6FFAC42F8D17D
:100BA00007B9F8BDBDE8F840FFF7E8BF70B540F2FF
:100BB0007002C2F200029578147856784CF2B8139D
:100BC000C0F6000382B033F8144033F8162033F82F
:100BD0001530014601A88DF804408DF805208DF8E8
:100BE0000630FFF7CFFF02B070BD00BF00B583B085
:100BF0000023014601A88DF804308DF805308DF8EA
:100C00000630FFF7BFFF03B000BD00BF30B5194B82
:100C10008DB01B68184DDBB100232A461C461169B4
:100C20001432890741BF0CA800EB840141F82C3C29
:100C3000013401330B2BF2D16CB9104A23461460F6
:100C400003EB830305EB83056B6898470DB030BD5C
:100C50000A4B1B68F4E70AF09BFAB0FBF4F303FBC2
:100C600014000CAA02EB800353F82C3C034A1360D7
:100C7000E6E700BF6C040020780000203803002065
:100C80000E2A30B436D81F4B0C789B5C48F689028C
:100C900004FB03F4C8F68802A2FB0452C2F3C702A5
:100CA00002700C7814B10AB9012202704C7848F62F
:100CB000890204FB03F4C8F68802A2FB0452C2F3C3
:100CC000C70242704C7814B10AB9012242708C7884
:100CD00048F6890204FB03F3C8F68802A2FB03422C
:100CE000C2F3C70282708B7813B10AB901238370F3
:100CF00030BC70470B7803704B7843708B788370EF
:100D0000F6E700BFACC2000810B5104B104C1A68D3
:100D100082B020460F49FFF7B3FF0F4B1B689BB112
:100D20000E4BA1782078627833F8104033F8122007
:100D300033F8113001A801218DF804408DF8052009
:100D40008DF80630FFF71EFF02B010BD54010020E1
:100D5000700000206C0000205C010020B8C1000879
:100D60000E4B1B68032B18D8DFE803F013100A02A0
:100D70000B4B00223F2119705A709A70FFF7C4BFC5
:100D8000084B012200201A60FFF730BF0020FFF758
:100D90002DBF054B1868FFF709BF704724040020DA
:100DA0006C000020700400205C0100202DE9F00F91
:100DB0000C0682B04BD46FEA020ADFF808C10AF1D0
:100DC000090A3F4B072A88BF4FF0000A00F10806C6
:100DD000C2F10708042703EBC10B8244CDF804805D
:100DE000B61A0124ACF14805072A16D801990BEB75
:100DF00007090346112B0CD819F8048C48FA01F89E
:100E000018F0010F1ABF4FF004080CF803800CF81B
:100E1000034001330139B342ECD1BAF1110F9FBF46
:100E200007EBC708534651464FEA480801D905E089
:100E3000194601334144112B6C54F9D901370C2F59
:100E40000CF1120CD0D102B0BDE8F00F7047B039F0
:100E50004C2932D8DFE801F02F31313131313131D5
:100E60003131313131313131313131312D31313176
:100E700031313131313131313131313131312B3168
:100E80003131313129313127313131312D31313168
:100E900031313131313131313131313131312B3148
:100EA000313131312900052185E7042183E7032110
:100EB00081E702217FE701217DE720217BE700BF59
:100EC000B8BD0008CC380020B0F5907F10D248F6AD
:100ED0003963C3F6E303A3FB00239B08DA0742BF91
:100EE00003EBC303C0EB83001130013008F0FCBDFD
:100EF000704700BF70B5294B82B01A6806460AB920
:100F000001261E60264A274B11785478907833F8D2
:100F1000111033F8142033F810300024224D8DF8CE
:100F200000108DF801208DF802308DF804408DF806
:100F300005408DF806400BE0FFF7C6FF15F8013CB1
:100F4000013443F00103B4F5907F05F8013C16D05D
:100F500015F8013B204603F00203DBB26946002B83
:100F6000EAD1204601A9FFF7AFFF15F8013C013493
:100F700023F00103B4F5907F05F8013CE8D116B1E8
:100F80000A4B1B6833B1FFF7F5FD094B01221A60CC
:100F900002B070BD0120FFF709FEF6E76C030020E8
:100FA00060010020B8C1000884380020240400201B
:100FB0008038002008B5064B1A6822B1002210467E
:100FC0001A60FFF797FF034B01221A6008BD00BFAC
:100FD0006C0400208038002008B50D4B0D481A68BD
:100FE0000D49FFF74DFE0D4B1B68032B03D00C4B37
:100FF0001B68990708D40B4B1B6803B908BD012077
:10100000BDE80840FFF776BFFFF784FDF3E700BFB8
:1010100094010020600100205801002024040020D9
:10102000740000205C0100202DE9F041864B84B063
:101030001A683AB985490B68002B00F0E48004B0C7
:10104000BDE8F081824A4CF6CD401678CCF6CC4013
:10105000A0FB06107D49002400091C600C60DFF82D
:10106000088200F0B580C8F8000055784CF6CD43F2
:10107000CCF6CC43A3FB05031B09DFF8F0C102D17A
:10108000002D40F0BE80CCF8003094784CF6CD4373
:10109000CCF6CC43A3FB04231B096E4F02D1002CDA
:1010A00040F0AD806C4A3B606C4B0020107050707B
:1010B00090701E705D709C70D8F800301C4693B123
:1010C000664A1478A34240F2968014B10020107052
:1010D0000124614A5E4815780078EB18834200F2DB
:1010E000A28013700124DCF800308BB15B48427899
:1010F00093427CD912B1002242700124564A5448CE
:1011000055784078EB18834200F2928053700124A6
:101110003868002863D0514B9A78904263D912B155
:1011200000229A7001244C4D494AAF7896783818BD
:10113000B0429CBFC0B2A87003D9B7424FD0AE70C6
:101140003046474992F800C092F801E06C782F7859
:101150005A781D789B7831F81C8031F8177031F877
:101160001EC031F8122031F816E031F8133031F892
:10117000146031F8104031F815008DF80A40394DEF
:101180008DF804808DF805C08DF806E08DF80870A4
:101190008DF809608DF80C008DF80D208DF80E305B
:1011A000002407E0012B34D0032B37D00134B4F5F1
:1011B000907F0AD0635D022BF4D1204602A901344E
:1011C000FFF782FEB4F5907FF4D1FFF7D3FC36E74A
:1011D000002E3FF448AF0123C8F8003045E764BB58
:1011E00001230B602BE7121A9A7001249BE7D21A95
:1011F0004270012482E7E41A1470012469E7012394
:1012000050E701233FE7DFF86080DFF860C0114F4F
:1012100052E7204603A9FFF757FEC7E7204601A97A
:10122000FFF752FEC2E785421CBF107001245AE747
:1012300085421CBF507001246AE7054A064D967826
:10124000A878064B7DE700BF6C04002080380020A2
:1012500060010020780400204003002044030020A7
:10126000B8C1000884380020CC03002064030020AB
:1012700070B5154A154B94781178557833F81110DC
:1012800033F8152033F8143082B00024104E054690
:101290008DF800108DF801208DF802308DF8044093
:1012A0008DF805408DF80640A35D20462B4201A92C
:1012B00018BF69460134FFF707FEB4F5907FF3D1FC
:1012C000FFF758FC02B070BD60010020B8C10008F3
:1012D000843800202DE9F8435A4B5B4E1A682AB92E
:1012E0003768002F00F09980BDE8F883DFF860814F
:1012F00000221A603260C8F80020544C4FF0000EF3
:101300007746A4460EEBCE056D0012230CEB0509C3
:101310005A1EA918605C611810F0010F46D0112AFE
:1013200005EB03074BD01CF8077020F00100FF0706
:1013300040D40870002A47D0023B0127002BE7D198
:101340000EF1010EBEF1100FDCD10120FFF790FF6E
:10135000002F5ED0D8F800300127012B08BF3B4C8E
:10136000C2D1DFF8E8E04FF0000CF1460CEBCC0501
:101370006D00002309EB0508EA18A15CA21801F032
:101380000600022827D00133112BF5D90CF1010CEE
:10139000BCF1100F0EF1120EE8D10420FFF768FF28
:1013A000002FA1D101233360BDE8F8831346002B41
:1013B000AED1C5E713460127002BA9D1C0E720F025
:1013C000010089F81100B7E70EF1010E0127BEF107
:1013D000100F97D1B9E73BB301F00400C0B2002869
:1013E000D1D141F00401112B117022D00133EA1840
:1013F000A25C02F00202D2B24AB1112B19D0013321
:101400001EF8032002F00202D2B2002AF5D1012711
:10141000BAE70123C8F80030A3E7DFF83480D8F832
:101420000030002B99D168E741F0040188F80010E2
:10143000DCE70CF1010C0127BCF1100F0EF1120ECC
:1014400094D1AAE76C040020803800208438002062
:10145000740300202DE9F00F6A4B1A6832B96A4A0A
:101460001368002B67D0BDE8F00F704700201860AC
:10147000654A664E664B0121106031601960336821
:101480008BB1644810256C1E0023C25C02F003017E
:10149000012936D00133122BF7D112382546002C02
:1014A000F1D134603FE0DFF868A1DAF800100029DC
:1014B0003ED0DFF874B1DBF80020002A3DD0564C56
:1014C000564A2168106801EBC105554A00EB4505F5
:1014D0000131575D01EBC10600EB4600514E27F08C
:1014E000040757553668155CB14245F0040708BF3C
:1014F00045F005051754216004BF1554CBF80030A2
:1015000011E0474904EBC40003EB400022F0010264
:101510000F2C0A5407D005EBC50503EB4503CA5C45
:1015200042F00102CA540520BDE8F00FFFF7A0BE4B
:101530000123136097E7354EA1E740F26441C2F200
:1015400000010F6840F2D03340F250313148C2F20E
:101550000003C2F20001D3F80090D1F80080944655
:101560001026A0F58775741ED30748D40023C25CEB
:1015700002F00301022905D00133122BF7D14B46AB
:10158000002210E0A4B112F0010216D006EBC60250
:1015900003EB4202A95CB04641F00401A9544FF0AC
:1015A000010C27460122264612388CB19946DAE70B
:1015B000EA5C42F00502EA54F3E7BCF1000FF0D117
:1015C000E95C4FF0010C41F00401E9549046E8E772
:1015D00040F26441C2F200010F6040F2D031C2F229
:1015E00000010B6040F25033C2F20003C3F80080E8
:1015F000CBF800C0002A96D1CAF8002093E74B46EA
:10160000D1E700BF6C04002080380020480400208F
:10161000480300209239002050030020D00300200E
:101620008438002064040020800400202DE9F84361
:10163000694B1A6832B9694D2B68002B00F0A18004
:10164000BDE8F88300201860654C644B206018608A
:101650004FEAC00C0CEB00035B00624A1918C0F1A2
:1016600012061546F3188A18EF18A846134619787B
:1016700041F0040103F8011BBB42F8D1C0F10F0E89
:10168000431C734528BF4FEACE0C1BD20CEB00075E
:10169000C0F1110300EB08014FEACE0C03EB470346
:1016A00012390CEB0E075B1901EB4707917C41F0F7
:1016B000040102F8121F997CBA4241F0040103F8B8
:1016C000121FF3D10CEB0E0205EB42020346D15C74
:1016D00041F00401D1540133B342F8D3002848D07B
:1016E000421EC0F11307BA420FD202EBC2014900F9
:1016F0000B185B197E19013B761813F8011B21F0BA
:101700000401B34203F8011CF7D1C0F110084045B1
:1017100028BF4FEAC8091DD200EBC0034FEAC80931
:1017200002EB4303511909EB080CC0F112065B19D7
:1017300001EB4C0C93F800E0991A2EF0040E83F89C
:1017400000E011F806E012332EF0040E634501F8B4
:1017500006E0EFD109EB080300EB43035B19013B03
:1017600013F8011B013221F00401BA4203F8011CF5
:10177000F6D30420FFF77CFD236801332360BDE826
:10178000F883174C206807287FF662AF08281CBF33
:10179000144B03F5907404D119E0A34203F8010C33
:1017A0000ED013F8012B02F00201C9B242F004007E
:1017B00022F004020029F0D1A34203F8012CF0D159
:1017C0000420FFF755FD01232B60BDE8F8830722B5
:1017D0000B27044D89E700BF6C04002080380020EF
:1017E0004C0400208438002070B5264A264813682F
:1017F0001BB90368002B3BD070BD00231360234D41
:10180000234A03602B6013602E6886B9214B03F5D1
:1018100090711A7822F0040203F8012B8B42F8D160
:101820000420FFF725FD2B6801332B6070BD184A9B
:10183000136801331360DA07DED5741EA4B2B4F561
:10184000907F10D213490B5D03F00202D2B22AB18D
:1018500010E00B5D03F00202D2B25AB90134A4B217
:10186000B4F5907FF5D10123036001362E6070BD81
:10187000064DC9E743F0040304200B55661CFFF72F
:10188000F7FCF2E76C0400208038002054040020AC
:101890004C030020843800202DE9F00F8D4A86B0DB
:1018A000136843B98C4B1A68002A00F0098106B00E
:1018B000BDE8F00F704700231360884C864A236010
:1018C00013600393864F002000EBC00207EB420237
:1018D00000231178013321F00401122B02F8011BBF
:1018E000F7D101301028EFD1039B002003F101094B
:1018F000C3F10806C4F800900196C21900231178BC
:10190000013321F00801122B02F8011BF7D112302C
:10191000B0F5907FF1D1019A714D5342CDF8089006
:1019200093469A4600269946BAF1080F2CBFD04636
:101930004FF008084A4601990023BBF1070F34BF56
:10194000DC464FF0070C17E0082934BF0846082092
:10195000082B644603D9092A2CBF1046092004EB42
:10196000C40400EB44003C5C44F008043C540133E4
:1019700001310132122B15D0E85C00F00200C0B238
:101980000028F4D0072EDFD9082B05D8082934BF4A
:10199000084608204446E2E7082A8CBF1046092082
:1019A0004446DCE701361235102E0AF1010A0BF12C
:1019B000010BB9D1039E002301936FF0110303FBC8
:1019C0000673DDF808906FF0120C02936FF023039A
:1019D0000CFB06FCDDF80CB003FB06F65A46D243BE
:1019E0000596CA464FF000080492039E0BEBCB0508
:1019F0006D00049BAA19019EED18F119D219ED1979
:101A00004C4600231DE0082B2ED8C14509D8994526
:101A100007D8059EA81910F8126C46F0040600F8C5
:101A2000126C11F8010B00F00806F6B21EB140F07E
:101A3000040001F8010C0133013201350134122B8D
:101A400029D012F80C00C007EBD5B8F1070FDAD98E
:101A5000082B16D8BAF10F0FE3D89945E1D8A87C26
:101A600040F00400A874DCE7C145DAD8112CD8D8BE
:101A7000029E301910F8126C46F0040600F8126C41
:101A8000CFE7BAF10F0FCCD8112C9EBFD07C40F01D
:101A90000400D074C5E7019A029B08F101081232D4
:101AA0001233B8F1100F01920BF1010B02930AF1FE
:101AB000010A9AD1042006B0BDE8F00FFFF7D8BBA9
:101AC000064C2268082A03927FF6FCAE01221A60B7
:101AD000EDE600BF6C040020803800207404002074
:101AE000843800202DE9F84FA64C2368002B40F0E5
:101AF000A980A54B1B68032B12D8DFE803F07646BC
:101B000013022368002B40F0CB80A04A13683BB936
:101B10009F490B68B3F5907FC0F0C9800123136023
:101B2000BDE8F88F2368002B00F0A28095490022C1
:101B30000A60984B95491A600A60974C02F11205A9
:101B400004F112081D600021C2EB08088B1A1B1952
:101B500008EB01000DE013F8126C16F0010F9E5C0B
:101B600000F0028146F004069E540133984200F0D2
:101B700002818D42EFD993F80E6106F00206F6B2AB
:101B8000002E00F0F0809E5CECE72368002B7AD0FA
:101B90007C4900230B60814A7C4913600B605F1C09
:101BA0007D4C1E46176003F5907C594203F11300EB
:101BB00033193A460DE05D7815F0010F5D5C00F0D9
:101BC000F28045F0040501325D540133824200F099
:101BD000F280112AEFD913F8115C05F00205EDB27D
:101BE000002D00F0DF805D5CEBE72368002B34D034
:101BF000644A002111606A4B644A19601160481CF4
:101C0000654C18604E42C1F59077331900220EE002
:101C100013F8015C15F0010F5D5C00F0978045F052
:101C2000040501325D540133122A00F0978090427E
:101C3000EED95D7C05F00205EDB2002D00F0858047
:101C40005D5CECE709F0A4FAC3179B0FC21802F021
:101C50000302D31A4C4A13604DE74C4A1368002B19
:101C60007FF45EAF4E4B196811293FF657AFC6E7B8
:101C700046490B68002B7FF453AF464B1A68B2F508
:101C8000907F09D259E741490B68002B7FF448AF98
:101C9000424A1368112B82D901230B60BDE8F88FEB
:101CA000384A002313603A49384A0B6013603A4CB3
:101CB0004FF6EE7A03F11202CFF6FF7A0A6003F5CF
:101CC000997B04F11208C3EB0A0A40F21F16A2F531
:101CD00090710AEB02000919131902EB080518E0CC
:101CE00091F82071C2EB030CFF0755BFC2EB03074D
:101CF0001CF8007017F800C047F0040756BF2CF01E
:101D0000040C0CF8007007F800C001330131AB423D
:101D100013D0B242E4D90F78C2EB030907F00207EF
:101D2000FFB2002F4CD019F80070013347F00407C0
:101D30000131AB4209F80070EBD112325A45C6D1DD
:101D40000420BDE8F84FFFF793BA5D5C25F0040569
:101D500001325D540133122A7FF469AF1236BE425C
:101D60007FF453AFECE79E5C26F004069E540133EB
:101D700098427FF4FEAE1231B1F5907F7FF4E6AE6B
:101D8000DEE700BF6C0400206803002080380020DC
:101D90006003002028030020843800205004002025
:101DA000340400205D5C25F0040501325D540133EC
:101DB00082427FF40EAF123666457FF4F9AEBFE77C
:101DC00019F8007027F0040709F800709DE700BFBC
:101DD0002DE9F04FB24A85B01368B24E33B933687B
:101DE000002B00F0968005B0BDE8F08F0023136053
:101DF000AD4AAE4C1360AE4AAE4D1360AE4A33608E
:101E000023602B6013602368002B43D1AB4A117809
:101E10001F295FD951781F2900F2C6803F228DF813
:101E200008308DF809208DF80A30A54B03A802A9C7
:101E30001A689D4FFEF724FFA2492E689DF80C807A
:101E40009DF80DC09DF80EE09F4B38689F4A31F811
:101E5000188031F81CC031F81EE006EBC60100EB1B
:101E600041000026194683F8008083F801C083F8FA
:101E700002E0167056709670FFF726F823682D68FA
:101E800093493868CD5493495A1CC8542260FEF7D0
:101E900071FEA8E72A681C2A24D98F4B03F5907499
:101EA00003E0A34203F8010C0ED013F8012B02F05B
:101EB0000201C9B242F0040022F004020029F0D16C
:101EC000A34203F8012CF0D10420FFF7D1F901233C
:101ED000336088E73F228DF808208DF809308DF8AF
:101EE0000A30A2E7DFF8C8E16F4FDEF80030D7F81C
:101EF00000C09A4277D0704B1B6802F00109B9F11B
:101F0000000F4AD163452DD90CF101033B602A68CB
:101F10002FE0664C674D76E7BBF1110F19D85B4691
:101F200008EBC80043F6840C03EB4000C2F2000C3F
:101F30001CF800C01CF0010FDDF800C004D0E0E088
:101F4000C85CC00700F1DD800133122BF8D1CDF859
:101F500000C008F101081231B8F1100F65D11D233E
:101F6000CEF80030DEF800309A4228D301232A68E8
:101F700033600F2A2ED92368DFF854810D2B78D0D7
:101F8000544E29683A680C2B08F80310F25401D813
:101F900001332360FEF7EEFD25E76345E2D20CF145
:101FA000FF333B602A68E4E792781F2A0AD88DF84D
:101FB00008308DF809303F238DF80A3035E70132BB
:101FC0002A60D6E73F228DF808308DF809208DF879
:101FD0000A202AE7386802EBC20200EB42003A49C5
:101FE000FEF772FFC7E740F23040C2F2000003681C
:101FF0009C4582D112F0010900F08B800CF1FF3B6F
:102000009246BCF1000F02D102F1010AE346BAF197
:102010000F0FA4D843F684030AEBCA01C2F20003EF
:1020200003EB4101D046CDF800C0D0455FD018F099
:1020300001033FF475AF112308EBC80043F6840C8D
:10204000C2F2000C03EB40001CF80000DDF800C0F9
:10205000C00706D4002B3FF47AAF013BC85CC00731
:10206000F8D540F23040C2F20000CEF800800360A4
:1020700045E798F80030174E0F2B2FD90023013376
:1020800018F803E0F15C08EB0300F2180C2B00F8E1
:1020900001EC02F8011CF2D12368013B236070E7D8
:1020A0006C040020803800203403002054030020FA
:1020B0001403002078030020300400205801002081
:1020C00094010020B8C10008200400202C04002046
:1020D000180300203804002084380020307803EBF7
:1020E000C303104900EB4300FEF7EEFEC6E718F00D
:1020F000010F3FF411AFBBF1FF3F18BF5B469BD10F
:1021000027E740F23041C2F20001CEF800800B60B8
:10211000F5E6BCF1100F9CBF0CF1010B92467FF667
:1021200076AF71E72C0400202DE9F04F7F4B85B08E
:102130001A687F4C002A40F098802368002B57D102
:10214000DFF800B2DBF800202F2A54D8DFF8ECA12A
:10215000DFF8F8819AF800009AF801109AF8022046
:102160008DF80C008DF80D108DF80E20994658F85A
:10217000044B182C2DD9A4F11805012D63D0A4F11E
:102180001A030F2B67D90F2D5DD904EBC407193C37
:10219000A9F5EA730126A51E0F2C03EB470709D901
:1021A0000E2D45D90136243F6B1C2C460FD0A51EA1
:1021B0000F2CF5D89AF8013007F11200B3FBF6F3B3
:1021C00003A98DF80D30FEF77FFE002CE8D158F8FA
:1021D000044C09F101090134B9F1120F48F8044C1B
:1021E000C5D1FEF7C7FCDBF800300133CBF8003077
:1021F00005B0BDE8F08F4F4B03F5907503E0AB429F
:1022000003F8010C0ED013F8012B02F00201C9B241
:1022100042F0040022F004020029F0D1AB4203F89E
:10222000012CF0D10420FFF723F801232360DFE71E
:102230009AF801303846B3FBF6F303A98DF80D3058
:10224000FEF742FEAEE705EBC50009EB40003A4958
:10225000FEF73AFE99E705EBC500A9F1240303EB6D
:1022600040003649FEF730FE8DE7354A00261768F4
:102270001E60344B3F253A4602A869461E60102373
:102280008DF806308DF800508DF801508DF805500E
:1022900026608DF802608DF80460FEF7F1FC3A4686
:1022A00003A801A9FEF7ECFC274B9DF80E709DF8E2
:1022B00008809DF809C09DF80AE09DF80C509DF833
:1022C0000D001D491D4A33F8155033F8188033F8B6
:1022D0001CC033F81EE033F8100033F817301570C7
:1022E0001A4F81F8008081F801C081F802E0507037
:1022F000937035460DE008F04BFFC3171B0FC01855
:1023000000F00F00C31ABB5101350436122D3FF403
:1023100014AFEA07EFD408F03BFFC3171B0FC01838
:1023200000F00F00C31A0833BB51EDE76C04002026
:1023300080380020843800206004002058040020E9
:102340009401002058030020B8C10008D8030020E1
:1023500010B582B0002914BFFF230023002814BF4A
:10236000FF240024002A14BFFF220022002001A91C
:102370008DF804408DF805308DF8062007F0B4FB89
:10238000012007F02BFB02B010BD00BF074B01205E
:1023900003F5907113F8012B12F0020214BF03F839
:1023A000010C03F8012C8B42F4D1704784380020D3
:1023B0002DE9F84F1746814688460AB9BDE8F88FDF
:1023C0000020FEF797FD39077FD4FA0679D44B4AEF
:1023D0004B4B126803EBC20113F832B07B0791F844
:1023E00001A0EBD5474E4B224748002108F03BFCAB
:1023F00006F590750122334613F8014B14F00204E0
:1024000014BF03F8012C03F8014CAB42F4D13F4B4D
:102410001B68002B67D03E4B1B68D80767D53A4B2B
:1024200001225A709A703B4BCBEB0B1B08EB8B01D4
:10243000354C03EBC10101200023CA185278013347
:1024400012B1072BA054F8D10B780AEB8A0A9944F1
:10245000B9F1180F88BFA9F119092F4B0AEB8A0AA5
:102460000AEB0904284803EB840401210023E25C01
:10247000013312B1042B8154F9D1284CDFF8A8C0E4
:10248000002504F14B0714F8013F93B105EB0C0351
:10249000987815F80C205B7858B102EBC202181836
:1024A00006EB4202D15C41F00201D1540133834278
:1024B000F8D10335BC42E6D1194B01221A60BDE8C0
:1024C000F88F0120FEF792FB81E706F095FDC8200A
:1024D000FEF7B6FA134B1B68002B7FF478AF012090
:1024E000FEF764FB73E7F9067FF568AFE4E7B8F140
:1024F000000F18BFB8F11E0F95D190E77C030020A4
:1025000070DC000884380020800300205C0100207B
:1025100074000020BCC200085CD700087F030020C4
:102520006C040020240400208CDB000840F27403BB
:10253000C2F200031868704738B50B4B04461B689D
:102540000A4D032B04D0830702D52B68980707D5C3
:10255000FEF706FC064B01222C601A60204638BDAF
:10256000FEF7D8FAF4E700BF24040020740000202E
:102570006C04002040F22443C2F200031868704744
:10258000032810B509D8074C2368834203D0206084
:10259000FEF7E6FB2368184610BD024B1B68184681
:1025A00010BD00BF2404002040F26813C2F20003F3
:1025B000186870473B28024B88BF3C201860704762
:1025C0006801002040F26413C2F2000318687047EB
:1025D0003A28024B88BF0020186070476401002031
:1025E00040F27C33C2F20003186870471128044B94
:1025F00004D81860034B01221A60704718687047AE
:102600007C0300206C040020064B1868102805D9B4
:1026100000201860044B01221A60704701301860D6
:10262000F8E700BF7C0300206C040020054B18680D
:1026300028B101381860044B01221A60704711203C
:102640001860F8E77C0300206C04002040F25C4333
:10265000C2F2000318687047074B10B5186000B14C
:1026600010BD064B0F241C60FEF7B6FC044B1C602B
:10267000BDE81040FEF748BB5C0400209401002038
:102680005401002040F29013C2F200031868704712
:10269000024B0A288CBF1868186070479001002010
:1026A000044B1868092802D90020186070470130CF
:1026B0001860704790010020044B186810B1013871
:1026C000186070470A201860704700BF9001002012
:1026D000064B1B68012B00D07047054B00223F21A1
:1026E00019705A709A70FEF777BC00BFD4030020AF
:1026F0005801002040F2D433C2F20003186870473A
:10270000012810B5034602D9054B186810BD044CCA
:102710002068984203D02360FFF7DAFF206810BDDD
:10272000D4030020F0B5584B83B01B680446012B3E
:1027300042D0022B01D003B0F0BD20B9534B1A6830
:10274000002A7AD018600020FEF750FA504B1B6820
:102750003B2B2ED81D2B73D967081E254D4A4E4B97
:1027600010785178927833F8100033F8111033F85C
:102770001220464B8DF804001B688DF805108DF86B
:102780000620002B46D1AF423CBF444E3C4606D308
:1027900039E000F2211007F0A7F9AC4233D23068DB
:1027A00001A920180134A842F3D33C383B28F4D8BF
:1027B000EFE727463C25D1E70020FEF717FA344B18
:1027C0001B683B2B48D9354A3C231268A418314A70
:1027D000A34298BFC3EB040411782F4B907855782F
:1027E00033F8111033F8152033F810303B2C8DF8E6
:1027F00004108DF805208DF8063004D804F221105D
:1028000001A907F071F9264B1B68002B93D0FEF746
:10281000B5F990E7214E002405E000F2211007F001
:1028200063F9BC42EFD8336801A9E0180134A8422B
:10283000F3D33C383B28F4D8EFE701221A6082E753
:10284000132B7FF678AF4AF6AB27CAF6AA27A7FB69
:10285000043714257F0881E71D2B0ED8132B7FF634
:102860006AAF4AF6AB23CAF6AA23A3FB04240B4A99
:102870001423126802EB5404A9E7084A1E231268C5
:1028800002EB5404A3E700BF2404002070040020DE
:102890006801002070000020B8C100086401002019
:1028A0005C01002038B5814B1B680A2B1AD8804A7E
:1028B000804C12687AB9804D2A68C2B97F4A804834
:1028C00003EB8303116800EB8303986801318142B5
:1028D000116045D238BD7A4A03EB830302EB8303D0
:1028E0005B689847744B1B68002BF3D0714C754B99
:1028F0001B68012B1FD0744B1B68032B06D0236869
:10290000002BE7D1BDE8384006F092BB6F4B704911
:102910001A68496B0132B2EB411F1A60EFD36D4A5E
:102920000020116818604B1E052B3AD8DFE803F031
:1029300059A19A938C50684B68491A6849690132C9
:10294000B2EB411F1A60D6D3654A002011681860A7
:102950004B1E052B0CD8DFE803F0625B544B70690B
:102960005B680021116098472B68002BBED1B1E74E
:102970005C490B680133072B00F096800B605A49C5
:1029800013600A68564801320D2A0A6000F08380FD
:102990000E2AB0D1013B08BF0623036000230B6061
:1029A000A9E752490B680133072B72D00B605049DD
:1029B00013600A68474801320D2A0A6060D00E2A67
:1029C0009DD1013B08BF0623036000230B6096E7FF
:1029D000484B99780029E4D001399970FEF794F9B1
:1029E0008DE7444B59783E29DBD801315970F5E722
:1029F000414B59780029BBD001395970FEF7ECFAE8
:102A000079E73D4B99783E29B2D801319970F5E7C5
:102A1000394B19780029ABD001391970EEE7364BE4
:102A200059783E29A4D801315970E7E7324B99789B
:102A300000299DD001399970E0E72F4B19783E2984
:102A400096D801311970D9E72A4B19783E29A8D8B0
:102A500001311970C2E7274B59780029A1D00139FB
:102A60005970BBE7234B99783E299AD80131997068
:102A7000B4E7204B1978002993D001391970ADE7DC
:102A80000133072B18BF03607FF439AF01230360C4
:102A900035E701238AE70133072B18BF03607FF472
:102AA0002AAF0123036026E7012367E79001002096
:102AB0006C0400205C01002080380020700300209E
:102AC00078000020D4030020240400207C0400208F
:102AD0002C0000202C0300205C0300206C0100204F
:102AE0006804002028040020980100203C030020F6
:102AF0008C0100206C00002058010020064B1A7841
:102B00003E2A07D803D13F221A70FEF765BA023277
:102B10001A70FAE7704700BF58010020064A137880
:102B200043B1012B03D100231370FEF755BA023BCA
:102B30001370FAE7704700BF58010020064B5A781F
:102B40003E2A07D803D13F225A70FEF745BA023217
:102B50005A70FAE7704700BF58010020064A5378C0
:102B600043B1012B03D100235370FEF735BA023B6A
:102B70005370FAE7704700BF58010020064B9A785F
:102B80003E2A07D803D13F229A70FEF725BA0232B7
:102B90009A70FAE7704700BF58010020064A937800
:102BA00043B1012B03D100239370FEF715BA023B0A
:102BB0009370FAE7704700BF5801002040F25813A5
:102BC000C2F200031A7802705A7842709B788370C0
:102BD000704700BF10B404784178827840F25813EF
:102BE000C2F200033F2C34BF20463F203F2928BFBC
:102BF0003F213F2A28BF3F22187059709A7010BC9D
:102C0000FEF7EAB940F26C03C2F200031A780270D0
:102C10005A7842709B788370704700BF10B4047874
:102C20004178827840F26C03C2F200033F2C34BF3B
:102C300020463F203F2928BF3F213F2A28BF3F226F
:102C4000187059709A7010BCFEF75EB840F2941379
:102C5000C2F20003186870470F2803D8034B1860AE
:102C6000FEF7BAB9014B0F221A60F9E79401002070
:102C7000034B1A6802B97047013A1A60FEF7ACB903
:102C800094010020044B1A680E2A00D970470132C3
:102C90001A60FEF7A1B900BF9401002040F254135E
:102CA000C2F20003186870470F2803D8034B18605E
:102CB000FEF72AB8014B0F221A60F9E754010020F1
:102CC00070B5012682B040F25D1516F0010F0CBF01
:102CD0000021392116F0020F0CBF0022392216F014
:102CE000040F0CBF002339238DF804108DF8052044
:102CF0008DF806300024204601A9013406F0F4FEC8
:102D0000AC42F8D1204606F069FE01360320FDF7FB
:102D1000A5FE082ED9D10020FEF7ECF800200146D0
:102D20000246FFF715FB02B070BD00BF2A4B2DE92C
:102D3000F04103F59071012413F8012B12F0020207
:102D400014BF03F8014C03F8012C8B42F4D1017835
:102D500000293FD08046074608260020C6F1080219
:102D6000FEF724F898F80110013759B3112E16D840
:102D70003D46344601E0112C11D820460022FEF7D2
:102D800015F815F8011F09340029F4D105E0204693
:102D9000202100220934FEF709F8112CF7D904206C
:102DA000FEF766FA3220FDF74BFE013E0CD017F815
:102DB000011C0020C6F10802FDF7F8FF98F8011089
:102DC0000029D3D13446E8E718F8011F0029C3D100
:102DD000BDE8F081BDE8F08184380020F8B5324BC1
:102DE0001B681BB1A0F114053B2D00D9F8BD0020D4
:102DF000FEF780F82D4B2E4C93F8883004F5907137
:102E0000C3EB031305EB83052A4B012003EBC50538
:102E1000234613F8012B12F0020214BF03F8010C31
:102E200003F8012C8B42F4D1234E7079F278337978
:102E300058B102EBC202181804EB4202D15C41F017
:102E40000201D15401338342F8D1307AB279F37957
:102E500058B102EBC202181804EB4202D15C41F0F7
:102E60000201D15401338342F8D10027EB195B787A
:102E7000ABB103EB4303F1188878F25C4B7858B19F
:102E800002EBC202181804EB4202D15C41F00201CD
:102E9000D15401338342F8D10137072FE6D1074BD4
:102EA00001221A60F8BD00BF5C01002070DC000840
:102EB00084380020BCC200088CDB00086C040020B1
:102EC0002DE9F04FBA4B04461B6893B0184613B96E
:102ED00013B0BDE8F08F3F268DF834603C26032503
:102EE0008DF82360162600230CA92A46A4208DF80D
:102EF00024600F268DF835308DF836308DF825306A
:102F00008DF826308DF82B308DF827508DF82960FC
:102F100000F0B0FB01220DF12101A72000F0AAFB77
:102F200001220DF12501A82000F0A4FB01220AA92D
:102F3000BD2000F09FFBBE2001220DF12A0100F010
:102F400099FBB4F5843F80F0A4809DF821809DF822
:102F500022C0B8F1110F88BF4FF000089DF825E09E
:102F600088BF8DF82180BCF1030F84BF4FF0000CA7
:102F70008DF822C09DF82610BEF10A0F84BF4FF0D5
:102F8000000E8DF825E0012902D900218DF82610C8
:102F90009DF828700F2F02D90F278DF828709DF803
:102FA00029600F2E71D89DF82A00012802D0002038
:102FB0008DF82A009DF823203C2A009203D93C2555
:102FC0008DF8235000959DF824303B2B02D9162311
:102FD0008DF82430774C07932568774B01959DF841
:102FE00027509DF834B002959DF830509DF835A0DB
:102FF00003959DF831509DF8369004959DF8325018
:1030000083F800B005959DF82B5083F801A0069534
:1030100040F27C35C2F20005C5F80080DFF8C481BB
:10302000029DC8F800C0DFF8C0C183F80290CCF858
:103030000050DFF8B8C1614BCCF800E0DFF8B0E138
:103040005F4ACEF800101F6003995E4B1170049D1B
:1030500005991E605C4B557091701860009A5B4B2F
:10306000079D1A605A4B06991D605A4B1960002340
:103070002360FDF749FEFDF7AFFF019A2260FFF7DD
:1030800027FBFDF76DFE012022E70F268DF8296052
:1030900089E7A92001220DF1260100F0EBFA40F6A4
:1030A000FF03C0F201039C427FF64FAF01220DF1F6
:1030B0002701BC2000F0DEFA0DA92A46D72000F037
:1030C000D9FA01220DF12901DA2000F0D3FADB2030
:1030D00001220DF1220100F0CDFAB4F5003FFFF41A
:1030E00034AF01220DF12301DC2000F0C3FADD2012
:1030F000012209A900F0BEFAFF23C0F202039C429C
:103100007FF623AF0DF12B010122E02000F0B2FA8F
:103110000FA90B22E52000F0ADFA0EAE0BA902229A
:1031200040F2251000F0A6FA40F235103146042294
:1031300000F0A0FA0DF14605274B0DF13B0005E02C
:1031400042F002021A611433A84212D010F8012F83
:10315000FF2AF8D002F01001C9B202F00F029A6003
:103160001A690029ECD122F002021A611433A84234
:10317000ECD19DF82C301948FF2B1EBF184A03F0E4
:103180000F0353609DF82D30FF2B1EBF144A03F030
:103190000F0353610023F25C00EB03110133FF2A9C
:1031A0001CBF02F00F024A60042BF4D1CDE600BF31
:1031B000A40400205C0100206C0000209401002089
:1031C00058010020540100205C0400206801002008
:1031D0006401002030030020780000202C00002033
:1031E0006C010020240400207400002090010020C5
:1031F000D40300202DE9F04F854BA3B01B68002BB2
:1032000000F08C80834B844A93F8008093F801C0CF
:1032100093F802E0814B92F800B01F68804B92F85F
:1032200001A01E687F4B92F802901D687E4B8DF8BE
:1032300019501C687D4B8DF81A401B688DF820B022
:1032400000937B4B009C1B688DF81B400193794BCE
:10325000019C1B688DF821A00293774B8DF822907A
:103260001B688DF824800393744B8DF825C0186873
:10327000734B8DF826E01968724B8DF815701A683B
:103280008DF816608DF81C40029C6F4B8DF81D4028
:10329000039C8DF817008DF81E408DF81810002043
:1032A0008DF81F2012ACFF250A2888BF255409D8A5
:1032B0009A68196902F00F028907225444BF42F04C
:1032C00010022254013014334028EDD15F4800230E
:1032D0000AAEFF22012B9BBF00EB03114968F25499
:1032E00001F00F0198BFF1540133102BF2D158486F
:1032F00000230EADFF21032B9BBF00EB031252688E
:10330000E95402F00F0298BFEA540133102BF2D1B6
:10331000A42008A9032200F0C7F918B9002023B09F
:10332000BDE8F08FA7200DF11501012200F0BCF9D6
:103330000028F3D0BC200DF11901012200F0B4F9EE
:103340000028EBD0A8200DF11A01012200F0ACF901
:103350000028E3D0A9200DF11B01012200F0A4F9FF
:103360000028DBD0BD2007A9012200F09DF900282C
:10337000D4D0BE200DF11E01012200F095F90028E5
:10338000CCD0D72009A9032200F08EF90028C5D09F
:10339000DA200DF11D01012200F086F90028BDD0D0
:1033A000DB200DF11601012200F07EF90028B5D0D6
:1033B000DC200DF11701012200F076F90028ADD0D4
:1033C000DD2006A9012200F06FF90028A6D0E02038
:1033D0000DF11F01012200F067F900289ED0E520C1
:1033E0002146402200F060F9002897D040F22510D5
:1033F0003146102200F058F900288FD0102240F2F8
:103400003510294600F050F9003018BF012086E73A
:10341000A40400206C000020580100207C03002040
:10342000240400207400002090010020D403002018
:1034300094010020540100205C0400206801002059
:103440006401002030030020780000206C0100207F
:103450002C00002006F072BB2DE9F8438146884617
:10346000174605F061FC10B90020BDE8F88355202F
:1034700005F002FD2E48082105F03AFD442005F034
:10348000FBFC002443F2144505F0B8FC0134AC42C7
:1034900098BF002814BF00260126F5D043F214433C
:1034A0009C4227D805F040FC0028DDD0552005F0CF
:1034B000E3FC204C08211E4805F01AFDBE2005F053
:1034C000DBFC0921204605F0C9FC05F02DFC1A4B58
:1034D0001B68222B13D0282B11D00923C9F80030E8
:1034E00094F901300120DB0FC8F8003023783B60ED
:1034F000BDE8F88305F018FC3046BDE8F883237971
:103500006278C3F341132578093302F00704C3F14D
:103510000C00191F45FA00F004FA01F1D209014329
:10352000C9F800300120C8F800203960BDE8F883F0
:10353000980400208404002094040020F8B5A0F131
:103540000905032D044602D900263046F8BD05F0D2
:10355000FFFC05F0E9FB0028F6D02E4F384605F0B9
:10356000D5FC3B782C4A012113602C4A222B0646BD
:10357000116001D0282BE8D105F0D6FB0028E4D05B
:10358000552005F079FC264F0821224805F0B0FCB3
:10359000BE2005F071FC0921384605F05FFC3B793F
:1035A000C3F341130933A342CFD005F0BDFB00287C
:1035B000CBD0552005F060FC0821164805F098FC9A
:1035C0004E2005F059FC7F2005F056FC802005F0C8
:1035D00053FC680100F0E00005F04EFC05F0A4FB90
:1035E00005F0A2FB0028B0D0552005F045FC0948A5
:1035F000082105F07DFC482005F03EFC002405F084
:10360000FDFB0134F92C98BF0028F8D005F08CFBA5
:103610009BE700BF98040020940400209004002041
:10362000840400202DE9F04184B003F02FF8DFF886
:10363000408000240127650045F0A0050126009781
:103640002846002132460DF10F03A419C8F8005096
:1036500003F054F830B1082CEDD1044B186804B0D5
:10366000BDE8F081014B30461E60F8E7A40400205D
:10367000A004002010B50A4B82B01C680B4614B998
:10368000204602B010BD0092064A0146126810465C
:10369000012203F033F8D0F1010038BF0020F0E739
:1036A000A4040020A00400202DE9F047144B82B0B0
:1036B0001B68174603B3EAB1DFF84CA0114C06466D
:1036C000C0EB01094FF001080025DAF80000CDF841
:1036D00000803146012209EB060303F08DF858B94A
:1036E00010202368002BFCD001382560F9D1013669
:1036F000013FEAD1012000E0002002B0BDE8F087E0
:10370000A4040020A4390020A004002030B53A4BC6
:1037100087B01A68044682426BD068461C6006F087
:1037200029FD02A807F09EF80420012106F0EEFE14
:103730000420012106F0EAFE4FF40030012106F0DA
:10374000F3FE04234FF400600325C4F20100694630
:10375000ADF8003018238DF803308DF8025006F0D4
:10376000A5FC08234FF40060C4F201006946ADF8DF
:10377000003048238DF803308DF8025006F096FC97
:103780004FF48840C4F20000012107F0A9F800239B
:103790004FF488401D46C4F2000002A9ADF80C3079
:1037A000ADF80E30ADF81030ADF814300C23ADF894
:1037B0001230029406F0F0FF4FF48840C4F200008B
:1037C000012107F05BF84FF48840C4F2000040F29A
:1037D0002551012207F060F826238DF8043001A856
:1037E00001238DF805508DF806508DF8073006F04E
:1037F00067FA07B030BD00BFA804002030B40F4AFC
:1038000013687F2BFCD80E490E4D0B685C1C7F2C77
:1038100045F8230098BF0C6001D900230B6072B6F5
:1038200013680133136062B64FF48840C4F200009D
:1038300040F22771012230BC07F02EB8B8060020F4
:10384000BC060020B004002010B50446007828B162
:10385000FFF7D4FF14F8010F0028F9D110BD00BF05
:1038600040F2AC43C2F200031868003018BF0120D8
:10387000704700BF30B40D4B1A6882B10C490D4D32
:103880000A68541C802C55F8225018BF0C6009D0CF
:1038900072B61A68013A1A6062B6012205601046D3
:1038A00030BC704700220A60F2E700BFAC04002081
:1038B000B0060020C0060020024A1368002BFCD18D
:1038C000704700BFB80600204FF4884038B5C4F2F6
:1038D000000040F2255107F011F800282BD14FF4D9
:1038E0008840C4F2000040F2277107F007F800B9E1
:1038F00038BD4FF48840C4F2000040F2277107F051
:1039000023F8234B1A68002A38D0224A224C116827
:10391000481C802808BF002054F8211010601A6845
:103920004FF48840013AC4F2000089B21A60BDE841
:10393000384006F0CDBF4FF48840C4F2000040F29A
:10394000255107F001F84FF48840C4F2000006F05A
:10395000C3FF124B1A687F2AC1D81149114D0A685A
:10396000C0B2541C7F2C45F8220098BF0C6001D9CE
:1039700000220A601A6801321A60B0E74FF48840EA
:10398000C4F2000040F22771BDE8384006F084BF61
:10399000B8060020C0080020B0040020AC040020BD
:1039A000B4060020C0060020F0B583B001A84FF493
:1039B0000065C4F2010506F0DDFB0420012106F0DC
:1039C000A5FD012402271026284601A9ADF80440D0
:1039D0008DF806708DF8076006F068FB042021461C
:1039E00006F094FD284601A9ADF804708DF8067024
:1039F0008DF8076006F05AFB0420214606F086FD8C
:103A0000284601A9ADF804608DF806708DF80760AE
:103A100006F04CFB28462146224606F0B9FB284614
:103A20003946224606F0B4FB28463146224606F0C7
:103A3000AFFB03B0F0BD00BFF8B5094D04460F461B
:103A4000002601E02B6833B92046FFF713FF00285A
:103A5000F8D00120F8BD0136BE422860F4D3F8BD8D
:103A6000A83900202DE9F04F85B0054603F00CFD84
:103A7000FFF722FFFFF7F4FE002843D00024624F37
:103A8000DFF888A10126A346294603A8FFF7D4FF43
:103A9000DFF874914FF001080346002835D0039BEE
:103AA0003E600A2B07D00D2BEED0FF2CECD80AF885
:103AB00004300134E8E70AF804B0002C32D103F0F6
:103AC000E3FCE1E7514852491A4607F0F8FB0028A9
:103AD0004CD04E484F49032207F0F1FB00284FD04D
:103AE0004A484D49052207F0EAFB002855D14B48CA
:103AF0004B49022207F0E3FB002849D10123C9F812
:103B00000830062005B0BDE8F08F4648019303F069
:103B10008DFC454803F08AFC444803F087FC019B78
:103B20001846EFE73F48019303F080FC374803F065
:103B30007DFC3E4803F07AFC34483D49022207F000
:103B4000BEFB38B131483B49052207F0B8FB18B934
:103B50000220D7E74046D5E72C483749022207F034
:103B6000AEFB019B0028ADD10320CBE709F13C005F
:103B700032490F2207F0BCFBC9F804800420C1E7DA
:103B800009F11C002E491F2207F0B2FB0520B9E7FE
:103B90000023C9F808300620B4E71C48294905224B
:103BA00007F08DFB98B119482749092207F087FBD8
:103BB00010B316482549042207F081FBA8B1134829
:103BC0002349092207F07BFB40B1FF209AE72148F7
:103BD00012490F2207F08CFB072093E71E481F496C
:103BE000FF2207F085FB0A208CE71D481D491F2294
:103BF00007F07EFB092085E71B4818490F2207F0D4
:103C000077FB08207EE700BFC4080020940A00204C
:103C100020DD00082CDD000830DD0008990A0020B6
:103C200038DD000800DD000804DD00080CDD0008B8
:103C300010DD000814DD00081CDD00089E0A0020CD
:103C4000970A00203CDD000844DD000850DD000834
:103C500058DD0008300A0020100900209D0A0020CD
:103C6000100A0020980A0020D0080020F0B583B088
:103C7000074607F01CFB06461A4803F0D7FBBEB107
:103C80003C46F61904E0184603F0AAFBB4420FD0F4
:103C900014F8013B6846A3F120055E2D12491A462F
:103CA000F1D907F0C1FA684603F0C0FBB442EFD186
:103CB0000E4803F0BBFB03F0E7FB3846FFF7C4FDFB
:103CC0000B48FFF7C1FDFFF7F7FD02E0022807D020
:103CD00020B10A20FFF7C6FE0128F7D103B0F0BDDE
:103CE0000020FBE764DD000878DD00086CDD0008DB
:103CF00040DF000838B539B10446451814F8010B07
:103D0000FFF77CFDAC42F9D1BDE83840FFF7D4BDE8
:103D100040F6C400C2F20000704700BF10B54FF477
:103D20000060C4F201000121002282B006F030FAE6
:103D30000C4A0521144600201368002BFCD00139E1
:103D40002060F9D101214FF40060C4F201000A465D
:103D500006F01EFA01A83221FFF76EFE0028F9D105
:103D600002B010BDA839002008B502460B4607482E
:103D7000074907F059FA0548FFF778FF20B1054BCE
:103D8000002283F83C205A6008BD00BF400A002092
:103D900080DD0008C408002008B502460B4607482D
:103DA000074907F041FA0548FFF760FF20B1054BCE
:103DB000002283F83C205A6008BD00BF400A002062
:103DC00090DD0008C408002008B5024608B1037859
:103DD00023B90748BDE80840FFF748BF0549064832
:103DE00007F022FA0448BDE80840FFF73FBF00BFD4
:103DF000BCE30008A0DD0008400A002030B54FF405
:103E0000E13083B003F0DAFBFFF7CEFD4FF4E13091
:103E1000FFF77CFC4FF40060C4F201001021002287
:103E200006F0B6F91F4C4FF400600022C4F2010006
:103E3000012106F0ADF9052522460023216800295D
:103E4000FCD0013D1360F9D101214FF400600A4616
:103E5000C4F2010006F09CF9124932222368002BBB
:103E6000FCD0013A0D60F9D14FF40060C4F20100BA
:103E70001021012206F08CF903E001A803F0E2FA18
:103E800060B901A8FFF7F6FC0028F6D0019803F00E
:103E9000A7FA01A803F0D6FA0028F2D00198FFF79C
:103EA000ADFCEEE7A839002008B50B4B1A6802B14B
:103EB00008BD01224FF4E1301A6003F07FFB074890
:103EC00003F0B4FAFFF770FD4FF4E130FFF71EFC8A
:103ED000BDE80840FFF722BF900A0020ACDD0008D3
:103EE00010B403781649FBB1002208601446013073
:103EF00005E001300E2A14DC10F8013C8BB13D2B9B
:103F000002BF01EBC20300F8014C5860F1D0262B30
:103F1000EFD1013200F8014C41F8320001300E2A95
:103F2000EADD531C0F2B08DC002201EBC300114615
:103F30000133815008320F2BFADD10BC704700BFEF
:103F4000E40B0020F8B50A4D0646002455F834303D
:103F5000E70031461846013423B107F096F918B14D
:103F6000102CF3D10348F8BD014BDF197868F8BD78
:103F7000E40B0020C8DE000808B5FFF7E3FF4DF6AC
:103F8000A461C0F6000107F080F9D0F1010038BF4C
:103F9000002008BD00B50B4685B04DF6AC61024669
:103FA000C0F60001684607F03FF96846FFF7CAFF10
:103FB00005B000BD10B5044607F079F9014600B917
:103FC00010BD2046BDE81040FFF794BE10B5044672
:103FD0004DF6B460C0F60000FFF7ECFF4DF6C4608C
:103FE000C0F60000FFF7E6FF4DF6CC60C0F600001B
:103FF000FFF7E0FF4DF6D860C0F60000FFF7DAFFEC
:104000004DF6E460C0F60000FFF7D4FF2046FFF74E
:10401000D1FF4DF6EC60C0F60000FFF7CBFF4DF688
:10402000F860C0F60000FFF7C5FF4DF60470C0F65B
:104030000000FFF7BFFF4DF61070C0F60000FFF75D
:10404000B9FF2046FFF7B6FF4DF61870C0F6000026
:10405000BDE81040FFF7AEBF38B504464DF62070FE
:10406000C0F600000D46FFF7A5FF2046FFF7A2FFB0
:104070004DF62C70C0F60000FFF79CFF2846FFF7B6
:1040800099FF4DF63070C0F60000BDE83840FFF7EC
:1040900091BF00BF4DF6C8604DF6447108B5C0F63B
:1040A0000000C0F60001FFF7D7FF4DF64C704DF64B
:1040B0005471C0F60000C0F60001FFF7CDFF4EF2CC
:1040C00060704DF65C71C0F60000C0F60001FFF7AD
:1040D000C3FF4DF668704DF66C71C0F60000C0F677
:1040E0000001FFF7B9FF4EF6DC004DF67071C0F627
:1040F0000000C0F60001FFF7AFFF4DF678704DF6F7
:104100008471C0F60000C0F60001FFF7A5FF4DF670
:1041100090704DF69C71C0F60000C0F60001FFF7EC
:104120009BFF4DF6A8704DF6B071C0F60000C0F6CA
:104130000001FFF791FF4DF6B870C0F60000BDE832
:104140000840FFF737BF00BF054A1368013313600B
:10415000DB0702D40348FFF72DBF0348FFF72ABF50
:10416000B00C0020D4DF0008BCDF000810B5044606
:104170004DF6DC70C0F60000FFF71CFF2046FFF78D
:1041800019FF4DF6E470C0F60000BDE81040FFF7DF
:1041900011BF00BF70B584B00C4605461B491646DA
:1041A00068461A4607F040F802A81849089A07F02E
:1041B0003BF83CB123782BB12046FFF7FBFE1448B7
:1041C000FFF7F8FE1348FFF7F5FE2846FFF7F2FE6B
:1041D0001148FFF7EFFE2846FFF7ECFE0F48FFF708
:1041E000E9FE3046FFF7E6FE0D48FFF7E3FE6846BE
:1041F000FFF7E0FE0B48FFF7DDFE02A8FFF7DAFE4F
:104200000948FFF7D7FE04B070BD00BFF8EA000808
:104210008CE60008ECDF000804E0000810E000086D
:104220001CE000082CE000082CDF000810B5044654
:104230004EF23800C0F60000FFF7BCFE2046FFF744
:10424000B9FE4EF26C00C0F60000FFF7B3FE4EF26E
:104250007C00C0F60000BDE81040FFF7ABBE00BF19
:1042600070B505460F480E46FFF7A4FE0E48FFF74F
:10427000A1FE002E0EDD043D00240C48FFF79AFE3F
:1042800055F8040FFFF796FE01340948FFF792FE38
:10429000B442F2D10748FFF78DFE074B00221A60A7
:1042A00070BD00BF84E00008D4DF0008A0E0000873
:1042B000B8E0000898E00008B00C00204EF2C800FA
:1042C000C0F60000FFF776BE38B504464EF2D800BF
:1042D000C0F600000D46FFF76DFE2046FFF76AFEB0
:1042E0004DF62C70C0F60000FFF764FE2846FFF77D
:1042F00061FE4EF20410C0F60000BDE83840FFF742
:1043000059BE00BF4EF2141008B5C0F60000FFF70A
:1043100051FE4EF22010C0F60000BDE80840FFF745
:1043200049BE00BFF0B5044683B01F481E460D4687
:104330001746FFF73FFE2046FFF73CFE1B48FFF7FE
:1043400039FE2046FFF736FE1948FFF733FE002EF0
:1043500024DD043D00240BE01648FFF72BFE55F842
:10436000040FFFF727FE1448FFF724FEB44215D0D0
:104370002246124901A806F057FF1148FFF71AFE1E
:1043800001A8FFF717FE0F48FFF714FEBC4204F127
:104390000104E1D10C48FFF70DFEDDE70B48FFF704
:1043A00009FE03B0F0BD00BF2CE1000804E00008E6
:1043B0003CE1000838E200086CE10008F8EA000877
:1043C00050E1000818E0000860E1000844E100083E
:1043D00070B50E4605460E481446FFF7EBFD304615
:1043E000FFF7E8FD0B48FFF7E5FD2846FFF7E2FD84
:1043F0000948FFF7DFFD14B10848FFF7DBFD084867
:10440000FFF7D8FD0748BDE87040FFF7D3BD00BFF8
:10441000DCDF000878E100089CE10008B0E100085A
:1044200038E20008E4DF00082DE9F041069F044669
:1044300016469846079D11B10B78002B49D12848A4
:10444000FFF7B8FD2046FFF7B5FD2648FFF7B2FDA0
:104450002046FFF7AFFD2448FFF7ACFD3046FFF7DD
:10446000A9FD2248FFF7A6FD4046FFF7A3FD20481F
:10447000FFF7A0FD3846FFF79DFD55B12B7843B1FE
:104480001C48FFF797FD2846FFF794FD1A48FFF7F1
:1044900091FD1A48FFF78EFD2046FFF78BFD184867
:1044A000FFF788FD2046FFF785FD1648FFF782FDE0
:1044B0001548FFF77FFD2046FFF77CFD1348FFF707
:1044C00079FD3046FFF776FD1148BDE8F041FFF772
:1044D00071BD0846FFF76EFD0E48FFF76BFDAEE7B6
:1044E000B8E1000804E0000810E00008D4E100088A
:1044F000DCE10008E4E10008F4E10008F8E100086C
:1045000004E2000814E2000820E2000830E200089B
:104510003CE200088CE600084EF24820C0F600009D
:104520000321FFF7E7BB00BF10B504464DF6DC7072
:10453000C0F60000FFF73EFD4EF24C212046C0F6CB
:104540000001FFF7C1FE4EF27C00C0F60000BDE89E
:104550001040FFF72FBD00BF70B506464DF6DC706A
:1045600082B0C0F600000D461446FFF723FD4DF65D
:10457000C8614EF25423C0F60001C0F60003304675
:10458000009301912A462346FFF74EFF4EF27C002E
:10459000C0F6000002B0BDE87040FFF70BBD00BFE1
:1045A00038B505460C46FFF7CFFD2846FFF7DEFD80
:1045B0002046FFF7DBFD4DF6C860C0F60000FFF7B0
:1045C000D5FD4EF29800C0F60000BDE83840FFF778
:1045D000F1BC00BF10B504464EF25820C0F60000F2
:1045E000FFF7E8FC2046FFF7E5FC4EF23C10C0F672
:1045F0000000BDE81040FFF7DDBC00BF10B5044669
:10460000FFF7A2FD2046BDE81040FFF7E3BF00BF63
:104610004EF27820C0F60000FFF7CCBC08B5FFF7DB
:10462000F7FF4EF29800C0F60000BDE80840FFF723
:10463000C1BC00BFF0B50E4683B014461F46089DAE
:10464000FFF7DCFF3046FFF791FD4DF6DC70C0F65A
:104650000000FFF7AFFC4DF6C861C0F600013A4616
:104660002B4620460095FFF795FD4DF6E470C0F609
:104670000000FFF79FFC2046FFF7D8FD03B0BDE820
:10468000F040FFF7CBBF00BFF8B5069D0E461446BD
:104690001F46FFF7B3FF3046FFF768FD2046394657
:1046A0002A46FFF795FE2046FFF7C0FDBDE8F8401B
:1046B000FFF7B4BF2DE9F0410F4614469846069E19
:1046C000079DFFF79BFF3846FFF750FD4DF6DC7066
:1046D000C0F60000FFF76EFC414632462B462046EE
:1046E000FFF720FE4DF6E470C0F60000FFF762FC15
:1046F0002046FFF79BFDBDE8F041FFF78FBF00BFED
:104700002DE9F04F83B08B46924699460C9D0D9F44
:10471000FFF774FF1148FFF729FD1148FFF74AFC26
:10472000DFF8488000242E595BF8040033463E59D8
:104730005AF8041059F804208DE84001FFF774FE80
:1047400004340848FFF736FC0C2CECD10648FFF780
:104750006DFD03B0BDE8F04FFFF760BF84E20008D5
:104760008CE2000898E2000844E9000894E200089E
:104770002DE9F04F05460E46C5B0A9482946934697
:1047800002F00CFF33781BB3741C4FF02008002795
:1047900006E02B2B08BF04F8018C14F8013BBBB1D9
:1047A000252BF6D120460221FBF7DCFDA27804F888
:1047B000010C002A00F04885234603F8012B9A7863
:1047C0001946002AF9D10F7014F8013B002BE7D1EC
:1047D0003146944802F0E2FE3046FFF781FB28465E
:1047E000914906F052FD002842D028468F4906F034
:1047F0004CFD0446002800F0D38328468C4906F07F
:1048000044FD002800F0788428468A4906F03DFDE2
:104810000446002800F097812846874906F035FDB8
:10482000002800F071852846844906F02EFD0028F6
:1048300000F0E8872846824906F027FD002800F0AE
:10484000518228467F4906F020FD002800F0FE86B0
:104850007D48FFF7AFFB7D48FFF7ACFB7C48FFF7D7
:10486000A9FB0026FFF758FE304645B0BDE8F08FA3
:10487000784C18AF3CAD04F1080694E803000395AA
:1048800087E803000FCE0FC596E8030023AA04F1C2
:104890002006914685E8030007920FCEA9E80F0095
:1048A000366828AD04F1480C06970DF1C8082DAF05
:1048B000C9F80060049504F1340EE2462E464446E1
:1048C0003D46BEE80F000FC6BCE80F000FC5BAE8B2
:1048D0000F000FC4DCF80030DEF800202B602360EE
:1048E00013A912A81AAC0DF158090DF1500A11AD17
:1048F00032603A910594CDF8DC9038953990CDF836
:10490000ECA002F09FFF089002F0A2FF5249C0F312
:104910000742C0F30723059806F086FC02F09EFFCD
:1049200042690446002A32DB0369002B2FDBC16891
:1049300000292CDB8068002829DB6568002D26DB38
:10494000B2F5966F23DC0C2B21DC1F291FDC172806
:104950001DDC3B2D1BDC02F26C7248463F4906F021
:1049600063FC226911A801323D4906F05DFCE26852
:1049700012A83B4906F058FCA26813A8384906F073
:1049800053FC50463649626806F04EFC0AE00023AC
:104990008DF858308DF844308DF848308DF84C3013
:1049A0008DF850302F48FFF7CDFA0546002801F06A
:1049B00074802D4906F069FC002841F03F802B4CA3
:1049C00049262B48FFF702FBDFF8BCA0FFF762FB8C
:1049D00006980221FFF744FC26480899FFF7E0FDFE
:1049E000DAF80030244A25492548002B18BF114623
:1049F000FFF7D6FDDAF80030002B41F01980FFF701
:104A00005DFC03980621FFF72BFC1E48FFF7F6FD1F
:104A10004FF0000A05950394079DDDF810B038E0CB
:104A20002CE4000840E4000858E4000880E5000891
:104A3000F4E60008D8E7000860E8000898E90008F4
:104A400054EA0008FCEA000848EB0008C4DE00084D
:104A500060EB0008C0DD00085CE4000868E40008C2
:104A60006CE4000874E400087CE40008B0E200088C
:104A7000CCE40008D8E4000864F3000800E3000870
:104A8000E0E40008C8DE0008A404002037AB5AF8B0
:104A900003907548FFF78EFA58F80A4055F80A0057
:104AA0005BF80A1057F80A304A460094FFF772FB89
:104AB0000AF1040A6D48FFF77DFABAF1140FE5D147
:104AC0006B48039C059DFFF7B1FBFFF7A7FDFFF7C0
:104AD000F5FB06980221FFF7C3FB66481E27034635
:104AE000654A66490097FFF7A5FDFFF7E7FB6148B8
:104AF000FFF770FD62486349FFF7E6FB62486349D0
:104B0000FFF7E2FB62486349FFF7DEFB6248634957
:104B1000FFF7DAFBFFF77CFD44B16148FFF74AFA83
:104B20002046FFF747FA5F48FFF744FA28465A49FC
:104B300006F0ABFB0446002800F0DD84FFF7E2FB43
:104B4000FFF7EAFC90E6584B3CAD93E80300039571
:104B500085E80300FDF77AFD80465448FFF7F2F937
:104B60000546002801F00282514906F08EFB0646F8
:104B7000002801F04C8128464E4906F086FB064687
:104B8000002801F00A8028464B4906F07EFB0546C6
:104B9000002841F0E7814948FFF7EEF910F10008DD
:104BA00018BF4FF00108CBF800804C2600238DF889
:104BB000B4300A24FBF76EFB0DF13200FBF77AFBF1
:104BC000002841F00E810A20FBF73AFF013CF3D1A7
:104BD00044AF3F2327F85C3D02F054FA384982B2D3
:104BE00032A806F021FB02F053FA354982B237A809
:104BF00006F01AFB3348FFF7E9F9FFF74BFA039881
:104C00000221FFF72DFB30483946FFF7C9FC2F483A
:104C100032A9FFF7C5FC2E4837A9FFF7C1FC274A88
:104C20002C4B29492C48CDF80080FFF72DFDFFF7CC
:104C300045FB2948FFF7CEFC1D482849FFF744FBF8
:104C40001C482749FFF740FBFFF7E2FC002D3FF42B
:104C500075AF1348FFF7AEF92846FFF7ABF91148D7
:104C6000FFF7A8F96AE700BFDCDF0008E4DF00080F
:104C70009CE40008C8DE0008C4E40008F8E400086A
:104C800084E4000800E500088CE400080CE5000856
:104C90007CE4000818E5000830E500083CE5000861
:104CA00048E50008E8E60008C0DD000874E40008F4
:104CB000E0E70008E8E70008F0E70008F4E700088C
:104CC000FCE7000800E800086CDF000810E80008B6
:104CD00014E8000818E8000868DF000830E8000859
:104CE00048E800083CAD039523AD924A079528ADEE
:104CF0000495039D02F150031EAC02F1180702F166
:104D00000C0E02F1240602F1300A07CA84E80700FB
:104D10000FCB85E80F009EE80700079DDFF878C2FB
:104D200085E8070097E80700049D0DF1C80885E8AD
:104D3000070096E8070088E807009AE80700DCF813
:104D400000300DF1DC0989E807007B4F53B97B4D3A
:104D50003B6A39683A69386B85E80E000123E860E0
:104D6000CCF80030FDF706FC0690FDF71DFC059021
:104D7000FDF728FC0890FDF7D9FB00F00200099030
:104D8000FDF78CFF8246FDF761FC0A900DA8FDF748
:104D900039FF6B48FFF7D6F80546002800F0028778
:104DA000684906F072FA0346002801F08780284619
:104DB000654906F06AFA0346002801F0FD8028469E
:104DC000624906F062FA0346002801F0A9812846EC
:104DD0005F4906F05AFA0646002801F0E7822846A5
:104DE0005C4906F052FA0646002801F0D4822846B3
:104DF0005949072206F063FA0646002801F0B482FA
:104E000028465649042206F05AFA0646002801F0C0
:104E100056832846524906F038FA0026B34610B9A0
:104E2000DFF878B153267A6B4E4913A806F0FCF9E7
:104E30004C49059A14A806F0F7F94A49089A16A8A9
:104E400006F0F2F9524647490EA806F0EDF90DF1C9
:104E5000400A44499DF834200FA806F0E5F911AF47
:104E600040499DF83520504606F0DEF99DF8362081
:104E70003C49384606F0D8F903250FA93A482D9148
:104E8000CDF8B8A02F97FFF7A1F8FFF703F9204658
:104E90002946FFF7E5F935483549364A14AB009500
:104EA000FFF7C8FB009531483349344A16ABFFF78A
:104EB000C1FB099C5CB90A9D002D01F01F818DE8A2
:104EC00000032A480799049A2DABFFF719FC069FA7
:104ED00004242B4A194B25482A4901940097FFF7CF
:104EE000E9FBFFF7EBF921460398FFF7B9F9264DE7
:104EF00000242B68DA0700F1958601341035042C64
:104F0000F7D1FFF7DBF91948FFF764FB14481F4995
:104F1000FFF7DAF9FFF77CFBBBF1000F3FF40EAEB1
:104F20001B48FFF747F85846FFF744F81948FFF7C2
:104F300041F803E624DE00082C000020680C002065
:104F400074E4000888E8000898E8000860EA0008AF
:104F500070EA000880EA000890EA0008A0EA000869
:104F6000E4E80008F8EA0008A8EA000890DF000872
:104F7000BCEA000874EA0008C4EA000884EA0008F1
:104F800064EA0008DCEA0008380000208CE9000828
:104F900048E50008E8E60008640C00200CE400087E
:104FA000AB4A3CAD02F108030DF1DC0992E80300C5
:104FB000039589E8030093E8070085E80700FEF7FA
:104FC000A7FE0546A348FEF7BDFF05F10C08824683
:104FD000AF68002800F0EB879F4906F056F90646B7
:104FE000002800F04A8650469C4906F04EF90646D5
:104FF000002800F0FF865046994906F046F906461B
:10500000002800F013875046964906F03EF9002824
:1050100000F047852646B24604F044FC9249024619
:1050200032A806F001F99148FEF7D0FFFFF732F8F9
:1050300003980321FFF714F905F13C018C48FFF7B1
:10504000AFFA41468B48FFF7ABFA8B48FFF7D6FA29
:105050008A48FFF78BF88A48FEF7ACFF4FF00F083D
:10506000884849463A460223FFF75CF905F11C02DD
:10507000854920238548CDF80080FFF78BF814255B
:105080008348FEF797FF8349834A4023834800956E
:10509000FFF780F88248FEF78DFF8248FFF7C6F8D9
:1050A000FFF7BCFA04F020FC032503467E49724852
:1050B0007E4ACDF80080FFF7BDFA7D497D4A32ABCC
:1050C0006D480095FFF7B6FAFFF7F8F86A48FFF762
:1050D00081FA64487849FFF7F7F8FFF799FA002C4E
:1050E00000F07F857548FEF765FF2046FEF762FFFA
:1050F0007348FEF75FFF21E5724B0DF1C80893E896
:10510000030088E803005348FEF71CFF044600280C
:1051100000F0DA846C4906F0B8F80646002800F082
:1051200056862046694906F0B0F80646002800F089
:105130008C862046664906F0A8F8002840F0C48412
:10514000644D5726644B1B68002B00F0628504F009
:10515000C5FA0DF1DC09044662084846424906F0EA
:1051600063F8E70700F1B886484606F0A0F85B4B05
:1051700009EB000201469C8818689B7949F80100F8
:1051800094809371564B1B68002B00F0398504F016
:10519000C5FA3CAF0446620838463349039706F027
:1051A00043F8E40700F1A586039806F080F8039C15
:1051B0004A4B2218039F01469C8818689B797850B7
:1051C0009480937104F07AFA0246002840F0CE856C
:1051D00044AF07F85C0D04F0F1FA0246002840F0F5
:1051E000668544AC04F8700D04943E48FEF7EEFE6C
:1051F000FEF750FF40460221FFF732F83A48494691
:10520000FFF7CEF9022439480399FFF7C9F9384866
:105210003849394A3B460094FFF70CFA3749384A77
:10522000049B33480094FFF705FAFFF747F830482E
:10523000FFF7D0F926483349FFF746F8FFF7E8F9BA
:10524000002D7FF406AD79E421460F70FFF7BCBA5C
:105250001CDE000874E400088CE5000828E600085D
:1052600038E6000848E60008F8EA0008ACE500085F
:1052700050E600085CE600084CDF000870E6000815
:10528000DCDF000898E5000878E60008A4E50008DF
:1052900080E6000894E60008C8DE000870F4000804
:1052A000E4DF000890E5000898E600082CE6000816
:1052B000A4E600083CE60008B8E60008C8E60008D6
:1052C000E4E60008C0DD000804E7000814E7000871
:1052D00024E70008C4E30008541300203CE700085A
:1052E0009004002044E700085CE700086CE7000831
:1052F00060E7000874E7000808E700089CE700087A
:1053000018E70008C4E70008A84B23AC07943CA8A2
:1053100003F10C0E03F1240503F13004039003F1B3
:10532000180693E8070028AF079B049783E8070057
:105330009EE80700049B2DAF0DF1DC0983E8070010
:1053400096E8070087E8070095E8070089E8070066
:1053500094E80700039C84E80700FDF741F90890F2
:10536000FDF7E4F80546FDF7C5F90990FDF76EFC79
:105370008046FDF76BF98E4C0A9013A8FDF71EFCD2
:10538000236805F00102C5F3400A069253B9894A21
:105390008948191849680833902B42F8041FF8D13E
:1053A000012323608548FEF7CDFD0446002800F068
:1053B000F785834905F069FF002800F04C832046FB
:1053C000804905F062FF002840F0B2857E48FEF774
:1053D000D3FD002800F02E86012045F0020505903F
:1053E000CBF8005047262046784905F04EFF054689
:1053F000002800F059852046754905F046FF002831
:1054000040F08285DFF840B2724B58260DF1500A09
:10541000424671495046029305F006FF6F4A6E49B5
:1054200052690DF158081CA805F0FEFE18AD6A4936
:105430009DF84C20404605F0F7FE1AAC66499DF8F1
:105440004D20284605F0F0FE9DF84E20204662498A
:1054500005F0EAFE029BCDF8C8801A6833953494B3
:10546000002A40F00E8544AC04F8982D5C48FEF705
:10547000ADFDFEF70FFE07980321FEF7F1FE069D36
:1054800058485949594A5A4B0095FFF7FDF8089D6D
:105490005448009512255749574A584B0195FFF734
:1054A00009F9059D4F4800955549474A554BFFF767
:1054B000EBF80A9D002D00F0D284099D002D00F02C
:1054C000E78423460224504A504951480094FFF78C
:1054D000B1F8FEF7F3FE4348FFF77CF84D484E491C
:1054E000FEF7F2FE4D484E49FEF7EEFE38484D49B4
:1054F000FEF7EAFE0AE54C48FEF75CFDA0461CAD4F
:105500001EAC42464949284605F08EFE2846FEF765
:1055100051FD4748FEF74EFD404621461022FEF75A
:10552000A9F800283DD000270DE0E25D414928465A
:1055300005F07AFE2846FEF73DFD01373E48FEF7AE
:1055400039FD102F0AD007EB0803B3F5A27F3B48C3
:10555000EBD90137FEF72EFD102FF4D13648FEF7B8
:1055600029FD002320212E2003EB0802B2F5A27FA3
:1055700088BFE15404D8E25C203A5E2A88BFE05438
:105580000133102BF0D1002320468DF8883008F12C
:105590001008FEF70FFD2A48FEF70CFDB8F5A87FAE
:1055A000AFD12848FEF706FDFFF7C8BA24DE000891
:1055B000780C0020940B002070DC000874E40008D4
:1055C0006CE8000878E800087CE80008C8E80008F3
:1055D000D8E8000830030020F8EA00086C01002039
:1055E000ECE80008DCE8000800E9000870E80008C2
:1055F00008E9000828E90008BCE80008980B00202A
:105600009CDF000838E90008CCE8000864E90008DD
:1056100060E7000884E4000800E500088CE4000866
:105620000CE500087CE9000860E5000868E5000872
:1056300070E500084CF20008ACE100087CE50008C9
:1056400040DF000874E50008F8E30008B44D3CAC06
:1056500003940FCD0FC495E80F0084E80F00B14804
:10566000FEF770FC044630B1AF49062205F027FE74
:10567000002800F02D82DFF834B30DF1DC09AB48CF
:10568000FEF7A4FC23ACFEF705FD03980821FEF706
:10569000E7FD18AD07941AAC4FF0000A0695059483
:1056A00028AD1EAC049556462DAF0DF1C8081CADB3
:1056B00003940BEB0A0CDCF8042048F68904C8F6C6
:1056C0008804A4FB02029A4952090598CDF808C043
:1056D00005F0AAFDDDF808C09549DCF80420A4FB1C
:1056E00002035B09C3EB0313A2EB8302284605F018
:1056F0009BFD9048FEF782FF32468F49069805F0E1
:1057000093FD32468D49039805F08EFD32468C4953
:10571000079805F089FD32468A49049805F084FD12
:1057200032468949384605F07FFD32468749404672
:1057300005F07AFD0698FEF719FD5BF80A20079838
:105740008349C2F3C012FEF743FE5BF80A2080498A
:10575000C2F380120498FEF73BFE32467D4948466C
:1057600005F062FD5BF80A207B48C2F3C204FEF735
:1057700021FC0723224679494846FEF7D3FD7848A5
:10578000FEF718FC32467749484605F04DFD5BF8B8
:105790000A20714802F00704FEF70CFC224607239A
:1057A0006E494846FEF7BEFD6D48FEF703FC022435
:1057B0006948FEF7FFFB6649059A23463846009480
:1057C000FEF7E8FC6648FEF7F5FB6348FEF7F2FBE0
:1057D0005F492A46234640460094FEF7DBFC6048BA
:1057E000FEF7E8FB01360398FEF720FDFEF716FFF3
:1057F000082E0AF1080A7FF45CAFFEF75FFD002671
:10580000FFF79CB9DFF8A8E13CAF3E460EF13C043F
:105810000DF1C8089EE8070088E807000FCC0FC606
:10582000514D039724682F680DF1DC090EF1500EDD
:105830009EE80F00346089E80F00002F00F01B8104
:105840004A4EFCF71FFF0746FCF754FF0546354854
:10585000FEF778FB0446002800F0E983444905F090
:1058600014FD8246002800F0D7822046414905F009
:105870000CFD8246002800F0838320463E49032227
:1058800005F01DFD8246002800F06B8420463B4950
:10589000062205F014FD8346002800F02E852046E0
:1058A0003749072205F00BFD0646002800F01B854E
:1058B00020463449042205F002FD0646002800F087
:1058C0005D852046304905F0E0FC0026B24610B95F
:1058D000DFF8E0A053262D48FEF778FB0B24FEF7F7
:1058E000D9FB40460321FEF7BBFC294829492A4A37
:1058F0002A4B019400970224FEF7DCFE2849294A2E
:10590000294B234800950194FEF7D4FEFEF7D6FC00
:1059100003980521FEF7A4FC144D002451E000BFBC
:1059200084DE000874E4000804EB00081CEB0008A7
:105930006CE40008A8DF0008F8EA000830EB000873
:1059400038EB00083CEB000840EB000844EB000893
:10595000C8DE000814EB0008DCDF000800000020AF
:10596000E4DF000818EB0008E00B002078000020BE
:10597000A4E90008B4E90008C8E90008CCE9000877
:10598000E4E90008F4E90008E4E80008FCE900089C
:1059900078DF000814EA0008A8E90008840C002059
:1059A00020EA0008B8E900087C0C0020D03900206B
:1059B00024DE00080CE40008013414350B2C00F040
:1059C000F5802B69D807F7D52246BD4918A805F000
:1059D0002BFC2246BB491AA805F026FC2246BA49F0
:1059E0001CA805F021FC2246B8491EA805F01CFCA5
:1059F000AA68B74916A805F017FCB648FEF7FEFDE1
:105A00002868FEF7B3FB16A91AA8B34AFEF7A4FD4F
:105A10001CA8FEF789FD2A69B049C2F340021EA8FE
:105A2000FEF7D6FC18A8FEF701FCFEF7F7FDC3E76A
:105A3000AB480599FEF7B4FDFEF7E1BF2846A9493A
:105A400005F023FC002832D10123CBF8003050268A
:105A5000A54CFEF7B6BFA548FEF78EFA002800F069
:105A60006382012345F001050693CBF80050CDF881
:105A700014A04726B7E49E4A9E4E3B4699591433DC
:105A8000DC2B42F8041FF9D19B4B9C491A681B6917
:105A900081E80C0001232B60D3E606460446FEF79E
:105AA00090BFDFF8C0A24E260446FFF7B5BA2846DD
:105AB000934905F0EAFB002840F04083CBF8000052
:105AC0005026904CFEF77DBF00263546FFF73ABBC7
:105AD000A01D05F063F8072804463FF6CCAD01464B
:105AE0008948FEF757FA894905F0CFFB002800F0F6
:105AF000F183DFF874B25BF8343023F080034BF8A5
:105B0000343021468248FEF745FA804905F0BDFB56
:105B1000002800F0D8835BF8343023F040034BF8C2
:105B200034300DF1DC0922467A49484605F07CFB09
:105B30004846FEF707FA05F031F822467649054651
:105B4000484605F071FB4846FEF7FCF905F026F8DB
:105B50005BF83430ED0000F0070023F03F0340EA2B
:105B6000030205F0380313434BF8343021466B48E9
:105B7000FEF710FA05F012F8214605466848FEF7D0
:105B800009FA05F00BF8C5EB05150BEBC40400EBA7
:105B90008500606003F060F871E501F09BFA614DEB
:105BA000FFF704B806468346FFF73DB9FEF786FBCC
:105BB00048460421FEF754FB5B4D00242B68D907AF
:105BC00000F1DB8001341035022CF7D1FEF776FBB3
:105BD0004048FEF7FFFC55485549FEF775FBFEF7B8
:105BE00017FDBAF1000F3EF4A9AF5248FEF7E2F9F3
:105BF0005046FEF7DFF95048FEF7DCF9FEF79EBF8E
:105C00004E4B3CAC93E80300039484E80300FFF799
:105C1000D9BA4A4B0DF1DC0993E8030089E8030087
:105C2000FFF7B0BA2246464918A805F0FDFA224609
:105C300044491AA805F0F8FA224643491CA805F081
:105C4000F3FA55F8082C224912A805F0EDFA3F485E
:105C5000FEF7D4FC55F80C0CFEF788FA12A93C4A62
:105C60001AA8FEF779FC1CA8FEF75EFC18A8FEF740
:105C7000DDFAFEF7D3FCFFF740B93648FEF762F9CC
:105C800004F08CFF07463448FEF75CF9824633483F
:105C9000FEF758F90446002F00F0AF8105F007FB2E
:105CA000092800F2CC812E4CB246FFF7B5B928ACDA
:105CB00020460749049405F0B7FAFFF796BA00BFEB
:105CC00030EA0008D4E9000838EA0008DCE90008F6
:105CD000F8EA000878DF000840EA0008C8DE00089B
:105CE000E8E4000884E40008D0E2000870E8000856
:105CF000800C0020780000206C0100207C0C00202B
:105D00008CE40008E8E200080CEB0008A4DE0008C0
:105D100010EB000814EB000818EB0008B4E40008CE
:105D200048EE0008E0E3000878010020E4E80008FD
:105D30008CE9000848E50008E8E6000800E30008F0
:105D4000ECEA000898EA0008F4EA000890DF00088E
:105D500060E9000898E50008A4E5000870F4000870
:105D600008E30008B0E30008D03900202DAF384622
:105D7000BF4905F059FAFFF72EBA2246BD4923A8BC
:105D800005F052FA2246BC4928A805F04DFA2246F1
:105D9000BA492DA805F048FA55F8082CB44914A8BA
:105DA00005F042FAB648FEF729FC55F80C0CFEF750
:105DB000DDF914A9B34A28A8FEF7CEFB2DA8FEF7FB
:105DC000B3FB23A8FEF732FAFEF728FCFAE6AE484A
:105DD000FEF7B8F804F0E2FE03F076FC3546FFF774
:105DE000B1B92DAF3846A949BDF8322005F01CFAEB
:105DF000FEF7F2BEA648FEF7A5F803F07BFD0028EB
:105E000000F0B8803446DFF8E0A2FFF705B901F0F2
:105E100045F9A04DFEF7CABE9F48FEF793F804F07F
:105E2000BDFE41260746CBF8000054E59B48FEF72F
:105E300089F804F0B3FE03F03BFD002800F0AA80CF
:105E40003446DFF8A8A2FFF7E7B89548FEF77AF8DE
:105E500004F0A4FE03F0B8FC3546FFF773B9884898
:105E6000FEF7CCFB8F48FEF781F95146854A8E48F4
:105E7000FEF772FB8C48FEF7D9F9FEF7CFFBFFF770
:105E80001CBB1EAC20467A4905F0CEF9FFF7EEBAEE
:105E9000039DCDF800900195794804993A4632ABBC
:105EA000FEF72EFCFFF70DBB8048FEF74BF804F021
:105EB00075FE7F4BAB461860FFF7A8BA7A4802938D
:105EC000FEF740F804F06AFECBF80000029B824621
:105ED00062269B46FEF7A7BF484605F0E8F9754BDA
:105EE00009EB000219889B7829F800109370FFF7DE
:105EF0003BB9039805F0DBF96E4B3A1819889B788B
:105F000039529370FFF750B920466B4905F0BDF93F
:105F1000002840F045810123CBF800305026DFF8FF
:105F2000D0B1634BFFF772BA25F0010506909CE5EE
:105F30002046624905F0A9F9002800F02481204696
:105F40005F4905F0A2F9002800F09D8120465D49D7
:105F500005F09BF9002800F03281CDF814A000264E
:105F6000FFF741BA26462546FEF720BE06460546FF
:105F7000FEF71CBE06460446DFF878A1FFF74CB8D2
:105F80005148FDF7DFFF04F009FE46260546CBF831
:105F90000000A0E406460446DFF85CA1FFF73CB829
:105FA0000646CDF814A08346414BFFF72FBA0646AC
:105FB00004468246FFF730B844480293FDF7C2FF1B
:105FC00004F0ECFD8DF834004148FDF7BBFF04F010
:105FD000E5FD8DF835003F48FDF7B4FF04F0DEFD28
:105FE0008DF836000D9A6326110CABF800208BF863
:105FF0000210029B9B46FEF716BF3748FDF7E6FFEF
:106000003648FDF7D7FFFEF77DF9FEF785FA4FF426
:10601000FA70FAF715FD324B6F6085F83C70504608
:1060200021461F603E46FDF79FFEFEF71DBC06465B
:10603000824650E425F002050590FFF7D1B92648C5
:10604000FDF7C4FF2748FDF7B5FFFEF75BF9FEF744
:1060500063FA4FF4FA70FAF7F3FC214B6E6085F89F
:106060003C60504621461E60FDF796FEFEF7FCBBE5
:10607000F8EA000844EA0008ECE900084CEA0008E5
:10608000DCE8000860E9000808E70008FCE7000811
:106090002CE60008E0E30008A8E900083CE6000858
:1060A00018E700084CE90008B4F70008CCE800083D
:1060B0003003002038E7000884E4000888E800087E
:1060C00098E80008B8E80008B8E90008A4E8000863
:1060D000A8E80008B0E80008ACE50008C0E5000842
:1060E00074120020F4E5000828E3000870E30008BB
:1060F000D0E200084CE3000890E30008BE48FEF739
:106100007DFABE48FEF732F80EA9BD4ABD48FEF73B
:1061100023FABC48FEF78AF8FEF780FAFEF7CFBEF6
:10612000B9480293FDF70EFF04F038FDCBF80000EC
:10613000029B069064269B46FEF775BE2846B3492F
:1061400005F0A3F80990002846D02846B04905F08C
:106150009CF80446002800F0438100263446FEF7F0
:1061600030BCE01C04F01AFD0A2884BF5646B24633
:106170003FF6B1AB00EB800006EB8003DA685646D1
:106180009A60FFF7A8BB9F48FDF7DCFE04F006FD10
:1061900042268046CBF80000CDF814A0FFF723B9C3
:1061A00020469C4905F071F8002840F00A81CBF8A0
:1061B00000005026DFF8B0B2974BFFF727B9974899
:1061C000FDF7C0FE04F0EAFC44260890CBF800007E
:1061D000CDF814A0FFF707B99148FDF7B3FE04F01E
:1061E000DDFC06468F48FDF7ADFE04F0D7FC034604
:1061F0008D480293FDF7A6FE04F0D0FC04468B48C0
:10620000FDF7A0FE04F0CAFC0A908948FDF79AFE4B
:1062100004F0C4FC32460B908649484605F004F869
:10622000029B85491A4611A804F0FEFF22468249C6
:1062300012A804F0F9FF80490A9A13A804F0F4FFA9
:106240007D490B9A504604F0EFFF029BA6F26C7159
:106250005A1E0A98CBF81C10CBF810200B99099AFB
:10626000CBF80C40CBF80800CBF80410CBF800209A
:10627000204632461946FAF73BF85426CBF8180068
:10628000099CFEF79EBB6D48FDF75CFE04F086FCA2
:106290008DF84C006A48FDF755FE04F07FFC8DF840
:1062A0004D006848FDF74EFE04F078FC8DF84E0076
:1062B000139BCDF814A01A0CABF800308BF8022019
:1062C0004326FFF790B85BF8343043F040034BF8B7
:1062D000343026E4DFF894B15BF8343043F08003C7
:1062E0004BF834300DE4E01D04F058FC012804465E
:1062F00040F2BE80B246FFF7EEBAA01D04F04EFC9D
:106300000A2888BF5E46824688BFB2463FF6E3AAA7
:106310004D4952461EAC1AA804F086FF52464B491E
:10632000204604F081FF1AA8FDF70CFE04F036FCAD
:10633000431E0E2B4FEA8A0B9EBF0BEB0A0306EBA4
:10634000830398602046FDF717FE0BEB0A0306EB6C
:1063500083031A69002800F0BF80002642F0020281
:106360001A61B246FFF7B7BAE81D04F017FC03281C
:10637000054640F29180B346FEF755BD201D04F05E
:106380000DFC0128B6D8324BB24603EB00139A68D5
:106390005A60FFF7A0BA2F48FDF7D4FD04F0FEFBCA
:1063A000FCF716F9B3460890FEF73DBD2A48FDF705
:1063B000C9FD04F0F3FBFCF7FDF8B3460590FEF7CA
:1063C00032BD2046254904F060FF254B00280CBF54
:1063D0009B464FF0000B08BF53260F4BFFF716B834
:1063E0002048FDF7AFFD1E220146584604F080FF0D
:1063F0007026FEF7E6BA00BF90DF00084CE90008FF
:1064000060E90008B4F7000864EA000898E40008AE
:10641000C0E400088CE4000830030020BCE8000859
:10642000A8E40008B0E40008B8E4000860F7000839
:10643000BCE4000868E400086CE40008A4E8000874
:10644000A8E80008B0E80008D4E90008DCE9000882
:106450006C01002084EA000874EA0008E4E80008FF
:106460000CE40008C4E40008E8E20008D039002089
:1064700002461D4928A804F0D7FE28A8FDF762FDB2
:1064800004F08CFB0F283FF635AF184BB24603EBF8
:1064900004146060FFF71FBA024615491AA804F0F9
:1064A000C3FE1AA8FDF74EFD04F078FB0F283FF657
:1064B00062AF07EB05156860B346FEF7B4BC281D54
:1064C00004F06CFB03283FF656AF07EB00139A6805
:1064D000B3465A60FEF7A7BC22F0020206461A61D4
:1064E0008246FFF7F8B900BFECE900086C01002014
:1064F00098EA000830B585B04FF48044684603F050
:1065000019FF0022200448F2A063C0F20103012118
:10651000ADF80420ADF8082040F4A8404FF48062A4
:106520004BF6FF75ADF80650ADF80A20ADF80C40FB
:10653000009303F00DFF200440F4A840694603F0E7
:1065400089FE05B030BD00BF10B54FF4A844C4F2B9
:1065500000042046012103F017FF2046012103F02B
:106560003FFF2046002103F03BFF204603F052FE90
:10657000BDE81040FFF7BEBF70B505460E4643F2BA
:10658000010401E0013C13D04FF4A8402946C4F2B5
:10659000000003F033FF0028F4D04FF4A840C4F209
:1065A0000000314603F02AFF0028EBD0012070BD27
:1065B000FFF7CAFF204670BD38B5054619B1BDE8E2
:1065C0003840FFF7D9BF43F2010401E0013C0AD093
:1065D0004FF4A840C4F20000294603F00FFF002842
:1065E000F4D0012038BDFFF7AFFF204638BD00BF13
:1065F000F8B507464FF4A840C4F200000E4601214A
:1066000015461C4603F0B2FE0120C1F20000002135
:10661000FFF7D2FF002832D04FF4A840C4F20000A8
:1066200034BB012103F0BEFE4FF4A844C4F20004C1
:106630002046F9B2002203F0C9FE0220C1F2000098
:106640000021FFF7B9FFB8B18020C1F2000000219E
:10665000238BFFF7B1FFA8B125B1C6F30721204670
:1066600003F0AEFE2046F1B203F0AAFE0020F8BD12
:10667000002103F097FED7E76FF00100F8BD4FF05F
:10668000FF30F8BD6FF00200F8BD00BF30B51A4B07
:1066900083B01C680CB103B030BD012501A81D609A
:1066A00003F068FD29464FF4001003F03DFF082079
:1066B000294603F02BFF0820294603F027FF29462F
:1066C0004FF4001003F03EFF21464FF4001003F09A
:1066D00039FFC023ADF804304FF440601C23C4F2EE
:1066E000010001A98DF8073003238DF8063003F06F
:1066F000DDFCFFF7FFFECEE7B40C00202DE9F041F2
:10670000069D1E466F1E7B427B418046FFF770FF51
:10671000074610B13846BDE8F08180200421C1F25F
:106720000000C1F20001FFF727FF00285BD04FF403
:10673000A844C4F200042046012103F017FE012002
:10674000C1F200003946FFF737FF00284ED020463F
:106750005FFA88F1012203F039FE0220C1F2000045
:106760003946FFF729FF002843D0238B8DB33C46E1
:1067700011E040200021C1F20000FFF71DFF18B317
:106780004FF4A840C4F2000003F01CFE3219AC42E2
:1067900002F8010C1DD00134AC42EAD14FF4A840FC
:1067A000C4F20000002103F0FDFD4FF4A840C4F244
:1067B0000000012103F0E8FD40200021C1F20000AB
:1067C000FFF7FAFE0028DBD16FF006073846BDE878
:1067D000F0814FF4A840C4F20000012103F0E2FD73
:1067E0003846BDE8F0816FF0030793E76FF00407C8
:1067F00090E76FF005078DE770B51C460023FFF7A3
:10680000F7FE064608B1304670BD8020C1F2000098
:106810003146FFF7D1FE28B3049BD3B1049BE518A2
:1068200001E0AC4215D04FF4A84014F8011BC4F2AB
:10683000000003F0C5FD80200421C1F20000C1F278
:106840000001FFF799FE0028EBD16FF003063046F8
:1068500070BD4FF4A840C4F20000012103F094FD84
:10686000304670BD6FF00206CDE700BF70B43A4A03
:106870003A49546A0B689C4215D8956AAB4212D2C9
:10688000D56B002D52D01C1B00FA04F4344D2E6839
:1068900026432E601268032A32D0052A15D0013310
:1068A0000B6070BC7047D46A2B4DA342F2D32E6BA1
:1068B000B342EFD2ED6B002D3ED01C1B00FA04F466
:1068C000284D2E6826432E60E4E7A3F11402032A24
:1068D00023D9A3F11804032C34D800FA02F2224C75
:1068E00025681543256003F00702012404FA02F429
:1068F00058BB1E48DA08855C25EA04048454CEE7B8
:10690000102BCCD9142BCAD8A3F1110400FA04F02F
:10691000174A146804431460C1E7A3F1080500FA9C
:1069200005F5104A14682C431460DCE70C4C25680C
:1069300040EA45052560ADE70A4C256840EA450573
:106940002560A7E72F2BAAD8CDE70848DA08855C91
:106950002C438454A3E700BFE40C0020CC0C00209F
:10696000280D0020440D0020400D0020BC0C00200C
:10697000380D002000B583B001A803F0FBFB082010
:10698000012103F0C3FD0823ADF804304FF440604B
:1069900002238DF80630C4F20100042301A98DF80A
:1069A000073003F083FB03B000BD00BFF0B4294AF9
:1069B0001368002B2BD028490B68022B17D0032B10
:1069C000264B26D0264C0F682168264DA0F80110D2
:1069D0001E680021A0F803602E68077019604671D8
:1069E00021600120296000231360F0BC70471B4B1D
:1069F0001D681C68E443E4B2B4EB152F1BD0184C9F
:106A000048F2EE752668AE421AD00020EBE7184631
:106A1000EBE71D681C68E443E4B2B4EB152FF4D136
:106A20001C68E4B21C60104C26681D680C4C45EADA
:106A300006251D60C7E71D68094CEDB21D60C2E761
:106A40000B250D601D68C5F3072525601D68EDB297
:106A50001D60B8E7480D0020E00C0020C80C0020A5
:106A6000300D0020340D0020D00C00202DE9F0471F
:106A70004FF440609E4CC4F20100082103F082FBF9
:106A8000236893B99B4E356895B99B4B002800F05D
:106A9000C2801B68002B40F00C81984B4FF6FE71B2
:106AA0001A688A4201D801321A602068BDE8F0876E
:106AB000934F3A68002A70D0002800F0B280914AC3
:106AC00011780131C9B2E929117000F206818E4BAB
:106AD0008E495A6B09688A42E7D1996B0029E4D143
:106AE000DFF868828A49D8F800C00D68AC4500F02C
:106AF00079818848002707601B68012B00F06581B9
:106B0000052B00F07A810A2B18BF292B03D10068CE
:106B1000C00700F156810120022B206040F09C81CB
:106B2000002A40F0028275480368B3F5E16F80F0F7
:106B30001682794D794FD5F800903B68DFF8F4A1C3
:106B400049F00109C5F80090CAF80030C1F800C04A
:106B500002606546724A02201060724A3B60136010
:106B6000714B1A68714B1D60714B1A60236863B1D9
:106B70000B689C4500F0BA816E4A60481568674F03
:106B8000C8F8003000233D6003605B4A00231360B7
:106B90005C4A33600B60137087E7674F3B68002BDC
:106BA00000F08180584B002840F0D2801A68032AF8
:106BB00000F05581DFF84C81DFF83C915A68D9F834
:106BC000001051488A420BD88268914208D898F840
:106BD00000C0C268944503D30269944540F2B38172
:106BE0005B69494A99420BD39369994208D898F84E
:106BF0000010D369994203D3136A994240F2A981E4
:106C00000025356088F800500123C9F80030002DB8
:106C10003FF44BAF5BE71A6801321A602068BDE8A9
:106C2000F087DFF8D490DFF8DC80D9F80030A3F1EA
:106C30001F020A2A17D898F80020052A13D90A2A11
:106C400011D83E493048442204F004F82F4A00236A
:106C500013600122C9F8002088F800303B60002D45
:106C60003FF423AF33E7A3F15E02532A08D898F824
:106C700000202D2A00F2A080162A01D93049E1E730
:106C8000A3F13C020F2A40F28A80283B162B00F227
:106C9000908098F80030122B40F28B801F2B00F26E
:106CA00088802849CEE7E8B9134B1A6801321A6088
:106CB0000DE7134A012313601F4AFF211560144A90
:106CC000336015601B4A15601F4A1560164A15602F
:106CD0000E4A11600B4A1370E7E6074933600B60F8
:106CE0001370E2E6074A01233B601370EFE600BF32
:106CF000480D0020C40C00203C0D0020D40C0020C6
:106D0000B80C0020D80C0020E40C0020CC0C002093
:106D1000440D00202C0D0020340D0020A001002087
:106D2000E00C0020300D0020380D0020C80C0020A1
:106D3000D00C0020280D0020DC0C002000EC000806
:106D4000CCEC000844EC0008400D00209C01002021
:106D50008B49D3F83490D1F800C0E14500F0908021
:106D6000DFF850821A6898F800A0012A0AF1010A97
:106D70005FFA8AFA834888F800A000F09980BAF197
:106D8000E90F7FF644AF09F1FF32944500F0C3806C
:106D90007D4A00233360136088F8003085E698F858
:106DA00000203B2A7FF671AF4B2A3FF66EAF774942
:106DB00048E70025356049E7592A3FF661AF744935
:106DC00040E7744800230360D0E60268013A012AD4
:106DD00088BF2360F5D9704A704812680360704B11
:106DE0001A60BDE66B480068B0F5966FBFF481AEDF
:106DF0006C480768013707607EE60368012BE0D026
:106E000001232360684B1F7858789A7887EA000935
:106E100009F00F0989EA171787EA101002F00F0925
:106E2000814501D000202060D8781F7942405879F0
:106E300082EA0703984201D0002323605B4B5C4A3F
:106E40001F681068544A38431860544B0520186076
:106E50001268534B1A6083E6052BD3D0BBE7484931
:106E60000A68102A7FF4A6AEDFF81C91D9F800203A
:106E7000053A072A79D94F4B306018700546C3E6AA
:106E8000986B01287FF46CAFDFF8FC905869D9F853
:106E90000010884205D89869814298BF9A637FF6AE
:106EA000B6AE444A00233360C9F800301370FCE5E5
:106EB000BAF10B0F7FF6ABAEBCF10A0F7FF65FAFF6
:106EC000DFF8D490C16AD9F80020ACF10B0A614414
:106ED00042EA0A220CF1010C0131C9F800200A2211
:106EE000C0F834C0016388F8002065E62A48324FB4
:106EF00005683A682748AA427FF442AE026840F625
:106F0000C90C62459FBF294AD2F800C04CF0010C61
:106F1000C2F800C034E69B6B002B7FF439AFC1F898
:106F20000090002D3FF4C1ADD1E51B4B224F1B68F3
:106F300010E60A200F3A2021186010200F2AD8628C
:106F40001963596305D80120FFF790FC00233B60CB
:106F50005AE60020FFF78AFC00233B6054E6174BFB
:106F6000154F1A600C4B1B68F4E5124A12783B2A45
:106F7000DFD94B2ADDD800233B6011230B6043E6A9
:106F8000CC0C0020E40C00203C0D002010ED00088B
:106F900088EC0008D40C0020280D0020E00C002014
:106FA000300D00202C0D0020BC0C0020340D0020E2
:106FB000400D0020D80C0020A0010020480D00202A
:106FC000F9F768B910B582B004460DF10600F9F77B
:106FD00071F978B1084B09491B88BDF8062009886A
:106FE000D21AC2EB0212CB1A92FBF3F30F2B28BF7B
:106FF0000F23236002B010BD4C0D00204E0D002069
:1070000008B50F4B1B686BB1FF23C0F20203984217
:107010000AD80C4B00221A800B4B40F2FF321A8028
:10702000012008BD184608BD02220649E120FCF7F0
:1070300021FBE32004490222FCF71CFB012008BDD0
:10704000A40400204C0D00204E0D002008B50A4B72
:107050001B680BB9002008BDE12008490222FCF79B
:1070600023FB0028F6D00222E3200549FCF71CFB95
:10707000003018BF012008BDA40400204C0D0020E2
:107080004E0D002040F64C53C2F2000318887047A2
:1070900040F64E53C2F200031888704710B582B014
:1070A000F9F7F8F80A240DF10600F9F703F940B9E9
:1070B0000A20F9F7C5FC013CF5D1054C208802B047
:1070C00010BD034CBDF806302380FFF7BFFFF5E786
:1070D0004C0D002010B582B0F9F7DCF80A240DF150
:1070E0000600F9F7E7F840B90A20F9F7A9FC013CD6
:1070F000F5D1054C208802B010BD034CBDF8063018
:107100002380FFF7A3FFF5E74E0D0020F9F752B8F3
:10711000F0B507468DB00A20FCF7A4FC092828D05A
:107120000A2813D0072803D0002420460DB0F0BD54
:10713000FCF7EEFD0A2201A900F5B67004F006FA8C
:107140000146384602F0E8FB7424EEE7FCF7E0FD68
:1071500000F14C042021204604F08AF8014610B1C9
:10716000002301F8013B20463A46FDF701FB0446A7
:10717000DBE7FCF7CDFD01AE00F5A674002502E0CB
:1071800002340A2D12D0237820460221002B7BD016
:107190006378002B78D0F9F7E5F8A3780135202B38
:1071A00046F8040FECD103340A2DECD1029CA4F173
:1071B00041032F2BB8D801A252F823F07D720008AA
:1071C0007D720008D77200087D72000829710008DE
:1071D0007D7200087D72000829710008297100087D
:1071E00029710008297100087D72000829710008C2
:1071F00091720008297100087D7200082971000849
:107200002971000891720008B17200082971000804
:10721000297100089172000829710008297100087D
:1072200029710008297100082971000829710008D6
:1072300029710008297100082971000829710008C6
:107240007D720008D77200087D720008297100085D
:1072500029710008297100082971000829710008A6
:107260002971000829710008297100082971000896
:10727000297100082971000899720008022D7FF415
:1072800053AF039B3B6050E7002D3FF44DAF8DE7BC
:10729000012D7FF449AF48E72023384600F8013B31
:1072A0000DF109011E2204F023F80023FB773CE7CF
:1072B000072D7FF439AF039B03F16402049B7A61CD
:1072C000013B3B61059BFB60069BBB60079B7B60B2
:1072D000089B3B6029E7042D7FF426AF039B3B709E
:1072E000049B7B70059BBB701FE700BF30B53B4B19
:1072F00087B01A68044682426DD068461C6002F06E
:1073000039FF02A803F0AEFA0420012103F0FEF8D1
:107310000420012103F0FAF84FF48040012103F02A
:10732000F5F84FF400734FF400600325C4F2010038
:107330006946ADF8003018238DF803308DF80250FF
:1073400002F0B4FE4FF480634FF40060C4F2010019
:107350006946ADF8003048238DF803308DF80250AF
:1073600002F0A4FE4FF46050C4F20100012103F0CA
:10737000B7FA00234FF460501D46C4F2010002A981
:10738000ADF80C30ADF80E30ADF81030ADF814306B
:107390000C23ADF81230029403F0FEF94FF4605064
:1073A000C4F20100012103F069FA4FF46050C4F205
:1073B000010040F22551012203F06EFA25238DF8D9
:1073C000043001A801238DF805508DF806508DF882
:1073D000073002F075FC07B030BD00BF500D002033
:1073E00030B40F4A13687F2BFCD80E490E4D0B6842
:1073F0005C1C7F2C45F8230098BF0C6001D900234A
:107400000B6072B613680133136062B64FF46050BC
:10741000C4F2010040F22771012230BC03F03CBAF3
:10742000600F0020640F0020580D002010B50446A6
:10743000007828B1FFF7D4FF14F8010F0028F9D124
:1074400010BD00BF30B40D4B1A6882B10C490D4D10
:107450000A68541C802C55F8225018BF0C6009D0C3
:1074600072B61A68013A1A6062B6012205601046C7
:1074700030BC704700220A60F2E700BF540D0020C4
:10748000580F0020680F0020024A1368002BFCD11F
:10749000704700BF600F00204FF4605038B5C4F251
:1074A000010040F2255103F029FA00282BD14FF4B6
:1074B0006050C4F2010040F2277103F01FFA00B9D6
:1074C00038BD4FF46050C4F2010040F2277103F060
:1074D0003BFA234B1A68002A38D0224A224C116802
:1074E000481C802808BF002054F8211010601A683A
:1074F0004FF46050013AC4F2010089B21A60BDE84D
:10750000384003F0E5B94FF46050C4F2010040F296
:10751000255103F019FA4FF46050C4F2010003F052
:10752000DBF9124B1A687F2AC1D81149114D0A683C
:10753000C0B2541C7F2C45F8220098BF0C6001D9C2
:1075400000220A601A6801321A60B0E74FF46050F6
:10755000C4F2010040F22771BDE8384003F09CB945
:10756000600F002068110020580D0020540D0020ED
:107570005C0F0020680F002010B541F26C14C2F2BD
:10758000000402460B4620464FF4807104F008FBCD
:107590002046BDE81040FFF749BF00BF0FB400B55B
:1075A00083B004AB53F8040B19460193FFF7E4FFD3
:1075B00003B05DF804EB04B0704700BFFFF796BE60
:1075C00010B584B001A803F087F80120014602F04D
:1075D000ABFF0023ADF80A30ADF80630052301A952
:1075E000ADF808304FF0804040F21F33ADF8043062
:1075F00002F0B6FF01210A464FF0804003F09EF8EA
:1076000001240F2368461C228DF800208DF80340CA
:107610008DF801308DF8023002F052FB4FF08040BF
:10762000214603F06DF804B010BD00BF38B54FF02F
:107630008040012103F0ACF86A4B1C68002C34D068
:10764000694B43F698211A6801328A421A6000D0C9
:1076500038BD664A0120664910600C68654A2418E6
:107660000C601468002124181460146819603C2C04
:10767000EED1614B11601A6812181A605F4A1060EF
:107680001A683C2AE4D15E4A196013681B1813601B
:107690001368182BDCD15B4B11601A6812181A6042
:1076A0001A68072AD4D1196038BDFFF7DFF95049AD
:1076B0000B68012B07D9544B40F6A6601A680132BB
:1076C00082421A6043D0514B1A680132EA2A1A608A
:1076D00054D04F4B1A680132962A1A6048D04D4B4D
:1076E0001A680132962A1A603CD04B4B1A68013254
:1076F0000F2A1A6030D03C4B43F698201A680132AA
:1077000082421A60A4D1394A012010600C68394ABB
:1077100024180C60116800240918116011681C609D
:107720002D2931D01268334B3C2A38D01B681E2BD0
:1077300053D03A4B1A68002A8AD01A68013A1A6064
:107740001B68002B84D1364B01221A6080E7354A32
:10775000012010601C60B6E7334A0120106000224F
:107760001A60C8E7314A0120106000221A60BCE7A5
:107770002F4A0120106000221A60B0E72D4A012034
:10778000106000221A60A4E72B4B1B491C680D688F
:10779000AC421FBF09681960284B1860C2E7164A3F
:1077A000002119601368012001331360134B186026
:1077B00013683C2BBDD1124B11601A6812181A6065
:1077C0001A68182AB5D10F4A196013681B1813607C
:1077D0001368072B08BF1160ABE7194B01221A6031
:1077E000A7E700BFBC1200206C1200207812002016
:1077F000C412002088120020CC1200208C1200201D
:10780000AC1200207C12002094120020B012002044
:107810009012002084120020A8120020A401002051
:1078200070120020B4120020A4390020A8390020D2
:10783000A4120020C8120020AC01002098120020E1
:10784000B81200204EF65450C0F60000704700BF3A
:1078500040F2B013C2F200031868704741F2AC2145
:1078600041F2CC2241F28823C2F20001C2F20002AE
:10787000C2F20003096843F6AC1012681B68C2F23A
:107880000000816042600360704700BF2DE9F04F47
:107890009FB003F0BDF803F049F90120014602F062
:1078A00035FE4FF400700121C0F2300002F076FC8A
:1078B0004FF4E130FFF782FEFFF75CF801F074FB54
:1078C00001F09AFBFFF77CFE0120F9F7DDF8F8F7ED
:1078D00087FDF8F7A3FD01F04FFDFBF7A3FEF8F7D6
:1078E000B5FD002841F01B81BF48FFF79FFDBF4851
:1078F000FFF79CFDBE48FFF799FDBC48FFF796FDDA
:10790000BC48FFF793FDDFF81CB3BB48FFF78EFDC3
:10791000B648FFF78BFDDBF80030002B01F0A680A6
:10792000B648FFF783FDB148FFF780FDB44DFBF784
:1079300091FD2B68002B01F09080B248FFF776FD97
:10794000AA48FFF773FD2B68002B41F0C580AE4CB1
:10795000AE482168FFF722FE226822F47F0323F459
:107960007F43EBB940F2FF43C0F201039A4201F2B8
:10797000F48040F2FF632268C0F201039A4201F2F0
:10798000E280A348FFF752FD9848FFF74FFD2068BB
:1079900001F0DAFE206801F057FE2068FFF730FBA7
:1079A000FFF7B4FBF8F792FD01F0BCF941F2BC20FF
:1079B0000123C2F20000036001F010FF41F2BC217C
:1079C000C2F2000100260E60FAF7E0FCFAF708FEAA
:1079D00041F28022C2F200021060FAF753FE41F237
:1079E000A023C2F200031860FAF784FE41F29C293A
:1079F000C2F20009C9F80000FAF728FE41F2C02CD3
:107A00002B68C2F2000CCCF8000083B34FF48075F1
:107A10002368C0F20205AB427B4F28D07D4829463F
:107A2000FFF7BCFD764B3D601B68002B41F0C88022
:107A30007948FFF7FBFC6D48FFF7F8FC01F052FCBA
:107A4000002801F0B580FBF7D5FB002801F0A880E5
:107A500001F0FAFE002801F09B8001F0FDF80028FB
:107A600001F069804FF48073C0F20203236041F299
:107A7000982E0120C2F2000E41F2C421C2F2000190
:107A8000CEF800000C68024601460334FAF760FCA9
:107A900041F2C422C2F2000213680BA89C421ED914
:107AA000FEF784FF0028F3D000210A460120FAF7F0
:107AB0004FFC0120F8F7D2FF0BA8FEF777FF00205C
:107AC00001460246FAF744FC5448FFF7AFFC47482A
:107AD000FFF7ACFC01F00EFB08B101F003FC002045
:107AE0000146024604460890FAF732FCFCF7DCF93E
:107AF000FCF70EF9089E4FF0010900F13C0CDFF88D
:107B00002881474F0694824604253446CDF81C90C0
:107B1000CDF824C0059615A8FFF7FAFA814600288B
:107B200040F03081D8F8003043B141F2C02EC2F2AB
:107B3000000EDEF80030002B40F03C86069E002E42
:107B400040F09C83DAF80030002B40F0E0853448A8
:107B5000F8F78AFC002840F0A58341F29820C2F291
:107B6000000003685BB1DBF80030002B40F0D985E2
:107B700041F2982C0023C2F2000CCCF80030D8F867
:107B8000003073B141F2C02EC2F2000EDEF80030B8
:107B90003BB141F2B420C2F200000368002B40F078
:107BA0009A8641F27021C2F200010B688BB1DAF8BB
:107BB0000430002B40F03D8641F270220023C2F2D7
:107BC000000240F2A4161360C2F2000640F6D86329
:107BD000336041F28C29C2F20009D9F80030002B41
:107BE00040F0A78322E000BF5CED000840DF000802
:107BF0007CED00089CED000854ED0008A8ED00089D
:107C0000A4040020C8ED0008B0010020DCED00084D
:107C100094EE0008D0EE0008F4EE0008B4EF00087F
:107C2000AC390020541300208038002041F2B82CD9
:107C3000C2F2000CDCF80030002B00F0758240F23C
:107C40003039C2F20009B04AD9F800300021116081
:107C5000002B00F0698241F2CC2CC2F2000CDCF85F
:107C60000020B2FBF3F103FB1123002B40F05C82F8
:107C700040F2904EC2F2000EDEF80030002B40F0D1
:107C8000BB85DBF80030002B00F0288501F026FDD5
:107C90009E4B9F4A064610F0010F4FEA56019D4841
:107CA00018BF1A46FFF77AFCFF2E0AD03046FBF7C2
:107CB00095F841F2C42CC2F2000CDCF80030063317
:107CC0000893002D40F0448241F2C820C2F2000027
:107CD0000368002B40F0758241F27822C2F2000264
:107CE0001368002B40F07F8241F2A425C2F2000508
:107CF0002B68002B40F0898201F0B6F9FF28054679
:107D000000F08E82002101200A46FAF721FB132D94
:107D100000F2B486DFE815F0BC01E801D601F501F8
:107D20008701B30199016C0133011401EA00DD0000
:107D3000D000C300A900B60094007F00B206140072
:107D40007548FFF773FB7548FFF770FB0126322477
:107D500005960025069EDDF81C9016EA090F52D103
:107D6000002C3FF4D8AE013C7FF4D5AE204621462E
:107D70002246FAF7EDFA15A8FFF7CAF9814600285E
:107D80003FF4D0AE002101200A46A9F14109FAF7DB
:107D9000DFFAB9F1330F00F21B83DFE819F0690451
:107DA000560451043B0419038504050419030E030A
:107DB00019031903E3031903A30319038A0319031E
:107DC00019037F03250319031903D803CD031903EE
:107DD00019031903190319031903190319031903C3
:107DE000C203B30374031903190319031903190315
:107DF0001903190319031903190319036903190353
:107E0000190319031C03F8F721FB002840F01F8514
:107E100001260796A4E74248FFF708FB3F48FFF713
:107E200005FB41F2C026C2F200063368002B40F089
:107E3000DC850025FAF726FF32240595022589E71F
:107E40003848FFF7F3FA3548FFF7F0FA41F2C02659
:107E5000C2F200063368002B40F0B8850025FAF71F
:107E600007FF32240595022574E72F48FFF7DEFA55
:107E70002A48FFF7DBFA0025FAF790FE3224059531
:107E8000022567E72948FFF7D1FA2448FFF7CEFA21
:107E90000026FAF773FE3224059602255AE7244895
:107EA000FFF7C4FA1D48FFF7C1FA0026FAF746FEAD
:107EB0003224059602254DE71E48FFF7B7FA17480A
:107EC000FFF7B4FA0025FAF749FE3224059502259A
:107ED00040E71948FFF7AAFA1048FFF7A7FA00266B
:107EE000FAF70CFE32240596022533E71348FFF714
:107EF0009DFA0A48FFF79AFA0025FAF70FFE322496
:107F00000595022526E700BFB812002038E70008D3
:107F1000C8DE000814F4000864F6000840DF00081A
:107F200048F600082CF60008ECF500080CF60008EE
:107F3000C8F50008A4F5000884F5000864F50008F9
:107F4000B948FFF773FAB948FFF770FA41F2CC234A
:107F5000C2F200031A68B64B3A2A00F2EB841A68A0
:107F600001321A6041F288240023C2F20004236027
:107F7000DBF80060FEB9322405960425EAE6AD4838
:107F8000FFF754FAA948FFF751FA41F2CC20C2F2A8
:107F900000000268A64B002A00F0D8841A68013A53
:107FA0001A6041F28821DBF800600023C2F2000170
:107FB0000B60002EDFD041F2AC2941F2CC2C41F213
:107FC000882EC2F2000CC2F2000EC2F20009D9F8EB
:107FD0000010DCF80020DEF8003000259648B9607B
:107FE0007A603B60322401F023FA05950425B1E65E
:107FF0009248FFF71BFA8D48FFF718FA41F2AC2CB4
:10800000C2F2000CDCF800208D4B162A00F2968498
:108010001A6801321A6041F2882E0023C2F2000E63
:10802000CEF80030A4E78748FFF700FA7F48FFF753
:10803000FDF9FAF741FB41F2A0260025C2F2000645
:10804000059532243060042584E67F48FFF7EEF979
:108050007648FFF7EBF941F2AC26C2F2000632682F
:10806000774B002A00F06E841A68013A1A6041F2D8
:1080700088290023C2F20009C9F8003078E7734864
:10808000FFF7D4F96948FFF7D1F9FAF709FBD2E70E
:108090006F48FFF7CBF96548FFF7C8F940F25C1C61
:1080A000C2F2000CDCF800503224D5F1010538BFD3
:1080B00000250026CCF800500596B5420CBF1425CB
:1080C0000C2547E66348FFF7B1F95848FFF7AEF9CA
:1080D000FAF7ACFA41F28025C2F2000500262860CA
:1080E00032240596042535E65B48FFF79FF94F4893
:1080F000FFF79CF900240594FBF77CF83224059DDA
:1081000028E65648FFF792F94848FFF78FF9FAF743
:108110007BFA41F280290025C2F20009059532243C
:10812000C9F80000042515E6059E002E7FF4A0ADD9
:10813000089E002E3FF4C5AD41F2C429C2F20009E9
:10814000D9F80030B342FFF4BCAD059E0425089673
:10815000434841F28029FFF769F9C2F20009334828
:10816000FFF764F9D9F80030112B40F0BF8240F2DC
:10817000904CC2F2000CDCF80030002B40F0BB83C6
:10818000DBF80030002B00F0AD8301F0A7FA354B8F
:10819000354A064610F0010F4FEA5601334818BF22
:1081A0001A46FFF7FBF9A6F1140100202A46FAF758
:1081B000FFF841F2C820C2F200000368002B3FF430
:1081C0008BAD40F25C112A4BC2F20001002208681C
:1081D0001A60FAF767FB41F27822C2F200021368D4
:1081E000002B3FF481AD234B00221A6041F288231B
:1081F000C2F2000341F2A4251868C2F20005FAF7A2
:1082000091FA2B68002B3FF477AD1B4B00221A60CC
:10821000F8F792F900F028FFFF2805467FF472ADC9
:1082200000260596354695E54CF5000840DF000828
:10823000CC12002034F50008AC3900201CF50008F1
:10824000AC120020C4F4000804F50008E4F40008AF
:1082500064F4000884F4000874F40008A4F400082E
:1082600054F4000838E70008C8DE000814F40008D9
:10827000C812002078120020A412002041F27429B4
:10828000C2F20009D9F8003023B9DAF80430002B23
:1082900040F003830126CA480696F8F7E5F800285F
:1082A0003FF45BAC012001460022FAF751F8DBF8FD
:1082B0000030002B40F0C78241F2AC29C2F2000925
:1082C000D9F80030BC68BE4A9C4200F0DA82D2F88D
:1082D00004E00425D7F8189040F20000C2F2000034
:1082E00050F829103E68F86841F27C2CC2F2000C6C
:1082F0007A693B698DE811400396CCF8009041F211
:10830000AC2941F2CC2CC2F2000CC2F20009C9F82F
:108310000040CCF800E041F2882EC2F2000EA948DD
:1083200002F26C720133CEF80060FFF737F93224A5
:1083300013E4A54B002241F27C2C41F2AC2E1A60D2
:10834000C2F2000CC2F2000E41F2CC20DCF80010A8
:10835000C2F20000DEF8003040F25C150268C2F2A2
:108360000005C3EB0313286802EB8302974D00F06E
:108370009FFC002800F01B822B68DFF874C2D3F149
:10838000010E38BF4FF0000E41F2AC2641F2CC296D
:108390008F49BEF1000FC2F20006C2F20009326836
:1083A0008C48D9F8003008BF6146C5F800E00CBF22
:1083B00014250C25FFF7F2F838E48748FFF736F864
:1083C0008648FFF733F800F095FE002840F08181E1
:1083D0003224FFF7A7BB159B40F2A412C3F56E63CE
:1083E0000233C2F200021360DBF80030002B40F0D1
:1083F0000B8341F2AC24C2F200042368DDF85CE098
:108400009E4500F00583DDF858C004251B9C40F212
:108410000009C2F2000959F82410159E189B41F278
:108420007C29C2F20009CDF804E00093CDF808C021
:108430000396C9F8004041F2AC29C2F20009C9F81C
:1084400000E01A9A199B41F2CC2E41F28829C2F21F
:10845000000EC2F20009CEF800C0614802F26C7250
:108460000133C9F800603224FFF798F8FFF75ABBD0
:1084700015A8FAF75BFC5B4815A9FFF78FF80425F0
:108480003224FFF74FBB1598FAF77AF801465648A1
:10849000FFF784F804253224FFF744BBFAF7AAFE5D
:1084A0005248FEF7C3FF4D48FEF7C0FF3224FFF7E6
:1084B00039BB40F25C1EC2F2000E159BDEF80020B4
:1084C000934285D04A4A4249002B08BF11463F4A91
:1084D000484814BF0C25142513603224FFF75EF8BA
:1084E000FFF720BB41F2702C0123C2F2000C42487E
:1084F000CCF80030FEF79AFF3848FEF797FF322499
:10850000FFF710BB15A8FAF789FB3C489DF85410FB
:108510009DF855209DF85630FFF740F83224FFF7BC
:1085200001BB1598FAF7C0FB35481599FFF736F8E7
:1085300002253224FFF7F6BA3248FEF777FF2748C4
:10854000FEF774FF3224FAF7BBFBFFF7EBBA2E48B5
:10855000FEF76CFF01242148FEF768FF05943224E2
:10856000FFF7E0BA159B002B00F05D8241F2C029B5
:1085700026480123C2F20009C9F80030FEF756FF71
:108580001648FEF753FF41F2C02EC2F2000E40F231
:10859000A811FF23C2F20001DEF800000B603224B4
:1085A000FAF75AF8FFF7BEBA1598F9F7C5FF184859
:1085B0001599FEF7F3FF04253224FFF7B3BA00BF85
:1085C000AC39002074F300088C1200205C010020FC
:1085D000A0F60008CCF30008C8F2000840DF00084D
:1085E00070F2000800F30008B8F00008E0F200089C
:1085F000B4F600087CF00008A8F2000850F000086B
:10860000A0F1000854F200082CF10008CCF1000899
:108610002CF2000841F28021C2F2000115980B688B
:1086200098423FF4D5AEF9F7E1FFD04A0346014640
:10863000CF4813600425FEF7B1FF3224FFF772BA6A
:1086400015A8FAF7C7FACB4860E741F2C025C2F295
:1086500000052B68002B40F0F3811598FAF7FCFA1F
:10866000C5481599FEF79AFF02253224FFF75ABA3A
:1086700041F2A022C2F200021598136898423FF41A
:10868000A7AEFAF705F8BD4A034641F2C8241946D9
:108690001360C2F200040023B94823600425FEF7EA
:1086A0007DFF3224FFF73EBA41F29C26C2F200065B
:1086B0001598336898423FF48BAEFAF721F8B14A27
:1086C00003460146B04813603224FEF767FFFFF708
:1086D00029BA00F007FE3224FFF724BAAB48FEF7B0
:1086E000A5FEAB48FEF7A2FEFFF7EBBA41F2AC2CB9
:1086F00041F2CC2EC2F2000CC2F2000EDCF80000F7
:108700002A46DEF80010F9F753FEFFF7DDBAA1485C
:10871000FEF78CFE01269E48FEF788FE0696FFF7C0
:1087200016BADFF88892484600F016FF00283FF49A
:108730001FAA41F2AC21C2F200010B68D9F808E08F
:108740009E4500F00781D9F804C00425BE69F86889
:1087500040F20003C2F2000353F826107A693B6925
:108760008DE80140CDF808C0386841F27C29C2F29A
:1087700000090390C9F8006041F2AC2641F2CC290F
:10878000C2F20006C2F20009C6F800E0C9F800C053
:108790003E6841F28829C2F200097F4802F26C72F9
:1087A0000133C9F80060FEF7F9FEFFF7E1B90425CF
:1087B000FFF73CBA0AA8FEF705FC00283FF4BEA963
:1087C00040F2A8100A9AC2F200000168531C8B42C2
:1087D00003D34B1C9A427FF6B1A97048FEF7DEFE28
:1087E0000A9B40F2A811C2F20001184602250B6054
:1087F000FAF732FAFFF7A2B941F2BC200123C2F224
:108800000000036000F08AFF654B664A10F0010F1C
:10881000064641F2BC2918BF1A46C2F200090023DD
:1088200061484FEA5601C9F80030FEF7B7FEFFF77E
:108830003BBA002001460122F9F78AFD322401F0FB
:1088400065F8FFF7B9B9594800F0F2FD34E558482A
:10885000FEF7ECFD4E48FEF7E9FD4FF0000941F24E
:10886000742CC2F2000CCAF804908AF83C9051496A
:108870005148CCF80090CDF81C90FBF78DFAFFF72B
:108880006FBA41F2CC2CC2F2000CDCF80030D2F806
:1088900004E09E457FF41DAD1CE5484B4FF00109F7
:1088A0004748C3F80090FEF7C1FD3948FEF7BEFD0A
:1088B0004449099A0DA802F0B7FC0DA8FAF736FA58
:1088C00041F2702CC2F2000C0425CCF80090CDF8D7
:1088D0001890FFF73CB9FEF773FB3B4B00221A6080
:1088E000FFF75FB92948FEF7A1FD2948FEF79EFD75
:1088F0006FF0130159E441F2BC2E0123C2F2000EC5
:10890000CEF8003000F00AFF254B264A10F0010F88
:10891000064641F2BC294FEA560118BF1A462248C2
:108920000023C2F20009C9F80030FEF737FEA6F1B5
:1089300014013AE400221A60FFF714BB00221A6007
:10894000FFF769BB17221A60FFF791BB3B221A6041
:10895000FFF727BB41F2CC22C2F200021368D9F81C
:1089600004C09C457FF4F1AEF0E600BF8012002009
:1089700094F0000824F0000848F10008A01200203C
:10898000DCF000089C12002000F1000838F4000818
:1089900040DF000848F30008A0F300081CF30008BB
:1089A00038E70008C8DE0008ECF30008AC39002006
:1089B000D0EF000818F000080CF000087412002036
:1089C00058F300086CF30008B4120020814A002319
:1089D00040F2A81918461360C2F20009FF23C9F833
:1089E0000030F9F739FEFFF739BA7A4A002340F22E
:1089F000A81918461360C2F20009FF23C9F8003015
:108A0000F9F72AFEFFF715BA15A800F011FDF0E4FA
:108A100041F2CC26C2F200063368DDF858C09C450E
:108A20007FF4F3ACF2E441F2C02CC2F2000C6A48CD
:108A3000CCF80030FEF7FAFC6848FEF7F7FCA2E538
:108A4000644A002340F2A81618461360C2F20006DA
:108A5000FF233360F9F700FEFFE56148FEF7E6FC0F
:108A60005E48FEF7E3FC5F4CFEF79ABF5E48FEF7F8
:108A7000DDFC5A48FEF7DAFCFEF758BF132D54D838
:108A80000FF2040959F825F09D800008F5800008D0
:108A9000D18000080F810008338000088B80000817
:108AA00057800008FD7F00088B7F00084D7F00087D
:108AB000F97E0008DF7E0008C57E0008AB7E000856
:108AC000777E0008917E00084D7E0008237E000816
:108AD000E78A00084D7D0008002042490422FAF789
:108AE000C9FDFEF734BF41F2C029C2F20009D9F82E
:108AF000003040F2A81CD3F1010338BF0023184610
:108B0000C9F80030C2F2000CFF230025CCF8003079
:108B10003224F9F7A1FD05950225FFF71BB9F7F7F8
:108B20004BFCFBF76BF9FEF7DFBE00240594002534
:108B30003224FFF70FB92D48FEF778FC2748FEF7DF
:108B400075FCFEF78FBF2A48FEF770FC2348FEF73E
:108B50006DFC00F05BF8FEF714BF2648FEF766FCDC
:108B60001E48FEF763FC00F093FB2348FEF75EFC13
:108B70001A48FEF75BFC2068FAF7A2F91F48FEF7D7
:108B800055FC1648FEF752FC00F02CFEFEF7F1BE35
:108B90001B48FEF74BFC1148FEF748FCFEF75DBF93
:108BA0001848FEF743FC0D48FEF740FCFEF750BFA7
:108BB0001548FEF73BFC0948FEF738FCFEF743BFBB
:108BC000304639460422FAF76FFD00287EF436AFAE
:108BD000FEF72EBFC0120020FCF1000840DF0008A5
:108BE000BCEE0008B0010020B8ED000888EF0008D6
:108BF00070EE000800EE000820EE00084CEE0008C1
:108C00005CEF00083CEF000818EF000830B5104B8F
:108C100087B01B6813B9002007B030BDBF2069467C
:108C20001822FAF727FD0028F5D00A486A460023E3
:108C30001478517895781C50C1EB01111C18083339
:108C400005EB81010332402B6160F1D10120E3E7A4
:108C5000A4040020D0390020F0B548F6890787B079
:108C6000114C6A460023C8F68807191948681D592F
:108C7000A7FB00614909C1EB0116A0EB8600083390
:108C80001570517090700332402BEED1074B18686D
:108C900038B1BF2018226946FAF706FD003018BF28
:108CA000012007B0F0BD00BFD0390020A40400208F
:108CB000F0B400231A4D02E00833402B21D05C5958
:108CC0005E1914F0800FF7D076689642F4D1C4F3A1
:108CD000C20604F0070704F0400418B1D4F10104FF
:108CE00038BF0024002CE7D0BE420DD8B14234BFBB
:108CF00000260126B94288BF0026002EDCD00120C4
:108D000000E00020F0BC7047B9428CBF002701276B
:108D1000B14234BF3E4647F00106002ECCD0EEE70C
:108D2000D0390020704700BF70B56420F7F774FE9B
:108D30004FF4406020210022C4F2010001F028FA23
:108D40004FF40C70F7F768FE4FF44060C4F2010076
:108D50002021012201F01CFA274D1420F7F75CFEB8
:108D600000264FF496732B60344603E004B92C6858
:108D70002B68ABB14FF440602021C4F2010001F038
:108D800001FAD6F1010338BF0023002C08BF0023ED
:108D90000028EBD0002BEBD02E682B68002BE9D1FC
:108DA0003220002E18BF002C0CBF0025012515D045
:108DB000F7F732FE4FF440602021C4F2010001F0C9
:108DC000E1F905467820F7F727FE6B1E5842C6EBFF
:108DD000040458411E2C98BF002070BDF7F71CFEFC
:108DE0004FF440602021C4F2010001F0CBF978205B
:108DF000F7F712FE284670BD7C38002010B54FF4FE
:108E00004064C4F2010420210022204601F0C0F990
:108E10000520F7F701FE01222021204601F0B8F9D4
:108E20000A20F7F7F9FD2021204601F0ABF90446AE
:108E30003220F7F7F1FD621E5042504110BD00BFD5
:108E400070B5082401250026FFF7D8FF6B0000B19C
:108E50002E43013CDDB2F7D1304670BD38B54D1E12
:108E60000446EDB239B101354519FFF7E9FF04F8C1
:108E7000010BAC42F9D138BD70B506460825012476
:108E800018E04FF440600022C4F2010001F080F9C4
:108E90000520F7F7C1FD4FF4406020210122C4F204
:108EA000010001F075F950206400F7F7B5FD013DB0
:108EB000E4B21BD04FF44060202114EA0602C4F251
:108EC0000100DED101F064F95020F7F7A5FD4FF461
:108ED000406020210122C4F2010001F059F905206F
:108EE0006400F7F799FD013DE4B2E3D170BD00BF26
:108EF00038B54D1E0446EDB239B10135451914F8A7
:108F0000010BFFF7B9FFAC42F9D138BD10B50446EB
:108F1000FFF70AFF80B9234603F8010B01336070A5
:108F200003F8010B03F8010B03F8010B03F8010B25
:108F300003F8010B187010BD3320FFF79DFF20468A
:108F40000821FFF78BFFFFF7EFFE012010BD00BFE8
:108F500030B5144B83B01A680AB103B030BD012498
:108F600001A81C6001F006F92020214601F0CEFA8C
:108F700014234FF44060202501A98DF80730C4F276
:108F800001000323ADF804508DF8063001F08EF88F
:108F90004FF44060C4F201002946224601F0F8F87F
:108FA000DBE700BFD012002000B583B001A801F0BC
:108FB000E1F80820012101F0A9FA0123ADF80430FD
:108FC0004FF44060022301A98DF80630C4F201007D
:108FD00010238DF8073001F069F84FF27C60C0F67D
:108FE0000000FEF723FA4DF64070C0F60000FEF7D1
:108FF0001DFA03B000BD00BF10B50A4C2368012B59
:109000000FD001214FF440600A46C4F2010001F084
:10901000BFF80548FEF70AFA0448FEF707FA0123ED
:10902000236010BDB401002090F6000840DF000866
:1090300010B50A4C23687BB14FF440600121002237
:10904000C4F2010001F0A4F80548FEF7EFF9054865
:10905000FEF7ECF90023236010BD00BFB40100202F
:10906000A4F6000840DF0008F0B583B06846FDF7BD
:109070009DFC68B31C4B1D4A1868116801301860CC
:10908000002928D09DF8050000F0010018490023B0
:10909000BDF80170BDF803C09DF8004010600E4699
:1090A000184602E00130782B12D0CA5C0633A24287
:1090B000F8D100EB400206EB4202B2F80150BD428B
:1090C000F0D1B2F80320624503D00130782BECD107
:1090D000FF2003B0F0BD9DF8053013F00100D5D09E
:1090E00001231360F4E700BFD4120020D81200203F
:1090F000DC1200202DE9F04FDFF8908100274D4D64
:1091000083B001263C46C2462846F9F70FFE2846A2
:10911000FEF78CF94848FEF789F96846FDF746FCEA
:1091200004EB440908EB49090AEB07054846FDF73B
:109130003DFC0028FAD06A7912F00102F6D1C4B3DE
:1091400099F80010134602E00133A3422FD018F81B
:10915000020006328842F7D103EB430C0AEB4C0CB9
:10916000B9F80100BCF801E08645EDD1B9F803E09B
:10917000BCF803C0F445E7D1FF2B18D000221346FA
:1091800002E00133A342D1D018F802C006328C4568
:10919000F7D103EB430C0AEB4C0CBCF801B0834550
:1091A000EFD1BCF803C0F445EBD1002BBED1142E97
:1091B00037D0731E122B3BD8DFE803F02F2D2B295D
:1091C000272523211F1D1B19171513110F0A310005
:1091D0001A4D01340136063796E7194DF9E7194D56
:1091E000F7E7194DF5E7194DF3E7194DF1E7194D7B
:1091F000EFE7194DEDE7194DEBE7194DE9E7194D8B
:10920000E7E7194DE5E7194DE3E7194DE1E7194D9A
:10921000DFE7194DDDE7194DDBE7194DD9E7194DAA
:10922000D7E71948F9F782FD012003B0BDE8F08FB8
:10923000004DCEE7CCF6000840DF000894F80008A7
:1092400074F8000854F8000838F800081CF8000802
:10925000FCF70008DCF70008C0F70008A4F70008D6
:1092600090F700087CF7000868F7000854F700083A
:1092700038F700081CF7000800F70008E4F60008BB
:10928000DCF60008B8F60008B0F80008DC12002090
:10929000F0B5124B83B01868E8B10025104F0426D2
:1092A0002C46052230466946FAF7E4F99DF800C0DD
:1092B000BDF80110BDF8032004EB4403013407F8A6
:1092C00005C007EB430305360635142CA3F801103F
:1092D000A3F80320E5D103B0F0BD00BFA404002033
:1092E000DC120020F0B5124B83B01868E8B10025FD
:1092F000104F04262C4604EB440307EB430317F8F6
:1093000005C0B3F801E0B3F80330052230466946E2
:1093100001348DF800C0ADF801E0ADF80330B618A7
:109320000635FAF7C1F9142CE5D103B0F0BD00BF42
:10933000A4040020DC12002010B5044682B00B46C5
:109340000092D02000222146FDF7D8F9D0F101008B
:1093500038BF002002B010BD10B5044682B00B46E5
:109360000092D02000222146FDF746FAD0F10100FC
:1093700038BF002002B010BD30B583B0FDF786F9CC
:109380003F200DF107010122FFF7D6FF054620B36C
:1093900001240720244B0DEB000122461C60FFF73F
:1093A000CBFF10B39DF80730002B29D100200DF121
:1093B00007010122FFF7C0FF0446B0B19DF8073056
:1093C0001A0619D503F07F0300200DF107010122D1
:1093D0008DF80730FFF7C0FF0EE00E200DF10701FA
:1093E0000122FFF7A9FF044618B90024204603B064
:1093F00030BD9DF807306BB90C4B01221A60F5E7C0
:10940000072000230DEB000122468DF80730FFF7FF
:10941000A3FFCBE70E200DF1070101228DF80750C5
:10942000FFF79AFFE8E700BF5C1300205413002009
:109430002DE9F04F474B89B01B681BB9184609B09E
:10944000BDE8F08F836802690193C36841690293A4
:10945000D0F800E0013246F26763C6F26663039219
:109460006439049183FB0EBA0199DDF80CB04768AA
:1094700083FB0118029A83FB0B1B83FB07C983FB49
:10948000022C049ACDF800B083FB02B20199059238
:10949000039B029ADDF810B04FEAEE76C6EBAA06FF
:1094A000DDF814A0FD17CC178069D117DA174FEA41
:1094B000EB73C5EBA905C1EBAC01C3EBAA03DDF867
:1094C00000C0059005EB850A03EB8300C4EBA804FC
:1094D0000090C2EBAC020198A7EB4A07DDF80CA0A4
:1094E00006EB860B04EB840902EB820CAEEB4B0E11
:1094F000A0EB4909DDF810B00298AAEB4C0CDDF89E
:1095000000A009EB041901EB8108059CA0EB4808B9
:10951000ABEB4A0008EB01180CEB021C00EB031349
:109520000EEB061E07EB05170134002006A90722E3
:109530008DF818E08DF819708DF81A908DF81B4091
:109540008DF81C808DF81DC08DF81E30FFF704FFCC
:1095500075E700BF541300202DE9F04F394B8BB055
:109560001B6804461BB900200BB0BDE8F08F00203B
:1095700008A90722FFF7E0FE0028F4D09DF825A0F7
:109580009DF820709DF826804FEA1A1B9DF8243024
:109590004FEA171C0BEB8B0B4FEA1819CDF81CB0D8
:1095A0000CEB8C0C05939DF822209DF8233009EBE1
:1095B000890908F00F08CDF800C0DDF81CC00AF0DA
:1095C0000F0ACDF80890CDF804809DF821501109BC
:1095D0000693DDF81490DDF80480059BCDF80CA00F
:1095E0000AEB4C0ADDF808C002F00F0201EB810122
:1095F0002E091B0909F00F0B02EB410108EB4C0986
:10960000069ADDF8008005F00F05049307F00F07B8
:1096100006EB860603EB830305EB460602F1FF3CEF
:1096200007EB48070BEB43030AF1FF3509F164022E
:1096300027606660A160C4F818C0E36025616261BC
:1096400092E700BF5413002000B50E4B83B01B6897
:1096500053B1FF23C0F20203984207D80022012031
:10966000094B1A6003B000BD1846FBE70122DF205A
:109670000DF10701F9F7FEFF9DF807200A2A88BFC0
:109680000022EDE7A40400205813002000B5094B88
:10969000094A1B68106883B08DF8073040B1DF209D
:1096A00001220DF10701F9F7FFFF003018BF01207B
:1096B00003B000BD58130020A404002041F2583329
:1096C000C2F200031868704710B541F25834C2F274
:1096D00000042060FFF7DAFF206810BD00B50D4BD5
:1096E00083B01B68FF200BB903B000BD112001A996
:1096F0000222FFF721FE0028F6D09DF80500064B58
:109700009DF80420C0F340001B6840EA4200C01AE4
:10971000EAE700BF541300205813002000B585B0BD
:1097200001A802A903AAF9F797FE10B9FF2005B016
:1097300000BD029B002BF9D1024B1868039B181A3D
:10974000F5E700BF6013002000B50E4B83B01B6827
:1097500053B1FF23C0F20203984207D80022012030
:10976000094B1A6003B000BD1846FBE70122DF2059
:109770000DF10701F9F77EFF9DF807200A2A88BF3F
:109780000022EDE7A40400206013002000B5094B7F
:10979000094A1B68106883B08DF8073040B1DF209C
:1097A00001220DF10701F9F77FFF003018BF0120FA
:1097B00003B000BD60130020A404002041F2603318
:1097C000C2F200031868704710B541F26034C2F26B
:1097D00000042060FFF7DAFF206810BD0920F9F7C8
:1097E000ADBE00BF00B5144B83B01B682BB1AA20DF
:1097F00012491022F9F73EFF50B910220F481049C4
:1098000001F076FD0F4B01221A60002003B000BD6D
:10981000BA2001A90222F9F72DFF0028EDD09DF80A
:1098200004109DF80520074B01202D291A60EDD169
:1098300052421A600120E9E7A4040020BC01002084
:10984000C0F80008B801002000B5134B83B01B68B6
:10985000002B1ADB2B228DF804208DF805300F4BDE
:109860001B6813B9002003B000BDAA200C491022C8
:10987000F9F71AFF0028F5D0BA20022201A9F9F75A
:1098800013FF003018BF0120EDE75B422D228DF859
:1098900004208DF80530E2E7B8010020A404002080
:1098A000BC01002040F2B813C2F2000318687047F0
:1098B00010B5014604460A48FDF770FE04F10C039A
:1098C000182B0AD8074B1A68A24204D01C60FFF775
:1098D000BBFF012010BD012010BD002010BD00BF46
:1098E000D0F80008B801002040F2BC10C2F200001D
:1098F000704700BF014640F2BC1008B5C2F200003C
:1099000001F0CDFCBDE80840FFF79EBF40F2BC105F
:10991000C2F20000FAF758BA70B5284A48F280132C
:109920001268C7F65543CB184FF4616101FB02334F
:1099300082B002AE46F8043D0546304601F06CF9AF
:1099400003690446DA1E052A0CD9022B2BD0092BF9
:1099500010D18369C268D21A182A03DD53B983680B
:10996000022B07DC019B304603F56163019301F094
:1099700053F90446636904F10C006B6123692B61A0
:10998000E368EB6007C8013102F26C72F6F7B0FCD5
:10999000A861236A2B62A368AB6063686B6023686D
:1099A0002B6002B070BD8369C268D21A182AE1DD4B
:1099B000002BD7D18368012BD4DCDBE7B801002072
:1099C00008B5202000F05AFB28B1202000F064FBED
:1099D000014B00221A6008BD641300202DE9F843F2
:1099E000DFF800E10646DEF80030002BFBD1002E48
:1099F0006FD03A48770007EB060C394984441825A4
:109A000010F8029CA5F11803A5F11008802212EAB3
:109A1000090F0CBF22243A24CC5401335208434589
:109A2000F5D110F8039CA5F10808802212EA090F6D
:109A30000CBF22243A24CC54013352084345F5D1BB
:109A400010F8018C802212EA080F0CBF22243A245D
:109A5000CC54013352089D42F5D10330183560458E
:109A6000CED10022CB18104698540132302AFBD1B7
:109A70004FF4305001240021C4F20100CEF8004020
:109A800000F03EFE1C200021C4F2020000F0DEFACD
:109A9000BB19DB0030331C204FF6F8711940C4F2BB
:109AA000020000F0E9FA1C2002212246C4F2020062
:109AB00000F0D8FA1C202146C4F2020000F0C6FAD9
:109AC0004FF43050C4F201002146BDE8F84300F0E5
:109AD00017BE334602493746C3E700BF6B13002069
:109AE0008017002064130020B0F5AE7F09D80A78F3
:109AF000044B00EB40001A544A78181842708B78D7
:109B00008370704768130020F0B469B10A4D01EB0F
:109B1000410700230678EC18EE544678033366704C
:109B20008678BB42A670F5D10AB9F0BC70470846EA
:109B3000F0BCFFF753BF00BF681300202DE9F041D0
:109B40005D4D94B0002468462C6000F013FB0420A7
:109B5000012100F0DBFC18234FF400604FF4807803
:109B6000C4F2010069468DF8033003238DF80230FA
:109B7000ADF8008000F09AFA4FF4006022464146AA
:109B8000C4F2010000F004FB02A800F0A5FD05A846
:109B900000F0ACFD01214FF4006000F0B7FC0120A3
:109BA000014600F0A5FC4FF430505B23C4F20100E5
:109BB00002A9ADF80C30ADF80840ADF80E40ADF894
:109BC0000A4000F0CDFC4FF4305060230126C4F26F
:109BD000010005A9ADF81430ADF81660ADF81A40D3
:109BE000ADF81C4000F01CFD4FF430500821C4F2C9
:109BF000010000F0C5FD4FF43050C4F201003146C1
:109C000000F0B0FD4FF43050C4F20100314600F0D6
:109C100085FD4FF4305032464FF40071C4F201001C
:109C200000F096FD0C2301A88DF804308DF8054056
:109C30008DF806408DF8076000F042F809A800F0A2
:109C4000F7F91C202146C4F2020000F0FFF91C20A5
:109C5000C4F2020000F020F942F63443C4F20103DA
:109C6000099342F2E8031C200C9380230E934FF4D7
:109C70004053129310230B93104BC4F2020009A916
:109C80001194CDF83C8010940D9413940A932746B8
:109C900000F0AEF98DF824408DF825408DF826406F
:109CA0002B68002BFCD109A840F25D110122FFF7BF
:109CB0002BFF14B0BDE8F081641300208017002052
:109CC000C37830B47BB90378012103F01F0201FA95
:109CD00002F15A094FF46143CEF20003203243F8F7
:109CE000221030BC70474FF46D43CEF20003DB68A6
:109CF0004478DB43C3F302230F22C3F1040122FAA9
:109D000003F304FA01F48578017803EA050222439B
:109D100001F160431201D2B203F5614383F80023DD
:109D20000278012102F01F0301FA03F14FF46143AD
:109D3000CEF20003520943F82210D2E742680B68C2
:109D400022F4702270B422F480720C79134343EA37
:109D50000423436086688C68CA684FF2FD73CFF6AF
:109D6000F1734D7922433340134343EA4503836043
:109D70000B7CC26A013B22F47002DBB242EA03535D
:109D8000C36270BC704700BF00230360037143715E
:109D90008360C36001230374704700BF836819B9EF
:109DA00023F001038360704743F001038360704731
:109DB000836843F008038360704700BF8068C0F386
:109DC000C0007047836843F004038360704700BF9E
:109DD0008068C0F380007047836819B923F4A0033A
:109DE0008360704743F4A00383607047092970B40F
:109DF00001EB41041ED91E3C072606FA04F603FABD
:109E000004F4C568062A25EA060343EA0403C3608E
:109E10001DD90C2A02EB820227D9413A1F2404FAE9
:109E200002F401FA02F1C36A23EA04020A43C2629D
:109E300070BC7047072606FA04F603FA04F40569B5
:109E4000062A25EA060343EA04030361E1D8013A3E
:109E500002EB82021F2404FA02F401FA02F1436BBE
:109E600023EA04020A434263E2E7233A1F2404FA86
:109E700002F401FA02F1036B23EA04020A430263CB
:109E8000D6E700BFC06C80B2704700BF03681942BC
:109E90000CBF002001207047082110B404684FF661
:109EA000FE72C4F202010023224088420260036075
:109EB00043608360C36050D01C23C4F20203984205
:109EC00052D03023C4F20203984255D04423C4F246
:109ED0000203984258D05823C4F2020398425BD040
:109EE0006C23C4F2020398425ED08023C4F20203C2
:109EF000984228D04FF48163C4F2020398422AD0DA
:109F000040F21C43C4F20203984255D04FF48663DA
:109F1000C4F20203984258D040F24443C4F2020310
:109F200098425BD04FF48B63C4F20203984201BFA6
:109F30004FF48063C4F202035A6842F4702208BFEF
:109F40005A6010BC70470023C4F202035A6842F002
:109F500070625A60F5E74FF48063C4F202035A68F6
:109F600042F00F025A60ECE70023C4F202035A6881
:109F700042F0F0025A60E4E70023C4F202035A6898
:109F800042F470625A60DCE70023C4F202035A68AC
:109F900042F470425A60D4E70023C4F202035A68C4
:109FA00042F470225A60CCE70023C4F202035A68DC
:109FB00042F470025A60C4E74FF48063C4F20203B3
:109FC0005A6842F0F0025A60BBE74FF48063C4F273
:109FD00002035A6842F470625A60B2E74FF4806339
:109FE000C4F202035A6842F470425A60A9E700BF03
:109FF0008B68F0B40D6A0C694A691D432C438B6968
:10A000001443CA6905684F6A23438E6A13431F438A
:10A0100025F4FF4525F070053E432E430660CB68CE
:10A0200043600B6883604B68C360F0BC704700BF3F
:10A030000023036043608360C36003614361836105
:10A04000C361036243628362704700BF29B902683B
:10A050004FF6FE73134003607047036843F001033B
:10A060000360704703681AB923EA01010160704771
:10A0700019430160704700BF41607047C1004CBF89
:10A080004FF480630023C4F202031B6803420CBF39
:10A0900000200120704700BFC3004CBF4FF4806315
:10A0A0000023C4F202035860704700BFCB782DE94B
:10A0B000F00303F00F06DB0648BF8B780A8848BF21
:10A0C0001E4312F0FF0F27D00768002301254FF031
:10A0D0000F0803E00133082B1CD00A8805FA03F4AB
:10A0E0002240A242F6D19C0008FA04F906FA04F4D0
:10A0F00091F803C027EA0907BCF1280F47EA0407D3
:10A1000008BF4261E6D0BCF1480F08BF02610133CD
:10A11000082BE2D107600A88FF2A28D94768002364
:10A1200001254FF00F0803E00133082B1ED00A88E9
:10A1300003F1080405FA04F42240A242F4D19C0081
:10A1400008FA04F906FA04F491F803C027EA0907AB
:10A15000BCF1280F04BF426191F803C02743BCF152
:10A16000480F08BF02610133082BE0D14760BDE80A
:10A17000F00370474FF6FF730380022383700423BC
:10A18000C3707047836819420CBF002001207047DC
:10A190000AB9416170470161704700BF30B40023C4
:10A1A0000028C4F2010300F44012B4BFDB695B680D
:10A1B000B2F5401F84B222D0C20217D5C0F30342C9
:10A1C000032505FA02F223EA020343F0706321B18A
:10A1D000420D120104FA02F423430022C4F20102E8
:10A1E0000028B4BFD361536030BC7047420D1201E8
:10A1F00004FA02F223EA020343F07063E7E7002265
:10A20000C4F20102556823F0706325F07065556053
:10A21000DDE700BF08B54FF4A843C4F2000398423D
:10A220000BD001214FF4800000F08CF94FF4800036
:10A230000021BDE8084000F085B901214FF400106D
:10A2400000F080F94FF400100021BDE8084000F054
:10A2500079B900BFF0B587B00446868801A80D46DD
:10A2600000F0F2F8039A4DF68363C4F21B33A3FBAC
:10A27000021326F03F06980C3604360C87B23E4394
:10A28000A680238848F2A06123F001031B041B0C65
:10A2900023802B68C0F201018B4222D85B00B2FB05
:10A2A000F3F292B201372784032A98BF0422A283D3
:10A2B00023889BB243F0010323802388698923F418
:10A2C0008163AA8823F002031B040A431B0C134377
:10A2D0009BB223802A89AB8913439BB2238107B0A9
:10A2E000F0BDEE884BF6FF718E421DBF03EB83037A
:10A2F00003EB8303B2FBF3F203EB43030CBFB2FBAC
:10A30000F3F242F4804292B213051B0D0BB942F0F6
:10A3100001024FF4967101FB00F044F6D351C1F2F3
:10A32000620181FB00318909013142F4004221843C
:10A33000BDE700BF002341F28832026083804BF604
:10A34000FF72038143814FF48043C2808381704751
:10A35000038829B923F001031B041B0C03807047F9
:10A360009BB243F001030380704700BF038829B903
:10A3700023F480731B041B0C038070479BB243F4CF
:10A3800080730380704700BF038829B923F40073EA
:10A390001B041B0C038070479BB243F400730380C3
:10A3A000704700BF038829B923F480631B041B0C8A
:10A3B000038070479BB243F480630380704700BF03
:10A3C00001827047008AC0B2704700BF1AB901F01D
:10A3D000FE010182704741F001010182704700BF18
:10A3E000038819B95B045B0C038070476FEA434331
:10A3F0006FEA53439BB20380704700BF82B00023D3
:10A400000A0F0093019301900092009B21F07F417D
:10A4100053B1019B14330193019B1B6819420CBF7C
:10A420000020012002B07047019B090C18330193F2
:10A43000F2E700BF4FF48053C4F202035A6822F4DB
:10A44000404210435860704710B44FF48053C4F238
:10A4500002035A6802F00C02042A01D0082A28D00C
:10A460004FF49052C0F27A0202604FF48053C4F26B
:10A4700002035C681C49C4F303140C5D22FA04F265
:10A4800042605C68C4F302240C5D22FA04F4846028
:10A490005C68C4F3C224095D22FA01F2C2605B6801
:10A4A0001249C3F38133CB5CB2FBF3F2026110BCFF
:10A4B00070475A685968C2F383420232CC030AD506
:10A4C0005B68990307D44FF49053C0F27A0303FBFF
:10A4D00002F20260C9E74FF41063C0F23D0303FBD0
:10A4E00002F20260C1E700BFD4010020D0010020C9
:10A4F0004FF48053C4F202035A6919B922EA0000EA
:10A500005861704710435861704700BF4FF4805343
:10A51000C4F202039A6919B922EA000098617047EF
:10A5200010439861704700BF4FF48053C4F2020398
:10A53000DA6919B922EA0000D86170471043D8617E
:10A54000704700BF4FF48053C4F202031A6919B96F
:10A5500022EA00001861704710431861704700BF7D
:10A5600070B44FF430524FF45054C4F201020388D7
:10A57000C4F20104904218BFA0429BB214BF002253
:10A58000012208D04FF48064C4F20004B0F1804F7F
:10A5900018BFA04236D14FF68F754C881D4045EA52
:10A5A00004034FF4A0564FF48055C4F20005C4F2E2
:10A5B0000006B04218BFA8421FBFCD884FF6FF4427
:10A5C0001C4044EA050303808B8883850B88038540
:10A5D0005AB94FF488424FF48043C4F20102C4F2E6
:10A5E0000103984218BF904205D10B7A03860123DC
:10A5F000838270BC70474FF49043C4F201039842C9
:10A60000F5D1F2E74FF440654FF40064C4F2000561
:10A61000C4F20004A04218BFA842C2D1BBE700BFE9
:10A62000038C2DE9F00123F001031B041B0C0384B0
:10A63000038C0D8984884F88028B2F4322F073028C
:10A6400023F002034FF450564FF4305512041B040C
:10A65000B1F800C0C4F20106C4F20105120C1B0CD3
:10A66000BFB2A84218BFB042A4B242EA0C0247EA05
:10A6700003030BD04FF488464FF48045C4F2010623
:10A68000C4F20105A84218BFB0421ED14FF6F775BB
:10A69000B1F80AC0B1F80E808F891D4045EA0C0C54
:10A6A0004FF6FB738E884FF6FF4548EA07072540B3
:10A6B0000CEA0303BCB233432C4384800283CA8870
:10A6C00082860384BDE8F00170474FF49045C4F2E0
:10A6D0000105A842F1D1D9E700234FF6FF7181802F
:10A6E0000380C38043800372704700BF0023038050
:10A6F00043808380C380038143818381C38170470A
:10A70000038829B923F001031B041B0C0380704745
:10A710009BB243F001030380704700BFB0F84430A0
:10A7200021B95B045B0CA0F8443070476FEA4343E7
:10A730006FEA53439BB2A0F84430704783899BB2C1
:10A740001AB923EA01018181704719438181704759
:10A7500083899BB21AB923EA0101818170471943A9
:10A7600081817047038829B923F080031B041B0CE7
:10A77000038070479BB243F080030380704700BFA3
:10A78000038B23F008031B041B0C19430183704740
:10A79000C94389B20182704770B5038ACA8823F41D
:10A7A00040531B041B0C13430382838904468A888D
:10A7B000088923F4B0530D4623F00C034989024362
:10A7C0001B040A431B0C13439BB2A381A38AAA89CF
:10A7D00023F440731B041B0C86B01343A38201A80F
:10A7E000FFF732FE4FF46053A289C4F201039C428A
:10A7F00012B20CBF049B039B002A21DB286803EBE9
:10A80000830303EB83038000B3FBF0F148F21F5393
:10A81000C5F2EB13A3FB0102A089520900B2160195
:10A820006425002802FB151213DB12013232A3FB50
:10A830000203C3F3431333439BB2238106B070BDBD
:10A840002A6803EB830303EB83035200B3FBF2F1AB
:10A85000DCE7D2003232A3FB0213C3F342133343CB
:10A86000EAE700BF4FF41652002302600C228380F7
:10A87000C380038142818381704700BF838929B9E6
:10A8800023F400531B041B0C838170479BB243F4D9
:10A8900000538381704700BF01F01F0310B4C1F360
:10A8A00042110124A14204FA03F30DD002290DD074
:10A8B00014302AB9026822EA0303036010BC70470F
:10A8C000026813430360F9E70C30F2E71030F0E759
:10A8D000C905C90D818070478088C005C00D7047CB
:10A8E000838919B95B045B0C838170476FEA43432A
:10A8F0006FEA53439BB28381704700BFC1F3421399
:10A9000010B401F01F020124012B04FA02F416D046
:10A91000022B0CBF028A828A92B222400123090ACA
:10A9200003FA01F103889BB219420CBF00200120F9
:10A93000002A0CBF002000F0010010BC7047828983
:10A9400092B22240EAE700BF090A012303FA01F3A9
:10A95000DB439BB2038070470649074A074B9A4284
:10A96000BEBF51F8040B42F8040BF8E704488047D7
:10A970000448004794FA000800000020A8020020C4
:10A9800011AA0008410100081F49204A002301E0E4
:10A9900041F8043B9142FBD3FCF778FFFEE7FEE76A
:10A9A000FEE7FEE7FEE7FEE7FEE7FEE7FEE7FEE77F
:10A9B000FEE7FEE7FEE7FEE7FEE7FEE7FEE7FEE76F
:10A9C000FEE7FEE7FEE7FEE7FEE7FEE7FEE7FEE75F
:10A9D000FEE7FEE7FEE7FEE7FEE7FEE7FEE7FEE74F
:10A9E000FEE7FEE7FEE7FEE7FEE7FEE7FEE7FEE73F
:10A9F000FEE7FEE7FEE7FEE7FEE7FEE7FEE7FEE72F
:10AA0000FEE7FEE7FEE7FEE7A8020020143A00207A
:10AA10004FF48053C4F202031968002241F001018F
:10AA200019605968CFF6FF020A405A601A6800217F
:10AA300022F0847222F480321A601A6882B022F402
:10AA400080221A6058681A4620F4FE0058604FF4BD
:10AA50001F00986000910191196841F480311960DC
:10AA600003E0009BB3F5A06F09D0136803F4003333
:10AA70000193009B01330093019B002BF1D04FF415
:10AA80008053C4F202031B6813F4003308BF019320
:10AA900001D001230193019B012B08D04FF46D439A
:10AAA000CEF200034FF000629A6002B070474FF49C
:10AAB0000052C4F2020211684FF4805341F01001B9
:10AAC00011601168C4F2020321F0030111601068E3
:10AAD000194640F0020010605A685A605A685A607D
:10AAE0005A6842F480625A605A6822F47C125A60B2
:10AAF0005A6842F4E8125A601A6842F080721A608A
:10AB00000A684FF480539201C4F20203F8D55968E1
:10AB10001A4621F003015960596841F00201596059
:10AB2000536803F00C03082BFAD1B7E74FF48053B6
:10AB3000C4F202035A6802F00C02082A1CBF4FF448
:10AB40009052C0F27A020DD04FF48053C4F2020347
:10AB50005B681049C3F30313CB5C22FA03F20E4B7C
:10AB60001A6070475A685968C2F383420232C803B8
:10AB700009D55B68990306D44FF49053C0F27A0369
:10AB800003FB02F2E0E74FF41063C0F23D0303FB66
:10AB900002F2D9E7E4010020F401002000210A229A
:10ABA00000F046BC08B5074B044613B10021AFF3D3
:10ABB0000080054B1868836A03B19847204601F06E
:10ABC00071F800BF00000000E8F8000870B50E4BF7
:10ABD0000E4D0024ED1AAD101E4603E056F8242059
:10ABE00090470134AC42F9D101F05EF8084D094BB1
:10ABF0000024ED1AAD101E4603E056F824209047BD
:10AC00000134AC42F9D170BDA0020020A0020020A6
:10AC1000A4020020A002002038B5074B05461C689E
:10AC2000E36B1BB9242000F00DF8E063E16B2846CC
:10AC3000BDE8384000F002B858020020002200F0C1
:10AC4000C3B80000024B0146186800F047BA00BFC5
:10AC50005802002010B5002302E0CC5CC45401333C
:10AC60009342FAD110BD8218034601E003F8011B9C
:10AC70009342FBD1704700002DE9F74F064600F0E4
:10AC80009FFF40F2B1739E42024640F396806FF4FC
:10AC9000F663F318A6F2B2719B1040F26D1505FB36
:10ACA0000135A6F26D716FF0630391FBF3F36FF45E
:10ACB000C861ED1871184FF4C87391FBF3F16D186A
:10ACC000642196FBF1FC01FB1C6C96FBF3F103FB8A
:10ACD00011614660D1F1010106F0030638BF002181
:10ACE00001960346022407261F7A4A2F11D15F6975
:10ACF000019805EB070810B9BCF1000F00D121B194
:10AD00003B2FD4BF0027012700E00F464744013FF7
:10AD10003FE0442F02D15F69EF193AE0019F37B954
:10AD2000BCF1000F0CBF89464FF0010900E08946D5
:10AD300023484FF0300808FB0909D3F80CA0A846B7
:10AD4000012705E009EB870B5BF804BC0137D84409
:10AD50005745F7DB08F1040797FBF6FB06FB1B7B67
:10AD60005F691869BAF1010FB8BF4FF0010AB7EB7C
:10AD70000B0748BF073700F1FF3B0AF1FF3A0720F6
:10AD800000FB0B7759F82A9000E0073F4F45FCDAAB
:10AD900047449869DFF82C80013C08FB0707186AD4
:10ADA000074443F81C7F9FD1936BD1699942ACBF94
:10ADB000002301231360012000E00020BDE8FE8F86
:10ADC000ECF80008805101002DE9F84380460C465C
:10ADD000174600F0F5FED8F800109B4A064691FB96
:10ADE000F2F302FB131104E001F5A83101F5C07183
:10ADF000013B0029F8DB4FF4616091FBF0F200FBAE
:10AE000012113C20A26091FBF0F200FB1211626073
:10AE100021601A1D072192FBF1F001FB1022002A8C
:10AE2000B8BF0732002BA26140F2B2754FF4C87070
:10AE30004FF0640CDFF81C9217DBA90704D195FBD7
:10AE4000FCF20CFB125242B995FBF0F100FB1151E0
:10AE5000D1F1010138BF002100E0012159F8212082
:10AE6000934218DB01359B1AE7E7013DAA0704D19D
:10AE700095FBFCF20CFB125242B995FBF0F100FB82
:10AE80001151D1F1010138BF002100E0012159F831
:10AE900021209B18E9D4A5F26C7262616B4A4FF0D5
:10AEA000300909FB01290022E361226102E001313E
:10AEB0009B1A2161216959F821209342F7DA013365
:10AEC000E360002F40F0BB8000F0A6FC604B1B68E5
:10AED0001BB373689D4205D13168D8F80030F26920
:10AEE00031B90CE02846FFF7C7FE0028F4D110E086
:10AEF00093420CDBB26B934209DA01230BE09342DD
:10AF0000FBDAB26B9342ACBF0023012303E00023C2
:10AF100001E04FF0FF33236200E02762236A4FF421
:10AF20006160012B0CBFF36B336A256893FBF0F271
:10AF300000FB12333C2093FBF0F100FB11336068FF
:10AF4000EB1A411AA0683B2BC2EB00022360616040
:10AF5000A26003DD013161603C3B04E0002B03DAB9
:10AF6000013961603C33236063683B2B03DD0132B0
:10AF7000A2603C3B04E0002B03DA013AA2603C33C0
:10AF80006360A368172B1FDDE2690132E261A269E9
:10AF90000132062AC8BF0022A261E268183B0132D2
:10AFA000A3602369E26059F823108A4244DD01332B
:10AFB000521A0C2BE26023613ED1626900230132F8
:10AFC00023616261E36137E0002B35DAE269013A1F
:10AFD000E261A269013A48BF0622A261E268183321
:10AFE000013AE260A3603ABB2369013B01D42361CB
:10AFF0001EE00B23236163695A1E12F0030F626186
:10B0000003F26B7305D1642293FBF2F102FB113260
:10B0100052B94FF4C87293FBF2F102FB1133D3F132
:10B02000010338BF002300E0012303F5B673E36199
:10B03000236959F82330E36000F0EFFB01E00023BF
:10B0400023622046BDE8F88380510100ECF8000837
:10B05000703800204CF9000830B500293BD051F879
:10B06000042C0B1F1C49002AB8BF9B180A6812B990
:10B070005A600B6030BD93420CD219685818904248
:10B0800003D15A588918426819605A60124A1360ED
:10B0900030BD0A46516809B19942FAD914681519A8
:10B0A0009D420AD11B68E318D0188842136012D160
:10B0B00008681B1813604B680CE002D90C2303606E
:10B0C00030BD18681C188C4203D10C6849680019FF
:10B0D00018605960536030BD6C380020F8B5CD1C45
:10B0E00025F0030508350C2D38BF0C25002D06462C
:10B0F00045DB8D4200D242E0234B1B681C4612E028
:10B100002268521B0DD40B2A02D92260A4181EE01B
:10B11000A34203D163681C4A136021E062685A604D
:10B120001EE023466468002CEAD123E03046214625
:10B1300000F06AF838602946304600F065F8431C94
:10B1400001461CD0C41C24F00304844201D12560B4
:10B1500006E03046611A00F057F80130F7D10EE0F2
:10B1600004F10B00231D20F00700C31A0AD05A4235
:10B17000E250F8BD054F3B68002BDCD1D6E70C232D
:10B1800033600020F8BD00BF6C3800206838002014
:10B190001A4B10B51C68A36BD3B91820FFF752FDEA
:10B1A00043F20E33A06303804AF6CD33438041F26D
:10B1B000342383804EF26D63C3804DF6EC630381CC
:10B1C000052343810B23838101220023C0E904234B
:10B1D000A46B0B492069626941430A4B03FB0212CD
:10B1E000A0FB0301511801220023121843EB0103B5
:10B1F000C4E9042323F0004010BD00BF5802002022
:10B200002DF451582D7F954C38B5064C002305463A
:10B210000846236000F02CFD431C02D1236803B1D3
:10B220002B6038BD103A00200EB400B54FF4027107
:10B230009CB0ADF814106FF00041049107914FF6E7
:10B24000FF711DABADF81610084953F8042B02909E
:10B250000690086802A9019300F0E6F9029B00221B
:10B260001A701CB05DF804EB03B070475802002060
:10B27000C9B2034610F8012B12B18A42F9D102E09B
:10B28000002918BF00231846704710F8012B11F849
:10B29000013B012A28BF9A42F7D0D01A70470346D3
:10B2A00011F8012B03F8012B002AF9D1704703464E
:10B2B00013F8012B002AFBD1181A0138704770B51A
:10B2C000A2B108E0012A03D128781B78C01A70BD0A
:10B2D000013A002CF8D00B460546002AF4D010F8AD
:10B2E000016B1C780131B442ECD0EDE7104670BD23
:10B2F00030B50139034609E011F8015F013A03F85E
:10B30000015B1C4615B99B18002205E01C46002A6B
:10B31000F2D1F8E704F8012B9C42FBD130BD0000CC
:10B320002DE9F74F01904148D0F8009008460446B7
:10B3300014F8015B09EB05067778204607F008074B
:10B34000FFB2002FF3D12D2D03D114F8015B01279B
:10B3500004E02B2D04BF244614F8015B002B5ED0C3
:10B36000102B08D158E02078782801D058284ED1E9
:10B37000657810230234002F0CBF6FF000404FF0AF
:10B380000040B0FBF3FA002603FB1A08304609EB35
:10B39000050C9CF801C00CF0040B5FFA8BFBBBF1B1
:10B3A000000F01D0303D0BE01CF0030C1BD0BCF1B2
:10B3B000010F14BF4FF0570C4FF0370CCCEB0505C5
:10B3C0009D4210DAB6F1FF3F0AD0504506D801D1B0
:10B3D000454503DC03FB0050012601E04FF0FF363A
:10B3E00014F8015BD3E7731C0AD1002F01990CBF3D
:10B3F0006FF000404FF0004022230B6022B912E0B2
:10B4000007B140427AB106B1611E11600BE03025F0
:10B41000002BB0D10823AEE7302DACD1A3E7302DFF
:10B42000A1D00A23A7E7BDE8FE8F00BF5C02002081
:10B4300030B51346044A05460C4610682946224694
:10B44000BDE83040FFF76CBF580200202DE9F74FF0
:10B4500001903D48D0F800900846044614F8015B7E
:10B4600009EB05067778204607F00807FFB2002FA2
:10B47000F3D12D2D03D114F8015B012704E02B2D0E
:10B4800004BF244614F8015B002B57D0102B08D1C1
:10B4900051E02078782801D0582847D165781023CA
:10B4A00002344FF0FF3ABAFBF3FA03FB0AF000262E
:10B4B0006FEA0008304609EB050C9CF801C00CF05F
:10B4C000040B5FFA8BFBBBF1000F01D0303D0BE0AA
:10B4D0001CF0030C1BD0BCF1010F14BF4FF0570C34
:10B4E0004FF0370CCCEB05059D4210DAB6F1FF3F6B
:10B4F0000AD0504506D801D1454503DC03FB005076
:10B50000012601E04FF0FF3614F8015BD3E7731C0E
:10B5100005D1019922230B60304622B912E007B110
:10B5200040427AB106B1611E11600BE03025002B5C
:10B53000B7D10823B5E7302DB3D1AAE7302DA8D075
:10B540000A23AEE7BDE8FE8F5C02002030B513464B
:10B55000044A05460C46106829462246BDE830409C
:10B56000FFF774BF580200202DE9F0478D6881462F
:10B57000AB420C4692461F463FD38A8912F4906F25
:10B5800039D0266809696369C1EB060803265E4362
:10B59000022508F1010302F4806296FBF5F6DB193F
:10B5A00012B29E4238BF1E4682B13146FFF796FD69
:10B5B000054600B913E021694246FFF74BFBA3891A
:10B5C00023F4906343F08003A3810CE0324600F043
:10B5D00022FB054638B948462169FFF73DFD0C239B
:10B5E000C9F8003018E0256166614544C8EB0606DD
:10B5F0002560A6603D46AF4200D23D462A462068FF
:10B60000514600F0EFFAA36800205B1BA36023689B
:10B610005D192560BDE8F087A3894FF0FF3043F046
:10B620004003A381BDE8F0872DE9F04F9DB003935F
:10B630008B89064603F080031BB20D46144663B1A6
:10B640000B6953B94021FFF749FD2860286110B903
:10B650000C233360D0E040236B6100230993202347
:10B660008DF82930DFF89C813023DFF89C918DF82C
:10B670002A3023469A4613F8012B1AB9BAEB040B69
:10B680000FD002E0252AF5D1F8E7304629462246B8
:10B690005B46FFF769FF013000F0A780099B5B4420
:10B6A00009939AF80030002B00F09F8000234FF0A0
:10B6B000FF3204930793059206938DF853301A9343
:10B6C0000AF1010A4FF0010B05E0C8EB00000BFA8C
:10B6D00000F00343049354464A482178052200F0C1
:10B6E00073FA0AF1010A049B0028EED1D90602D5AB
:10B6F00020228DF853201A0702D52B228DF85320D3
:10B7000022782A2A03D0079B21460A2010E0039AB8
:10B71000111D12680391002A01DB079204E05242D6
:10B7200043F0020307920493013408E000FB032373
:10B730000C4622780131303A092AF7D90793237849
:10B740002E2B19D163782A2B09D1039B02341A1DA1
:10B750001B680392002BB8BF4FF0FF330BE0611C56
:10B7600000230A2001E000FB03230C46227801316C
:10B77000303A092AF7D9059323482178032200F0AB
:10B7800023FA40B14023C9EB000003FA00F0049B08
:10B7900001340343049314F8011B1C4806228DF85E
:10B7A000281000F011FA88B1194B33B9039B073305
:10B7B00023F007030833039313E003AB00933046F1
:10B7C00004A92A46134BAFF3008007E003AB0093B4
:10B7D000304604A92A460F4B00F092F8431C074656
:10B7E00003D0099BDB19099343E7AB8903F04003BE
:10B7F0001BB20BB9099801E04FF0FF301DB0BDE856
:10B80000F08F00BF54F900085AF900085EF90008EB
:10B810000000000069B50008704770472DE9F04747
:10B8200015461F468A680B6906469A42A8BF13460A
:10B830002B6091F843200C46DDF820800AB10133DB
:10B840002B602368990602D52B6802332B6023688E
:10B8500013F0060916D094F843302268003318BF5D
:10B860000123920616D41EE0012330463946524683
:10B87000C047013003D14FF0FF30BDE8F08709F138
:10B88000010901E004F1190AE1682B68CB1A994516
:10B89000EADBE0E7E218302182F8431094F8451023
:10B8A000023382F844103046394604F14302C0475F
:10B8B0000130E0D023682A68E16803F00603042B16
:10B8C00008BFC2EB01052369A2680CBF25EAE57534
:10B8D00000259A42C4BFC3EB0203ED184FF00009E4
:10B8E0001A3408E00123304639462246C047013069
:10B8F000C1D009F10109A945F4DB0020BDE8F087BA
:10B900002DE9FF470E7E91466E2E80460C469A46E4
:10B910000C9D01F1430200F0AF800FD8632E1DD0C3
:10B9200006D8002E00F0C080582E40F0D0804FE0A6
:10B93000642E1CD0692E40F0CA8018E0732E00F0EF
:10B94000B78005D86F2E2BD0702E40F0C08043E01A
:10B95000752E25D0782E40F0BA8041E02B6801F199
:10B9600042071A1D1B682A6081F84230B3E0216843
:10B970002B6811F0800F02D0191D296008E011F02A
:10B98000400F03F10401296002D0B3F9005000E038
:10B990001D68002D45DA2D236D4284F8433040E0C8
:10B9A00021682B6811F0800F02D0191D296007E073
:10B9B00011F0400F03F10401296001D01D8800E05F
:10B9C0001D68237E5F486F2B14BF0A23082324E0E1
:10B9D00081F845605B4807E00B6843F020030B608B
:10B9E0007823594884F8453021682B6811F0800F7E
:10B9F00003F104062E6000D003E04F0601D51D8838
:10BA000000E01D68CE0744BF41F0200121601DB950
:10BA1000236823F0200323601023002184F84310BF
:10BA200001E048480A236668002EA66003DB21680F
:10BA300021F00401216005B96EB104F14201B5FBAA
:10BA4000F3F603FB1655455D0F4601F801593546DF
:10BA5000002EF4D100E01746082B0AD12368DB073B
:10BA600007D561682369994203DC302307F8013C5C
:10BA7000013FD21B226133E009682B6811F0800F6F
:10BA800005D0191D2960196863690B600CE011F07D
:10BA9000400F03F10401296003D0196863690B802A
:10BAA00002E061691B68196000232361174617E0F3
:10BAB0002B681A1D2A601F683846FFF7F8FB636879
:10BAC0002061984288BF23612369636005E004F127
:10BAD000420784F8426001232361002384F8433045
:10BAE000CDF800A04046214603AA4B46FFF796FE3C
:10BAF000013002D14FF0FF3021E0404649463A463E
:10BB00002369D0470130F5D0236898070ED4E06848
:10BB1000039B9842B8BF184611E0012340464946AE
:10BB20003246D0470130E5D0013502E0002504F16E
:10BB30001906E168039BCB1A9D42EEDBE7E704B0F0
:10BB4000BDE8F08765F9000876F9000830B5141EE5
:10BB50009BB0054604DA8B2303604FF0FF301DE0F5
:10BB60004FF40272ADF80C200091049101D0611ED7
:10BB700000E021464FF6FF7202910591ADF80E20CC
:10BB800028461A4669461E9BFFF74EFD431C01DA04
:10BB90008B232B6014B1009B00221A701BB030BDA8
:10BBA00073B50093054B06460D461446186831469A
:10BBB0002A462346FFF7CAFF7CBD00BF580200207B
:10BBC000004870476002002010B5C9B203468218D1
:10BBD00003E0047801338C4203D093421846F8D135
:10BBE000002010BD814210B511D28C18A0420ED297
:10BBF00053428118E418CB1801E0A15C995412F16A
:10BC0000FF32FAD210BDCC5CC454013300E00023F3
:10BC10009342F8D110BDF8B5064615460C4621B939
:10BC20001146BDE8F840FFF759BA1AB9FFF714FA00
:10BC30002C4612E000F013F8A8420ED230462946F6
:10BC4000FFF74CFA074638B121462A46FFF702F8BB
:10BC500030462146FFF700FA3C462046F8BD51F831
:10BC6000040C002802DA04390B58C0180438704755
:10BC7000094A136863B118186946884298BF106072
:10BC800004D9064B0C221A604FF0FF331846704758
:10BC9000034B1360EFE700BF74380020103A002018
:10BCA000183A0020FEE700BFF8B500BFF8BC08BC9A
:10BCB0009E467047F8B500BFF8BC08BC9E4670476A
:10BCC00065617374657220646174653A202530344F
:10BCD000642D253032642D253032640D0A000000B9
:10BCE000536F00004D6F0000446900004D69000073
:10BCF000446F00004672000053610000537500005D
:10BD000054750000576500005468000044434637EE
:10BD100037204572726F723A2048696768207075E3
:10BD20006C7365203C3D20350000000044434637DD
:10BD300037204572726F723A2048696768207075C3
:10BD40006C7365203E3D2032350000004443463789
:10BD500037204572726F723A20706172697479206F
:10BD6000503120696E636F72726563740000000069
:10BD70004443463737204572726F723A20706172C1
:10BD800069747920503220696E636F7272656374D2
:10BD9000000000004443463737204572726F723A04
:10BDA0002070617269747920503320696E636F72FC
:10BDB00072656374000000000000000000000000D5
:10BDC0003C42423C00000000241824427E424200D3
:10BDD00024003C4242423C002400424242423C0099
:10BDE0007C427C427C4040000000000000000000DB
:10BDF0000000000000000000000000000000000043
:10BE00000000000000000000000000000000000032
:10BE10000000000000000000000000000000000022
:10BE20000000000000000000000000000000000012
:10BE30000000000000000000000000000000000002
:10BE400000000000000000000000000000000000F2
:10BE500000000000000000000000000000000000E2
:10BE600000000000000000000000000000000000D2
:10BE700000000000000000000000000000000000C2
:10BE800000000000000000000000000000000000B2
:10BE900000000000000000000000000000000000A2
:10BEA0000000000000000000000000000000000092
:10BEB0000000000000000000000000000000000082
:10BEC0003838381000383800EEEE4400000000002A
:10BED0002828FE28FE2828007C92907C12927C0064
:10BEE000E2A4E8102E4A8E00304830708A847A002E
:10BEF0003838102000000000182040404020180072
:10BF00003008040404083000004428EE28440000EF
:10BF10000010107C101000000000003838102000C5
:10BF20000000007C000000000000000038383800ED
:10BF300002040810204080003844A2928A4438004D
:10BF40001030501010107C007C82027C8080FE003B
:10BF50007C82027C02827C00808484FE04040400D3
:10BF6000FE80807C02827C007C8280FC82827C005D
:10BF7000FE840810202020007C82827C82827C004B
:10BF80007C82827E02827C00102810001028100023
:10BF900038380038381020000810204020100800E1
:10BFA00000007C007C000000201008040810200025
:10BFB0007C82020C100010007C82BAAABC827C0039
:10BFC00010284482FE828200FC8282FC8282FC0075
:10BFD0007C82808080827C00FC8282828282FC0063
:10BFE000FE8080F88080FE00FE8080F880808000E7
:10BFF0007C82809E82827C00828282FE828282009B
:10C0000038101010101038000202020282827C00E8
:10C01000848890E090888400808080808080FE000A
:10C0200082C6AA928282820082C2A2928A868200FC
:10C030007C82828282827C00FC8282FC8080800002
:10C040007C8282828A847A00FC8282FC88848200DC
:10C050007C82807C02827C00FE1010101010100088
:10C060008282828282827C008282828244281000C4
:10C070008292929292926C0082442810284482000C
:10C080008244281010101000FE0408102040FE000A
:10C090007C40404040407C0080402010080402006A
:10C0A0007C04040404047C00102844000000000008
:10C0B000000000000000FE003838100800000000FA
:10C0C000001824427E424200007C427C42427C00B6
:10C0D000003C424040423C00007C424242427C00E4
:10C0E000007E407C40407E00007E407C404040001E
:10C0F000003C42404E423C000042427E42424200EE
:10C1000000080808080808000002020202423C0079
:10C1100000424478484442000040404040407E0095
:10C120000042665A42424200004262524A4642007F
:10C13000003C424242423C00007C42427C40400083
:10C14000003C42424A443A00007C42427C44420065
:10C15000003C403C02423C00003E08080808080041
:10C160000042424242423C00004242424224180005
:10C17000004242425A6642000042241818244200FB
:10C180000022140808080800007E040810207E0021
:10C19000384040C04040380010101000101010000F
:10C1A000380404060404380060920C00000000000B
:10C1B000000000000000000000000100010002007B
:10C1C000020003000300040004000500050006004F
:10C1D0000700080009000B000D000E0010001200FF
:10C1E0001400170019001C001F0021002400280063
:10C1F0002B002E003200360039003D004200460080
:10C200004A004F00540059005E00630069006E0050
:10C2100074007A00800086008C0093009900A000D2
:10C22000A700AE00B600BD00C500CD00D500DD0002
:10C23000E500EE00F600FF004E6F6E6500000000A6
:10C240005261696E626F77004661646500000000AC
:10C25000526F6C6C000000004578706C6F64650074
:10C2600052616E646F6D0000536E616B650000007B
:10C2700054656C65747970650000000043756265F3
:10C28000000000004D6174726978000044726F70A4
:10C290000000000053717565657A65004E6F726D20
:10C2A000616C0000436C6F636B3200000808090981
:10C2B0000A0A0B0B0C0C0D0D0E0E0F0000000000F7
:10C2C0000000000000052200000000000015220010
:10C2D0000000000000072200000000000012220001
:10C2E000000000000010220000000000000C2200EE
:10C2F00000000000000E22000000000000132200D9
:10C3000000000000001122000000000000172200C1
:10C3100000000000000F22000000000000162200B4
:10C320000000000000071722000000000012172282
:10C33000000000000010172200000000000B172270
:10C3400000000000000D172200000000001317225B
:10C350000000000000111722000000000019220058
:10C360000000000000041819220000000015181930
:10C3700022000000000718192200000000121819FE
:10C38000220000000010181922000000000C1819EB
:10C3900022000000000E18192200000000131819D6
:10C3A000220000000011181922000000001B2200CA
:10C3B000000000000004181B220000000015181BDC
:10C3C000220000000007181B220000000012181BAA
:10C3D000220000000010181B22000000000C181B97
:10C3E00022000000000E181B220000000013181B82
:10C3F000220000000011181B22000000001A220079
:10C40000000000000004181A220000000015181A8D
:10C41000220000000007181A220000000012181A5B
:10C42000220000000010181A22000000000C181A48
:10C4300022000000000E181A220000000013181A33
:10C44000220000000011181A22000000001C220027
:10C45000000000000004181C220000000015181C39
:10C46000220000000007181C220000000012181C07
:10C47000220000000010181C22000000000C181CF4
:10C4800022000000000E181C220000000013181CDF
:10C49000220000000011181C220000000000000013
:10C4A0000000000000091E220000000000151F22ED
:10C4B0000000000000071F220000000000121F22E1
:10C4C0000000000000101F2200000000000C1F22CE
:10C4D00000000000000E1F220000000000131F22B9
:10C4E0000000000000111F220000000000171F22A2
:10C4F00000000000000F1F220000000000161F2295
:10C50000000000000007171F220000000012171F84
:10C51000220000000010171F22000000000B171F50
:10C5200022000000000D171F220000000013171F3B
:10C53000220000000011171F2200000000191F2216
:10C5400000000000000418191F220000001518192F
:10C550001F220000000718191F22000000121819DE
:10C560001F220000001018191F220000000C1819CB
:10C570001F220000000E18191F22000000131819B6
:10C580001F220000001118191F220000001B1F228B
:10C59000000000000004181B1F2200000015181BDB
:10C5A0001F2200000007181B1F2200000012181B8A
:10C5B0001F2200000010181B1F220000000C181B77
:10C5C0001F220000000E181B1F2200000013181B62
:10C5D0001F2200000011181B1F220000001A1F223A
:10C5E000000000000004181A1F2200000015181A8D
:10C5F0001F2200000007181A1F2200000012181A3C
:10C600001F2200000010181A1F220000000C181A28
:10C610001F220000000E181A1F2200000013181A13
:10C620001F2200000011181A1F220000001C1F22E8
:10C63000000000000004181C1F2200000015181C38
:10C640001F2200000007181C1F2200000012181CE7
:10C650001F2200000010181C1F220000000C181CD4
:10C660001F220000000E181C1F2200000013181CBF
:10C670001F2200000011181C1F22000000410000B2
:10C680000000000000091E220000000000151F220B
:10C690000000000000071F220000000000121F22FF
:10C6A0000000000000101F2200000000000C1F22EC
:10C6B00000000000000E1F220000000000131F22D7
:10C6C0000000000000111F220000000000171F22C0
:10C6D00000000000000F1F220000000000161F22B3
:10C6E000000000000007171F220000000012171FA3
:10C6F000220000000103000000000000000B171FD3
:10C7000022000000000D171F220000000013171F59
:10C71000220000000011171F2200000001171F2037
:10C720002600000001111F202600000001131F2019
:10C7300026000000010E1F2026000000010C1F2013
:10C740002600000001101F202600000001121F20FB
:10C750002600000001071F202600000001151F20F1
:10C760002600000001091F2026000000012600000D
:10C770000000000001091E222600000001151F22F2
:10C780002600000001071F222600000001121F22C0
:10C790002600000001101F2226000000010C1F22AD
:10C7A00026000000010E1F222600000001131F2298
:10C7B0002600000001111F222600000001171F2281
:10C7C00026000000010F1F222600000001161F2274
:10C7D000260000000107171F222600000112171F64
:10C7E0002226000001240000000000000112171F93
:10C7F000200000000107171F2000000001161F2065
:10C8000000000000010F1F200000000001171F2082
:10C810000000000001111F200000000001131F2074
:10C8200000000000010E1F2000000000010C1F206E
:10C830000000000001101F200000000001121F2056
:10C840000000000001071F200000000001151F204C
:10C850000000000001091E2000000000004100004F
:10C860000000000000091E220000000000151F2229
:10C870000000000000071F220000000000121F221D
:10C880000000000000101F2200000000000C1F220A
:10C8900000000000000E1F220000000000131F22F5
:10C8A0000000000000111F220000000000171F22DE
:10C8B00000000000000F1F220000000000161F22D1
:10C8C000000000000007171F220000000012171FC1
:10C8D000220000000003220000000000000B171FD0
:10C8E00022000000000D171F220000000013171F78
:10C8F000220000000011171F2200000000191F2253
:10C900000000000001111F202600000001131F205D
:10C9100026000000010E1F2026000000010C1F2031
:10C920002600000001101F202600000001121F2019
:10C930002600000001071F202600000001151F200F
:10C940002600000001091E2026000000012600002C
:10C950000000000001091E222600000001151F2210
:10C960002600000001071F222600000001121F22DE
:10C970002600000001101F2226000000010C1F22CB
:10C9800026000000010E1F222600000001131F22B6
:10C990002600000001111F222600000001191F209F
:10C9A000000000000111171F200000000113171FD5
:10C9B00020000000010D171F20000000010B171FB1
:10C9C0002000000001240000000000000112171FD9
:10C9D000200000000107171F2000000001161F2083
:10C9E00000000000010F1F200000000001171F20A1
:10C9F0000000000001111F200000000001131F2093
:10CA000000000000010E1F2000000000010C1F208C
:10CA10000000000001101F200000000001121F2074
:10CA20000000000001071F200000000001151F206A
:10CA30000000000001091E2000000000004100006D
:10CA40000000000000091E220000000000151F2247
:10CA50000000000000071F220000000000121F223B
:10CA60000000000000101F2200000000000C1F2228
:10CA700000000000000E1F220000000000131F2213
:10CA80000000000000111F220000000000171F22FC
:10CA900000000000000F1F220000000000161F22EF
:10CAA000000000000007171F220000000012171FDF
:10CAB000220000000003220000000000000B171FEE
:10CAC00022000000000D171F220000000013171F96
:10CAD000220000000011171F2200000000191F2271
:10CAE0000000000001111F202600000001131F207C
:10CAF00026000000010E1F2026000000010C1F2050
:10CB00002600000001101F202600000001121F2037
:10CB10002600000001071F202600000001151F202D
:10CB20002600000001091E2026000000012600004A
:10CB30000000000001091E222600000001151F222E
:10CB40002600000001071F222600000001121F22FC
:10CB50002600000001101F2226000000010C1F22E9
:10CB600026000000010E1F222600000001131F22D4
:10CB70002600000001111F222600000001191F20BD
:10CB8000000000000111171F200000000113171FF3
:10CB900020000000010D171F20000000010B171FCF
:10CBA0002000000001032000000000000112171FF8
:10CBB000200000000107171F2000000001161F20A1
:10CBC00000000000010F1F200000000001171F20BF
:10CBD0000000000001111F200000000001131F20B1
:10CBE00000000000010E1F2000000000010C1F20AB
:10CBF0000000000001101F200000000001121F2093
:10CC00000000000001071F200000000001151F2088
:10CC10000000000001091E2000000000004100008B
:10CC20000000000000091E220000000000151F2265
:10CC30000000000000071F220000000000121F2259
:10CC40000000000000101F2200000000000C1F2246
:10CC500000000000000E1F220000000000131F2231
:10CC60000000000000111F220000000000171F221A
:10CC700000000000000F1F220000000000161F220D
:10CC8000000000000007171F220000000012171FFD
:10CC9000220000000103000000000000000B171F2D
:10CCA00022000000000D171F220000000013171FB4
:10CCB000220000000011171F2200000000191F228F
:10CCC0000000000001111F202600000001131F209A
:10CCD00026000000010E1F2026000000010C1F206E
:10CCE0002600000001101F202600000001121F2056
:10CCF0002600000001071F202600000001151F204C
:10CD00002600000001091E20260000000126000068
:10CD10000000000001091E222600000001151F224C
:10CD20002600000001071F222600000001121F221A
:10CD30002600000001101F2226000000010C1F2207
:10CD400026000000010E1F222600000001131F22F2
:10CD50002600000001111F222600000001191F20DB
:10CD6000000000000111171F200000000113171F11
:10CD700020000000010D171F20000000010B171FED
:10CD80002000000001240000000000000112171F15
:10CD9000200000000107171F2000000001161F20BF
:10CDA00000000000010F1F200000000001171F20DD
:10CDB0000000000001111F200000000001131F20CF
:10CDC00000000000010E1F2000000000010C1F20C9
:10CDD0000000000001101F200000000001121F20B1
:10CDE0000000000001071F200000000001151F20A7
:10CDF0000000000001091E200000000000410000AA
:10CE00000000000000091E220000000000151F2283
:10CE10000000000000071F220000000000121F2277
:10CE20000000000000101F2200000000000C1F2264
:10CE300000000000000E1F220000000000131F224F
:10CE40000000000000111F220000000000171F2238
:10CE500000000000000F1F220000000000161F222B
:10CE6000000000000007171F220000000012171F1B
:10CE7000220000000003220000000000000B171F2A
:10CE800022000000000D171F220000000013171FD2
:10CE9000220000000011171F2200000001171F20B0
:10CEA0002600000001111F202600000001131F2092
:10CEB00026000000010E1F2026000000010C1F208C
:10CEC0002600000001101F202600000001121F2074
:10CED0002600000001071F202600000001151F206A
:10CEE0002600000001091E20260000000126000087
:10CEF0000000000001091E222600000001151F226B
:10CF00002600000001071F222600000001121F2238
:10CF10002600000001101F2226000000010C1F2225
:10CF200026000000010E1F222600000001131F2210
:10CF30002600000001111F222600000001171F22F9
:10CF400026000000010F1F222600000001161F22EC
:10CF5000260000000107171F222600000112171FDC
:10CF60002226000001032000000000000112171F0C
:10CF7000200000000107171F2000000001161F20DD
:10CF800000000000010F1F200000000001171F20FB
:10CF90000000000001111F200000000001131F20ED
:10CFA00000000000010E1F2000000000010C1F20E7
:10CFB0000000000001101F200000000001121F20CF
:10CFC0000000000001071F200000000001151F20C5
:10CFD0000000000001091E20000000000000000009
:10CFE000000000000035000000000000002B0000E1
:10CFF00000000000003300000000000000320000CC
:10D0000000000000002E00000000000000300000C2
:10D0100000000000002800000000000000310000B7
:10D02000000000000029000000000000003800009F
:10D03000000000000037000000000000003D00007C
:10D04000000000000033380000000000003238000B
:10D0500000000000002E380000000000002F380003
:10D0600000000000002738000000000000313800F8
:10D070000000000000293800000000000039000016
:10D0800000000000002C363900000000002B36396B
:10D09000000000000033363900000000003236394D
:10D0A00000000000002E3639000000000030363944
:10D0B0000000000000283639000000000031363939
:10D0C000000000000029363900000000003B00008D
:10D0D00000000000002C363B00000000002B363B17
:10D0E000000000000033363B000000000032363BF9
:10D0F00000000000002E363B000000000030363BF0
:10D10000000000000028363B000000000031363BE4
:10D11000000000000029363B00000000003C000039
:10D1200000000000002C363C00000000002B363CC4
:10D13000000000000033363C000000000032363CA6
:10D1400000000000002E363C000000000030363C9D
:10D15000000000000028363C000000000031363C92
:10D16000000000000029363C00000000003E0000E6
:10D1700000000000002C363E00000000002B363E70
:10D18000000000000033363E000000000032363E52
:10D1900000000000002E363E000000000030363E49
:10D1A000000000000028363E000000000031363E3E
:10D1B000000000000029363E0000000000000000D2
:10D1C0000000000000212D3F0000000000212B4046
:10D1D0000000000000213340000000000021324028
:10D1E0000000000000212E4000000000002130401F
:10D1F0000000000000212840000000000021314014
:10D2000000000000002129400000000000213840FB
:10D2100000000000002137400000000000213D40D8
:10D2200000000000002133384000000000213238A7
:10D230004000000000212E384000000000212F385F
:10D240004000000000212738400000000021313854
:10D250004000000000212938400000000021394032
:10D260000000000000212C363940000000212B3640
:10D2700039400000002133363940000000213236A9
:10D280003940000000212E363940000000213036A0
:10D290003940000000212836394000000021313695
:10D2A00039400000002129363940000000213B4070
:10D2B0000000000000212C363B40000000212B36EE
:10D2C0003B400000002133363B4000000021323655
:10D2D0003B40000000212E363B400000002130364C
:10D2E0003B400000002128363B4000000021313641
:10D2F0003B400000002129363B40000000213C401B
:10D300000000000000212C363C40000000212B369C
:10D310003C400000002133363C4000000021323602
:10D320003C40000000212E363C40000000213036F9
:10D330003C400000002128363C40000000213136EE
:10D340003C400000002129363C40000000213E40C6
:10D350000000000000212C363E40000000212B364A
:10D360003E400000002133363E40000000213236AE
:10D370003E40000000212E363E40000000213036A5
:10D380003E400000002128363E400000002131369A
:10D390003E400000002129363E4000000000000011
:10D3A000000000000111181C1F2000000113181CB0
:10D3B0001F200000010E181C1F200000010C181C6B
:10D3C0001F2000000110181C1F2000000112181C53
:10D3D0001F2000000107181C1F2000000115181C49
:10D3E0001F2000000104181C1F200000011C1F202A
:10D3F000000000000111181A1F2000000113181A64
:10D400001F200000010E181A1F200000010C181A1E
:10D410001F2000000110181A1F2000000112181A06
:10D420001F2000000107181A1F2000000115181AFC
:10D430001F2000000104181A1F20000001191F20DE
:10D44000000000000111181B1F2000000113181B11
:10D450001F200000010E181B1F200000010C181BCC
:10D460001F2000000110181B1F2000000112181BB4
:10D470001F2000000107181B1F2000000115181BAA
:10D480001F2000000104181B1F200000011B1F208B
:10D4900000000000011118191F20000001131819C5
:10D4A0001F200000010E18191F200000010C181980
:10D4B0001F200000011018191F2000000112181968
:10D4C0001F200000010718191F200000011518195E
:10D4D0001F200000010418191F20000001191F203F
:10D4E000000000000111171F200000000113171F8A
:10D4F00020000000010D171F20000000010C171F65
:10D50000200000000110171F200000000112171F4B
:10D51000200000000107171F2000000001161F2037
:10D5200000000000010F1F200000000001171F2055
:10D530000000000001111F200000000001131F2047
:10D5400000000000010E1F2000000000010C1F2041
:10D550000000000001101F200000000001121F2029
:10D560000000000001071F200000000001151F201F
:10D570000000000001091E200000000000173A0012
:10D5800000000000001723263A000000000F3A00B8
:10D5900000000000000F23263A00000000163A00A9
:10D5A00000000000001623263A0000000007173A8A
:10D5B0000000000000071723263A00000012173A67
:10D5C0000000000000121723263A00000010173A4E
:10D5D0000000000000101723263A0000000B173A45
:10D5E00000000000000B1723263A0000000D173A38
:10D5F00000000000000D1723263A00000013173A20
:10D600000000000000131723263A00000011173A0B
:10D610000000000000111723263A000000193A000C
:10D6200000000000001923263A0000000004181929
:10D630003A0000000004181923263A0000151819B2
:10D640003A4900000015181923263A49000718190D
:10D650003A4900000007181923263A490012181900
:10D660003A4900000012181923263A4900101819E7
:10D670003A4900000010181923263A49000C1819DD
:10D680003A490000000C181923263A49000E1819CF
:10D690003A490000000E181923263A4900131819B8
:10D6A0003A4900000013181923263A4900111819A5
:10D6B0003A4900000011181923263A49001B3A493B
:10D6C00000000000001B23263A4900000004181B3C
:10D6D0003A4900000004181B23263A490015181B7C
:10D6E0003A4900000015181B23263A490007181B69
:10D6F0003A4900000007181B23263A490012181B5C
:10D700003A4900000012181B23263A490010181B42
:10D710003A4900000010181B23263A49000C181B38
:10D720003A490000000C181B23263A49000E181B2A
:10D730003A490000000E181B23263A490013181B13
:10D740003A4900000013181B23263A490011181B00
:10D750003A4900000011181B23263A490000000036
:10D7600000000000000000000000000000000000B9
:10D7700000000000000000000000000000000000A9
:10D780000000000000000000000000000000000099
:10D790000000000000000000000000000000000089
:10D7A0000000000000000000000000000000000079
:10D7B0000000000000000000000000000000000069
:10D7C0003D000000350000002B0000003300000089
:10D7D000320000002E000000300000002800000091
:10D7E0003100000029000000380000003700000070
:10D7F0003D000000350000002B0000003300000059
:10D80000320000002E000000300000002800000060
:10D81000310000002900000038000000370000003F
:10D820003D0000003D4100002C4100002B41000064
:10D8300033410000324100002E4100003041000021
:10D84000284100003141000029410000384100001A
:10D85000374100003D4100002C4100002B410000F9
:10D8600033410000324100002E41000030410000F1
:10D8700028410000314100002941000038410000EA
:10D88000374100003D4100003D4147002C41470029
:10D890002B41470033414700324142482E41424824
:10D8A00030414800284148003141480029414800A2
:10D8B0003841434A3741434A3D414A002C414A00DE
:10D8C0002B41464A3341464A3241464A2E41464A56
:10D8D0003041440028414400314144002941440082
:10D8E00038414400374147003D4147002A4100008C
:10D8F0002C4100002B410000334100003241000068
:10D900002E4100003041000028410000314100005C
:10D910002941000038410000374100003D4100002E
:10D9200033384100323841002E3841002F38410051
:10D930002738410031384100293841003941000081
:10D940002C3639412B36394133363941323639415B
:10D95000141D0000041D0000151D0000071D00001F
:10D96000121D0000101D00000C1D00000E1D000007
:10D97000131D0000111D0000171D00000F1D0000E9
:10D98000161D0000041D0000151D0000071D0000ED
:10D99000121D0000101D00000C1D00000E1D0000D7
:10D9A000131D0000111D0000171D00000F1D0000B9
:10D9B000161D0000141D0000041D0000151D0000B0
:10D9C000071D0000121D0000101D00000C1D0000AE
:10D9D0000E1D0000131D0000111D0000171D00008A
:10D9E0000F1D0000161D000007171D0012171D0057
:10D9F00010171D000B171D000D171D0013171D001C
:10DA000011171D00191D00000418191D1518191DE6
:10DA10000718191D1218191D45000000000000000C
:10DA200000000000000000000000000000000000F6
:10DA300000000000000000000000000000000000E6
:10DA400000000000000000000000000000000000D6
:10DA500000000000000000000000000000000000C6
:10DA600000000000000000000000000000000000B6
:10DA70000000000000000000450000006868206D04
:10DA80006D202831322900006868206D6D20283211
:10DA900034290000686820756E64206D6D2028317F
:10DAA00032290000686820756E64206D6D20283270
:10DAB000342900006D6D206E61636820686820283D
:10DAC00031322B29000000006D6D206E61636820EB
:10DAD00068682028323429004F7373692F426572B9
:10DAE0006C696E2028313229000000004F73736981
:10DAF0002F4265726C696E202831322B290000009C
:10DB00004F65736920283132290000004F65736921
:10DB1000202831322B290000526865696E2F52751A
:10DB20006872202831322900526865696E2F52755B
:10DB30006872202831322B29000000005363687777
:10DB40006162656E202831322900000053636877D6
:10DB50006162656E202831322B290000576573738E
:10DB600069202831322900005765737369202831F4
:10DB7000322B2900436F756E74646F776E0000005E
:10DB800054656D706572617475720000000000006C
:10DB90000002000303000707000E03000E04000F3D
:10DBA000020100040102030102040102050107044D
:10DBB000010705010B04010B060200030202040227
:10DBC0000604020A04020E04030004030404030909
:10DBD00005030E04040003040407040B07050008F2
:10DBE000050807050F0306000606000706080306DA
:10DBF0000B03060E0407000307030B070707070EB6
:10DC000004080004080006080504080804080C04B9
:10DC1000080E03080E040900040904040904050998
:10DC20000A04090E040A00040A02030A02040A068E
:10DC3000030A0A030A0E040B00070B07040B0A0869
:10DC40000C00070C07050C0B070D00060D00070D57
:10DC500007030D0B040D0F030E00060E060B0E0C32
:10DC6000040E0C060F00070F07040F0B070000003F
:10DC7000070500007CDA00080706000088DA0008C3
:10DC80000805000094DA000808060000A4DA00087D
:10DC900001030000B4DA000801040000C8DA00083B
:10DCA00002010000D8DA000802030000ECDA0008E4
:10DCB0000301000000DB0008030300000CDB000888
:10DCC0000401000018DB00080403000028DB000842
:10DCD000050200003CDB0008050300004CDB0008E7
:10DCE000060100005CDB00080603000068DB00089A
:10DCF0000907000074DB00080A00000080DB000850
:10DD00002800000054696D656F757400290D0A00C4
:10DD10004F4B00004552524F520000002D20000092
:10DD20004950414444524553532000004150200083
:10DD30004D4F4445200000006170000054494D459E
:10DD4000200000004649524D574152452000000036
:10DD5000434D44200000000048545450204745548F
:10DD6000200000002D2D3E20000000003C30643ECD
:10DD70003C30613E0D0A00003C253032783E000008
:10DD800063617020222573222C222573220000005B
:10DD9000617020222573222C2225732200000000AE
:10DDA00074696D65202225732200000045535038A8
:10DDB000323636204C4F474745520D0A00000000CE
:10DDC00070EB000878EB000880EB000888EB000897
:10DDD0008CEB000890EB000894EB000898EB00082F
:10DDE000A8E40008B0E40008B8E4000860F7000800
:10DDF000BCE40008C8DE0008C8DE0008C8DE000871
:10DE0000C8DE0008C8DE00080400000002000000B0
:10DE1000020000000200000002000000A0EB000869
:10DE2000ACEB000870EB000878EB000898EB0008FA
:10DE3000A4E80008A8E80008B0E800080CE800081A
:10DE4000B0EB0008B4EB000860E9000860E90008E6
:10DE500060E90008B8EB0008B8EB0008B8EB000870
:10DE600070EB0008BCEB00084CE20008CCEB0008AB
:10DE700098EB000870EB0008BCEB00084CE20008CF
:10DE800098EB0008D8EB0008E0EB0008E8EB00088E
:10DE9000ECEB0008F4EB0008F8EB000810E80008D1
:10DEA00098EB00086163746976650000257325644A
:10DEB00000000000485454502F312E3020323030B2
:10DEC000204F4B000D0A0D0A000000003C68746DE5
:10DED0006C3E0D0A000000003C686561643E0D0A5E
:10DEE000000000003C7469746C653E003C2F74694E
:10DEF000746C653E0D0A00003C2F686561643E0D40
:10DF00000A0000003C626F64793E0D0A00000000C8
:10DF10003C48313E0D0A00003C2F48313E0D0A00BE
:10DF20003C6120687265663D222F0000223E0000A1
:10DF30003C2F613E266E6273703B266E6273703BAF
:10DF40000D0A00004D61696E000000006E65747777
:10DF50006F726B004E6574776F726B0054656D70F5
:10DF600065726174757265006C6472004C44520095
:10DF7000446973706C617900616E696D6174696F79
:10DF80006E730000416E696D6174696F6E7300009D
:10DF9000616D62696C69676874000000416D626957
:10DFA0006C6967687400000074696D6572730000C5
:10DFB00054696D65727300003C503E003C747220E1
:10DFC0006267636F6C6F723D236630663066303E09
:10DFD0000D0A00003C74723E0D0A00003C74643E61
:10DFE000000000003C2F74643E0000003C696E702D
:10DFF000757420747970653D227465787422206987
:10E00000643D220022206E616D653D22000000000B
:10E01000222076616C75653D2200000022206D6132
:10E02000786C656E6774683D220000002220736979
:10E030007A653D22000000003C74643E3C627574C9
:10E04000746F6E20747970653D227375626D6974AA
:10E0500022206E616D653D22616374696F6E2220BE
:10E0600076616C75653D227361766500223E53656D
:10E07000743C2F627574746F6E3E00003C2F7464A4
:10E080003E0D0A003C7461626C6520626F726465CB
:10E09000723D303E0D0A00003C2F74723E0D0A00A6
:10E0A0003C74683E3C666F6E7420636F6C6F723DAB
:10E0B000626C75653E0000003C2F666F6E743E3CDE
:10E0C0002F74683E0D0A00003C2F7461626C653E3F
:10E0D0003C503E0D0A0000003C627574746F6E2067
:10E0E000747970653D227375626D697422206E616A
:10E0F0006D653D22616374696F6E222076616C7577
:10E10000653D22003C2F627574746F6E3E266E6210
:10E1100073703B003C2F626F64793E0D0A00000073
:10E120003C2F68746D6C3E0D0A0000003C73656CFA
:10E130006563742069643D2200000000223E0D0AE0
:10E14000000000003C2F73656C6563743E0D0A008F
:10E150003C6F7074696F6E2076616C75653D22004E
:10E160002073656C65637465640000003C2F6F70FC
:10E1700074696F6E3E0D0A00266E6273703B3C69D7
:10E180006E70757420747970653D22636865636B89
:10E19000626F7822206E616D653D220022207661DB
:10E1A0006C75653D2261637469766522200000000C
:10E1B000636865636B6564003C696E707574207498
:10E1C0007970653D2272616E6765222069643D2227
:10E1D0000000000022206D696E3D220022206D614A
:10E1E000783D220022207374796C653D2277696442
:10E1F00074683A0070783B0022206F6E696E70750B
:10E20000743D22005F6F75747075742E76616C7545
:10E21000653D00002E76616C7565223E00000000B1
:10E220003C6F7574707574206E616D653D220000E1
:10E230005F6F7574707574223E0000003C2F6F751F
:10E24000747075743E0000002E0D0A00446566610E
:10E25000756C7400313500003C666F726D206D6521
:10E2600074686F643D224745542220616374696F6E
:10E270006E3D222F000000003C2F666F726D3E0D38
:10E280000A000000436F6C6F727300003C74643EC0
:10E290000D0A000036340000266E6273703B266E55
:10E2A0006273703B266E6273703B0D0A00000000C3
:10E2B0004C6561726E696E672049522072656D6FA0
:10E2C000746520636F6E74726F6C2E2E2E000000CA
:10E2D000537769746368696E6720706F7765722021
:10E2E0006F6E2E2E2E000000537769746368696E7E
:10E2F0006720706F776572206F66662E2E2E000085
:10E300006F66666C696E65004D696E696D756D202E
:10E310006C656E677468206F66206B657920697321
:10E32000203130210000000054696D6573657276FC
:10E330006572207375636365737366756C6C7920A1
:10E340006368616E6765642E000000005365747435
:10E35000696E67206F66206E65772074696D6573DE
:10E360006572766572206661696C65642E000000D6
:10E3700054696D657A6F6E65207375636365737339
:10E3800066756C6C79206368616E6765642E000049
:10E3900053657474696E67206F66206E65772074AC
:10E3A000696D657A6F6E65206661696C65642E00C3
:10E3B00047657474696E67206E65742074696D6555
:10E3C00000000000446973706C6179696E672074A5
:10E3D000656D70657261747572652E2E2E00000079
:10E3E00053746F726564206D696E696D756D20760A
:10E3F000616C75650000000054657374696E672078
:10E40000646973706C61792E2E2E000053617669F9
:10E410006E672073657474696E6773207065726DC2
:10E42000616E656E746C792E2E2E000068747470A7
:10E4300020706174683A20272573270D0A000000B8
:10E440006874747020706172616D65746572733A7E
:10E4500020272573270D0A002F0000002530326485
:10E460002E253032640000002534640025303264EB
:10E4700000000000616374696F6E00006C6561727A
:10E480006E697200706F7765726F6E00706F77657E
:10E49000726F666600000000736176656461746582
:10E4A00074696D650000000079656172000000000C
:10E4B0006D6F6E7468000000646179006D696E00B4
:10E4C000736176657469636B65720000576F72647F
:10E4D000436C6F636B00000056657273696F6E006A
:10E4E000454550524F4D0000454550524F4D205626
:10E4F000657273696F6E00005469636B657200002A
:10E50000506F776572204F6E00000000506F776586
:10E5100072204F66660000004C6561726E204952A1
:10E520002072656D6F746520636F6E74726F6C001E
:10E53000656570726F6D64756D7000004545505271
:10E540004F4D2064756D70003C503E0D0A3C666F67
:10E550006E7420636F6C6F723D677265656E3E000E
:10E560003C5052453E000000253034780000000049
:10E57000202000003C2F5052453E0000202020006B
:10E580002F6E6574776F726B0000000073617665A3
:10E59000776C616E00000000776C616E6D6F646572
:10E5A000000000007373696400000000576F72641C
:10E5B000436C6F636B204E6574776F726B00000065
:10E5C0003C423E436F6E6E656374696E6720746F84
:10E5D0002041636365737320506F696E742C2074DF
:10E5E000727920616761696E206C617465722E3C7E
:10E5F0002F423E003C423E53746174696E67206155
:10E60000732041636365737320506F696E742C20AF
:10E6100074727920616761696E206C617465722E15
:10E620003C2F423E000000007361766574696D65A1
:10E6300073657276657200007361766574696D65E5
:10E640007A6F6E65000000006E657474696D650018
:10E6500049502061646472657373000045535038FB
:10E66000323636206669726D77617265000000008F
:10E67000574C414E00000000535349440000000035
:10E68000266E6273703B266E6273703B266E6273F9
:10E69000703B00004B65790054696D6520736572AD
:10E6A0007665720054696D65207A6F6E6520284723
:10E6B0004D54202B29000000476574206E6574209E
:10E6C00074696D65000000003C503E0D0A3C666FA9
:10E6D0006E7420636F6C6F723D7265643E3C423EA7
:10E6E000000000003C2F423E3C2F666F6E743E0DD2
:10E6F0000A0000002F74656D706572617475726533
:10E70000000000007361766574636F7272727463E7
:10E71000000000007361766574636F727264733118
:10E7200038787800646973706C617974656D7065B0
:10E7300072617475726500002E350000266465678D
:10E740003B430000576F7264436C6F636B205465EA
:10E750006D706572617475726500000052544320DB
:10E7600074656D70657261747572650044533138FB
:10E770007878000054656D7020636F727265637401
:10E78000696F6E205254432028756E697473206F30
:10E790006620302E35B043290000000054656D70AE
:10E7A00020636F7272656374696F6E2044533138F1
:10E7B00078782028756E697473206F6620302E3546
:10E7C000B0432900446973706C61792074656D7081
:10E7D00065726174757265002F6C647200000000D0
:10E7E0006C64726D696E00006C64726D617800001B
:10E7F000736176656175746F000000002575000017
:10E80000576F7264436C6F636B204C44520000007E
:10E810004D696E004D6178004175746F6D6174696A
:10E8200063206272696768746E657373000000002C
:10E83000536574206173206D696E696D756D207606
:10E84000616C756500000000536574206173206D74
:10E850006178696D756D2076616C756500000000EA
:10E860002F646973706C61790000000073617665D4
:10E8700069746973000000007361766573796E6373
:10E88000616D62690000000073617665627269679C
:10E8900068746E657373000073617665636F6C6F87
:10E8A0007273000072656400677265656E00000037
:10E8B000626C756500000000736176656469737051
:10E8C0006C61796D6F6465007361766574696E74EF
:10E8D000657276616C0000007465737464697370AE
:10E8E0006C61790073617665616C6C00576F72645E
:10E8F000436C6F636B20446973706C617900000036
:10E9000045532049535400005065726D616E656E29
:10E910007420646973706C6179206F66202245539E
:10E920002049535422000000446973706C617920BF
:10E930004D6F646500000000557365206469737055
:10E940006C617920636F6C6F72730000427269674B
:10E9500068746E6573732028312D313529000000ED
:10E960003000000054656D7020646973706C6179CB
:10E9700020696E74657276616C0000005465737472
:10E9800020646973706C61790000000053617665E2
:10E9900020616C6C000000002F616E696D6174690C
:10E9A0006F6E730073617665616E696D6174696F16
:10E9B0006E00000073617665636F6C6F72616E69E3
:10E9C0006D6174696F6E00006465660073617665E1
:10E9D000616E00007370256400000000666176259A
:10E9E000640000007361766563616E006373702577
:10E9F000640000006364656600000000576F726485
:10EA0000436C6F636B20416E696D6174696F6E73E7
:10EA100000000000416E696D6174696F6E00000056
:10EA2000436F6C6F7220416E696D6174696F6E0027
:10EA3000616E2564000000006465662564000000C6
:10EA40003100000063616E25640000006364656648
:10EA5000256400002F616D62696C6967687400004D
:10EA600073617665616D62696D6F646500000000B9
:10EA700073617665616D62696C65647300000000A6
:10EA800073617665616D62696F66667365740000B7
:10EA90007361766561616E006173702564000000CA
:10EAA0006164656600000000576F7264436C6F63B9
:10EAB0006B20416D62696C6967687400234C454442
:10EAC000730000004F6666736574206F662073657F
:10EAD000636F6E64203D203000000000416D62696C
:10EAE0006C69676874204D6F6465000061616E2514
:10EAF0006400000061646566256400002F74696D20
:10EB000065727300736176656964000061000000DE
:10EB10006F0000006625640074256400576F7264FE
:10EB2000436C6F636B2054696D6572730000000065
:10EB30006964256400000000612564006F2564009D
:10EB4000682564006D256400485454502F312E30E0
:10EB500020343034204E6F7420466F756E64000090
:10EB6000343034204E6F7420466F756E640D0A0089
:10EB70004E616D650000000056616C756500000017
:10EB800059595959000000004D4D000044440000FF
:10EB9000686800006D6D0000416374696F6E00006D
:10EBA000574C414E20436C69656E74004150000023
:10EBB00047000000420000003633000044656365F2
:10EBC0006C65726174696F6E000000004661766F5B
:10EBD0007572697465000000536C6F74000000006A
:10EBE00041637469766500004F6E000046726F6D78
:10EBF00000000000546F0000486F757200000000B4
:10EC0000010000000F0000001500000007000000D8
:10EC10000B000000070000000B00000007000000D0
:10EC20000B0000000F0000001400000000000000B6
:10EC30000F000000140000000000000001000000B0
:10EC40000000000005000000020000000B000000B2
:10EC50000C0000001A000000020000000B00000081
:10EC6000020000000B000000000000001000000087
:10EC70001C0000002800000030000000010000001F
:10EC8000010000000000000002000000050000007C
:10EC90000C00000011000000220000000500000030
:10ECA0000C000000050000000C0000000000000047
:10ECB00010000000100000002000000020000000F4
:10ECC0000100000001000000000000000200000040
:10ECD000050000000C0000001100000022000000F0
:10ECE000050000000C000000050000000C00000002
:10ECF0000000000000000000000000000000000014
:10ED00000000000001000000010000000000000001
:10ED100003000000050000000C0000000F000000D0
:10ED20001E000000050000000C00000004000000B0
:10ED30000B000000000000001000000015000000A3
:10ED40002500000025000000010000000100000077
:10ED500000000000322E302E360000000D0A5765EC
:10ED60006C636F6D6520746F20576F7264436C6FB6
:10ED7000636B204C6F676765722100002D2D2D2D70
:10ED80002D2D2D2D2D2D2D2D2D2D2D2D2D2D2D2DB3
:10ED90002D2D2D2D2D2D2D2D00000000566572736B
:10EDA000696F6E3A20000000727463206973206FEF
:10EDB0006E6C696E65000000727463206973206F69
:10EDC00066666C696E650000656570726F6D2069BE
:10EDD00073206F6E6C696E6500000000637572725F
:10EDE000656E7420656570726F6D207665727369EB
:10EDF0006F6E3A203078253038780D0A0000000018
:10EE000072656164696E6720697220636F646573FF
:10EE10002066726F6D20656570726F6D0000000076
:10EE200072656164696E6720646973706C617920D2
:10EE3000636F6E66696775726174696F6E20667262
:10EE40006F6D20656570726F6D00000072656164A2
:10EE5000696E672074696D6573657276657220648A
:10EE60006174612066726F6D20656570726F6D00F0
:10EE700072656164696E67206E6967687420746981
:10EE80006D6572732066726F6D20656570726F6D4F
:10EE90000000000072656164696E672074656D70C2
:10EEA00020636F6E66696775726174696F6E206644
:10EEB000726F6D20656570726F6D000065657072B0
:10EEC0006F6D206973206F66666C696E6500000067
:10EED0007570646174696E6720454550524F4D20CE
:10EEE000746F2076657273696F6E203078253038C4
:10EEF000780D0A0077726974696E6720766572739F
:10EF0000696F6E20746F20454550524F4D206661E9
:10EF1000696C65640000000077726974696E67202F
:10EF2000495220636F64657320746F2045455052C9
:10EF30004F4D206661696C656400000077726974EA
:10EF4000696E6720636F6E66696720746F20454540
:10EF500050524F4D206661696C6564007772697428
:10EF6000696E672074696D65736572766572206479
:10EF700061746120746F20454550524F4D20666189
:10EF8000696C65640000000077726974696E6720BF
:10EF90006E696768742074696D65206461746120AE
:10EFA000746F20454550524F4D206661696C656411
:10EFB0000000000063616C6C696E67204952206C30
:10EFC0006561726E2066756E6374696F6E00000015
:10EFD0007573657220627574746F6E2070726573DC
:10EFE0007365643A20636F6E6669677572696E67F0
:10EFF0002065737038323636206173206163636533
:10F00000737320706F696E7400000000776F726414
:10F01000636C6F636B000000313233343536373840
:10F0200039300000636F6D6D616E643A20736574F2
:10F0300020646973706C617920636F6C6F727320E8
:10F04000746F2025642025642025640D0A000000CB
:10F05000636F6D6D616E643A2073657420616D62DB
:10F06000696C6967687420636F6C6F727320746F6A
:10F070002025642025642025640D0A00636F6D6DD2
:10F08000616E643A2073657420706F776572202515
:10F0900073000000636F6D6D616E643A2073657478
:10F0A00020646973706C6179206D6F646520746F82
:10F0B0002025640D0A000000636F6D6D616E643A77
:10F0C0002073657420616D62696C69676874206D76
:10F0D0006F646520746F2025640D0A00636F6D6D89
:10F0E000616E643A2073657420616E696D61746944
:10F0F0006F6E206D6F646520746F2025640D0A00AB
:10F10000636F6D6D616E643A2073657420636F6C1C
:10F110006F7220616E696D6174696F6E206D6F64CE
:10F120006520746F2025640D0A000000636F6D6D0B
:10F13000616E643A2073686F772074656D706572D4
:10F140006174757265000000636F6D6D616E643A85
:10F150002073657420646973706C617920627269D0
:10F160006768746E65737320746F2025642C206447
:10F17000697361626C65206175746D6F6D6174692E
:10F1800063206272696768746E65737320636F6E63
:10F1900074726F6C20706572204C44520D0A00002E
:10F1A000636F6D6D616E643A2073657420616D628A
:10F1B000696C69676874206272696768746E6573E8
:10F1C0007320746F2025640D0A000000636F6D6D5D
:10F1D000616E643A20656E61626C65206175746F62
:10F1E0006D61746963206272696768746E657373B8
:10F1F00020636F6E74726F6C00000000636F6D6D42
:10F20000616E643A2064697361626C652061757433
:10F210006F6D61746963206272696768746E65738B
:10F220007320636F6E74726F6C000000636F6D6D9E
:10F23000616E643A2073657420646973706C6179DF
:10F2400020666C61677320746F20307825303278C7
:10F2500000000000636F6D6D616E643A207374612D
:10F26000727420646973706C6179207465737400C2
:10F27000636F6D6D616E643A207365742074696D9F
:10F280006520746F202573202534642D2530326469
:10F290002D2530326420253032643A253032643AEC
:10F2A000253032640D0A0000636F6D6D616E643A43
:10F2B000207374617274206E65742074696D6520AA
:10F2C0007265717565737400636F6D6D616E643A1C
:10F2D000206C6561726E20495220636F6465730013
:10F2E000636F6D6D616E643A207361766520646949
:10F2F00073706C61792073657474696E6773000054
:10F30000636F6D6D616E643A207072696E74207403
:10F3100069636B65723A2027257327006C64723A23
:10F32000206F6C64206272696768746E65733A203E
:10F330002564206E6577206272696768746E6573F4
:10F34000733A2025640D0A00657370383236362012
:10F350006E6F772075700000657370383236362016
:10F360006E6F77206F6E6C696E65000020204950CB
:10F370002025730064636637373A202573202534CF
:10F38000642D253032642D253032642025303264DE
:10F390003A253032643A253032640D0A000000000C
:10F3A00072656164207274633A2025732025346489
:10F3B0002D253032642D2530326420253032643AD8
:10F3C000253032643A253032640D0A00466F756E7E
:10F3D000642054696D65723A20257320617420257C
:10F3E0003032643A253032640D0A0000676F7420B1
:10F3F00074656D70657261747572652066726F6D8B
:10F4000020445331387878783A20256425730D0AE2
:10F4100000000000676F742074656D706572617420
:10F420007572652066726F6D205254433A202564D0
:10F4300025730D0A000000006E6F2074656D706505
:10F4400072617475726520617661696C61626C6568
:10F450000000000075706461746520646973706CED
:10F460006179000049524D503A20504F5745522083
:10F470006B65790049524D503A204F4B206B6579AE
:10F480000000000049524D503A2064656372656D7A
:10F49000656E7420646973706C6179206D6F64654A
:10F4A0000000000049524D503A20696E6372656D4C
:10F4B000656E7420646973706C6179206D6F64652A
:10F4C0000000000049524D503A2064656372656D3A
:10F4D000656E7420616E696D6174696F6E206D6F09
:10F4E0006465000049524D503A20696E6372656D43
:10F4F000656E7420616E696D6174696F6E206D6FE9
:10F500006465000049524D503A2064656372656D30
:10F51000656E7420686F75720000000049524D508E
:10F520003A20696E6372656D656E7420686F7572DE
:10F530000000000049524D503A2064656372656DC9
:10F54000656E74206D696E757465000049524D508A
:10F550003A20696E6372656D656E74206D696E75B3
:10F560007465000049524D503A2064656372656DC0
:10F57000656E7420726564206272696768746E6576
:10F580007373000049524D503A20696E6372656D85
:10F59000656E7420726564206272696768746E6556
:10F5A0007373000049524D503A2064656372656D73
:10F5B000656E7420677265656E2062726967687433
:10F5C0006E6573730000000049524D503A20696E19
:10F5D0006372656D656E7420677265656E20627218
:10F5E000696768746E6573730000000049524D507E
:10F5F0003A2064656372656D656E7420626C756532
:10F60000206272696768746E6573730049524D5069
:10F610003A20696E6372656D656E7420626C756503
:10F62000206272696768746E6573730049524D5049
:10F630003A2064656372656D656E742062726967F5
:10F6400068746E657373000049524D503A20696EBC
:10F650006372656D656E74206272696768746E6549
:10F660007373000049524D503A20676574207465E9
:10F670006D7065726174757265000000706F7765FA
:10F68000725F696E697428292063616C6C6564001F
:10F69000737769746368696E6720706F776572202D
:10F6A0006F6E0000737769746368696E6720706FAE
:10F6B000776572206F666600202067657420746528
:10F6C0006D70657261747572650000002020706F46
:10F6D000776572206F66662F6F6E000020206F6B5B
:10F6E00000000000202064656372656D656E742003
:10F6F000646973706C6179206D6F6465000000004F
:10F700002020696E6372656D656E74206469737024
:10F710006C6179206D6F64650000000020206465D5
:10F720006372656D656E7420616E696D6174696F79
:10F730006E206D6F646500002020696E6372656DD8
:10F74000656E7420616E696D6174696F6E206D6F96
:10F7500064650000202064656372656D656E7420C9
:10F76000686F7572000000002020696E6372656D1D
:10F77000656E7420686F757200000000202064655B
:10F780006372656D656E74206D696E7574650000D9
:10F790002020696E6372656D656E74206D696E758B
:10F7A00074650000202064656372656D656E742069
:10F7B000726564206272696768746E6573730000B5
:10F7C0002020696E6372656D656E742072656420B9
:10F7D0006272696768746E657373000020206465E7
:10F7E0006372656D656E7420677265656E20627206
:10F7F000696768746E657373000000002020696E8D
:10F800006372656D656E7420677265656E206272E5
:10F81000696768746E65737300000000202064657A
:10F820006372656D656E7420626C756520627269C5
:10F830006768746E657373002020696E6372656D0E
:10F84000656E7420626C7565206272696768746E9B
:10F8500065737300202064656372656D656E742046
:10F86000676C6F62616C206272696768746E657341
:10F87000730000002020696E6372656D656E7420F0
:10F88000676C6F62616C206272696768746E657321
:10F89000730000002020746F67676C6520617574C9
:10F8A0006F206272696768746E6573730000000090
:10F8B00020205468616E6B20796F75210000000074
:10F8C0003139322E35332E3130332E313033000082
:10F8D0004E65772074696D657A6F6E653A20256490
:10F8E0000D0A000043000000F80100201F00000086
:10F8F0001C0000001F0000001E0000001F00000090
:10F900001E0000001F0000001F0000001E0000007D
:10F910001F0000001E0000001F0000001F0000006C
:10F920001D0000001F0000001E0000001F0000005E
:10F930001E0000001F0000001F0000001E0000004D
:10F940001F0000001E0000001F0000006D010000ED
:10F950006E010000232D302B2000686C4C00656682
:10F960006745464700303132333435363738394110
:10F970004243444546003031323334353637383926
:10F980006162636465660000202020202020202022
:10F99000202828282828202020202020202020203F
:10F9A000202020202020202088101010101010105F
:10F9B00010101010101010100404040404040404A7
:10F9C0000404101010101010104141414141410138
:10F9D0000101010101010101010101010101010117
:10F9E0000101011010101010104242424242420226
:10F9F00002020202020202020202020202020202E7
:10FA00000202021010101020000000000000000090
:10FA100000000000000000000000000000000000E6
:10FA200000000000000000000000000000000000D6
:10FA300000000000000000000000000000000000C6
:10FA400000000000000000000000000000000000B6
:10FA500000000000000000000000000000000000A6
:10FA60000000000000000000000000000000000096
:10FA70000000000000000000000000000000000086
:0CFA80000000000000000000000000007A
:08FA8C00B406FF7F0100000039
:10FA9400FCBC0008E4BC000800BD000804BD00086C
:10FAA40008BD0008F4BC0008F8BC0008FF00000012
:10FAB400FF000000E8030000010000009CC20008F1
:10FAC400000000000000000000000000D0E4000876
:10FAD400000000000000000000000000A4C20008B4
:10FAE40000000000000000000000000040C2000808
:10FAF40004000000040000000100000020000000D9
:10FB0400200000000300000038C20008B50F000800
:10FB140002000000020000000000000048C20008CB
:10FB24002910000804000000040000000300000085
:10FB340050C20008E51A000802000000020000009C
:10FB44000300000058C200089918000802000000D1
:10FB5400020000000300000060C200080D0C000851
:10FB640002000000020000000000000068C200085B
:10FB7400D11D000802000000020000000300000084
:10FB840070C20008E9170008040000000400000027
:10FB9400030000007CC200082D16000802000000CB
:10FBA400020000000300000084C2000829210008AC
:10FBB4000200000002000000030000008CC20008E4
:10FBC40055140008020000000200000003000000B9
:10FBD40094C20008D51200080400000004000000CC
:10FBE400030000000F0000002000000001000000DE
:10FBF40020000000160000003C00000038C200088D
:10FC040001000000010000000000000040C20008E4
:10FC140004000000040000000100000005000000D2
:10FC2400010000000F00000005000000FFFF0000BD
:10FC3400FFFF0000D80E0000FF000000FF000000DE
:10FC4400FFFFFFFFFF000000010000003139322EEA
:10FC540035332E3130332E313033000000000000B4
:10FC64000204060800000000010203040102030468
:10FC74000607080900000000000000000102030458
:10FC84000607080900A24A04000000000000000062
:10FC94000000000000000000000000000000000060
:10FCA4000000000000000000E4F80008000000006C
:10FCB4000000000000000000000000000000000040
:10FCC4000000000000000000000000000000000030
:10FCD4000000000000000000000000000000000020
:10FCE4000000000000000000F801002087F900086F
:10FCF40001000000000000004A00000000000000B5
:10FD040000000000000000000000000000000000EF
:10FD1400000000004A000000000000000000000095
:10FD240000000000000000000000000000000000CF
:08FD340011010008ED000008B8
:0400000508000000EF
:00000001FF
